:020000021000EC
:10F000000000012039F5010061F5010063F5010000
:10F0100065F5010067F5010069F5010000000000D9
:10F020000000000000000000000000006BF501007F
:10F030006DF50100000000006FF50100C9BB030081
:10F04000654C020073F50100A14F0200C54C02009F
:10F05000194D0200396002000D51020073F50100E4
:10F0600073F5010009BC030073F5010073F501009D
:10F0700073F50100755A020073F5010073F5010084
:10F08000131504002D28020073F5010073F501002B
:10F09000352902005DD703002919020073F501002C
:10F0A00073F5010073F5010073F501009962020028
:10F0B00073F5010073F5010000000000000000007E
:10F0C00073F5010073F5010073F5010073F501009C
:10F0D00073F50100415C020073F5010000000000BF
:10F0E0000000000000000000000000000000000020
:10F0F0000000000000000000000000000000000010
:10F1000000000000000000000000000000000000FF
:10F1100000000000000000000000000000000000EF
:10F4000010B5054C237833B9044B13B10448AFF35E
:10F4100000800123237010BD402D0020000000005B
:10F420001067060008B5034B1BB103490348AFF34F
:10F43000008008BD00000000442D00201067060079
:10F44000154B002B08BF134B9D46A3F5803A0021B6
:10F450008B460F461348144A121A00F063F80F4BFC
:10F46000002B00D098470E4B002B00D0984700206F
:10F47000002104000D000D48002802D00C48AFF315
:10F48000008000F02BF82000290024F0EDFE00F0B1
:10F4900011F800BF0000080000000120000000007B
:10F4A00000000000402D002048CF00200000000098
:10F4B0000000000008B5074B044613B10021AFF36C
:10F4C0000080054B1868836A03B19847204600F016
:10F4D00031F800BF000000003CB4050070B50D4DD0
:10F4E0000D4C641BA4100026A64209D10B4D0C4CF8
:10F4F0003BF098FF641BA4100026A64205D170BD06
:10F5000055F8043B98470136EEE755F8043B984719
:10F510000136F2E7182D0020182D0020182D0020AC
:10F520001C2D002002440346934200D1704703F88B
:10F53000011BF9E7FEE700BF0649074A074B9B1A84
:10F5400003DD043BC858D050FBDC06F079FCFFF724
:10F5500077FF00001C670600402C0020402D002093
:10F56000FEE7FEE7FEE7FEE7FEE7FEE7FEE7FEE773
:10F57000FEE7FEE71FB501238DF80030054B8DF83F
:10F58000080001916846D3E90012904705B05DF884
:10F5900004FB00BFD8BA002061DF704748DF704726
:10F5A00010B50388012B11D8094A02EB03124388D6
:10F5B0005189CC1A032C09D4C3F57F43FD330B4486
:10F5C0005381002303804380184610BD0420FCE7CC
:10F5D000E0BF002010B5124A0B6802EB0010426831
:10F5E00073B15888033003EB800302F580524FF665
:10F5F000FF749A4202D91868013004D1002009E052
:10F6000002F10803F1E79888A04204D0188810B1ED
:10F610000B60012010BD5888033003EB8003E8E73E
:10F62000E0BF002073B5436804460D4613B31E4A7D
:10F6300011688B421ED3526893421BD813F003000B
:10F6400018D11A4A21891289914213D121689A68E6
:10F6500091420FD1164A5268934201D80A2004E021
:10F6600002F580529342F9D22880B0FA80F0400926
:10F6700002B070BD00232B801E46019601A9288888
:10F68000FFF7A8FF30B92B8801339BB22B80002BEA
:10F69000F3D0EDE7019B226899689142EED1636057
:10F6A000024B1B892381E3E7202D00209CBC002016
:10F6B000E0BF0020033083B240F2FD32934230B508
:10F6C0000ED909200BE0228965892A441A4492B296
:10F6D000B2F5806F08D2088062891344638130BD1F
:10F6E000024C20780028EED00720F8E7E0BF002089
:10F6F00010B50A494A788C78531CDBB29C4208BF8B
:10F7000000230C789C421FBF0370486802EB420242
:10F7100000EBC20008BF002010BD00BF5CBF00208E
:10F72000AADF7047A9DF7047A7DF704785DF704702
:10F730007FDF70477EDF7047084A30B500230C2416
:10F7400004FB03F18D5A854202D10A44508830BD32
:10F750000133082BF4D14FF6FF70F8E706BC002008
:10F760006EDF704758B1CB0801F00701C25C01237E
:10F7700003FA01F10A4214BF184600207047012025
:10F780007047000070B50A4E3468054654B1706881
:10F7900060B1FF2D08D02946FFF7E4FF30B1F368D0
:10F7A00003FB0544204670BD0024FBE70446F9E74F
:10F7B00064C10020012804D0043804288CBF002034
:10F7C000012070478378013B072B07D8DFE803F05F
:10F7D0000706060606070409142303807047012361
:10F7E000FBE743689B8809339B08F6E770B5054D36
:10F7F0000646002455F8043B304601349847052C52
:10F80000F8D170BD6CB60500114BF0B5002214267E
:10F810001D4606FB02F4E75A874212D12344142600
:10F8200000249A788A420AD001342246072A0BD84B
:10F8300006FB02F3EF5A874208D1EB18F1D11846C4
:10F84000F0BD0132082AE4D10023F8E70132EDE7E8
:10F8500074C1002030B5072185B0FFF7D5FF0446FD
:10F8600000283AD04568002D39D1007CFFF78AFF87
:10F870000721CDE902558DF80A1040B3E3680390E3
:10F8800003EB83031B019BB29B0802A8ADF8083071
:10F89000FFF798FF9DF80A00FFF78CFFD8B1114BD6
:10F8A0001B789B0715D5BDF808500DF106012846B9
:10F8B000FFF700FF48B9BDF80630A380E5800A4B8A
:10F8C000185C092803D005B030BD0928F7D90320FA
:10F8D000F9E70220F3E70846F5E70520F3E7002003
:10F8E000F1E700BF99BC002058B4050038B54FF6C9
:10F8F000FF73984218BF01300D4614BF84B2002434
:10F90000FF2C03D94FF6FF74204638BD2146284608
:10F91000FFF728FF0028F7D10134A4B2F0E7000078
:10F92000F8B5074D074E074600243378A34200DCA4
:10F93000F8BD55F8043B384698470134F5E700BF59
:10F9400078BC002029BE00207DDF704779DF70473A
:10F950006DDF704738B5074C051E04F1080318BF6A
:10F960001C4623682BB11A6822605B6828469847BA
:10F97000F7E738BDB0BB002040DF70473FDF70477E
:10F9800037B5D0F818350A7DDBB28DF807300B7F1C
:10F990009A4282BF0A699DF80740D4540B7F0D7BC1
:10F9A0000133DBB25A1C95420B7705D98B689B5CFF
:10F9B000C0F81C3501200AE00C7D944201D9CB7EB1
:10F9C000F6E7AB42F6D3A3422CBF0020012003B0E0
:10F9D00030BD0023435082B043580193019B02B0D5
:10F9E00070472DE9F0470D789DF820609DF824A020
:10F9F00004460F469946002D60D1D0F8243192F884
:10FA000000809BB14FF49271FFF7E3FF0123636124
:10FA10003B70B04550D1D4F80431002B4CD04FF49A
:10FA200082712046FFF7D5FF00251DE0D0F81C317C
:10FA3000FBB14FF48E71FFF7CCFFD0F824311BB12E
:10FA40004FF492712046DFE713789E4207D919F8E8
:10FA50000330C0F81C35137801331370D9E7012344
:10FA6000BAF1000F03D0C3612846BDE8F0874361B7
:10FA7000CFE7D0F80831002BCBD04FF48471FFF7DB
:10FA8000A8FFD0F82431002BDAD113789E42C0D9D8
:10FA9000D0F8181509F8031013780133DBB213708E
:10FAA000721E934205D10223C0F800320123236263
:10FAB000AFE79E42FAD1ACE70125D5E74FF492714A
:10FAC000FFF787FF4FF48E71FFF783FF4FF48471C8
:10FAD000FFF77FFF9FE72DE9F3470C4605464FF4FC
:10FAE000827120461F469046FFF773FF4FF49271D4
:10FAF000FFF76FFF4FF48E71FFF76BFF4FF48471C8
:10FB0000FFF767FF0023012F85F8263085F82330A3
:10FB100008BF02224FF001030CBFC4F80022C4F852
:10FB20000032236223602E6846BB05F1260A05F1E8
:10FB30002309CDE900764346524649462046FFF761
:10FB400050FF0028F5D195F82330EBB1D4F8C43438
:10FB5000C4F8C434C3B113F0010F14BF4FF4024012
:10FB6000032048F2012213F0020F18BF104613F0D1
:10FB7000040F48F2022318BF184606E040F286231D
:10FB8000AB60AB68C4F80433002002B0BDE8F08776
:10FB90002DE9F3470C4605464FF4827120461F4677
:10FBA00016469DF82880FFF714FF4FF49271FFF777
:10FBB00010FF4FF48E71FFF70CFF4FF48471FFF7C5
:10FBC00008FF0023C4F8003285F8263085F823307A
:10FBD00001232362A36095F82620974232D9B35CB3
:10FBE000C4F81C3595F82630013385F826302B688B
:10FBF0007BBB05F1260A05F12309CDE900783346E0
:10FC0000524649462046FFF7ECFE0028F5D195F80C
:10FC1000233023B3D4F8C434C4F8C434FBB113F094
:10FC2000010F14BF4FF40240032048F2012213F0E9
:10FC3000020F18BF104613F0040F48F2022318BF3A
:10FC400018460DE0B8F1000F01D0E361CFE7636122
:10FC5000CDE740F28623AB60AB68C4F804330020E4
:10FC600002B0BDE8F0872DE9F04793F9005090B05D
:10FC70000024013D6E46AD002746A446A0465FF035
:10FC8000000E03E05FEA080EBEEB050EB8EB0E09AE
:10FC900052F809A051F80E90A9FB0A9A14EB090436
:10FCA00057EB0A075CF1000C1EF1040EAE4501DCB7
:10FCB000C645EBDD46F808403C4667465FF0000C61
:10FCC00018F10408A845DADDB8EB450FDADD46F88F
:10FCD0000840D3F8B0303146984710B0BDE8F087FF
:10FCE00013460A46FFF7BFBFF0B5154689B01C465C
:10FCF00007460E461A4629466846FFF7F1FF234697
:10FD00006A4639463846FFF7AEFF23462A4669461B
:10FD10006846FFF7A8FF23466A4631463046FFF79C
:10FD2000A2FF09B0F0BD00EB81010023884200D39F
:10FD3000704751F8042D43EA52030B60D307F5E7EF
:10FD400010B5013A52B2130601D5002010BD50F88B
:10FD5000224051F822309C4205D802F1FF32F2D203
:10FD60004FF0FF30F2E70120F0E710B500235CB25E
:10FD7000A24200DC10BD51F8234040F8234001337B
:10FD8000F5E7013910B549B2041D0A06CBB204D417
:10FD9000013954F82120002AF7D001335BB273B146
:10FDA00003F18042013A50F82220002022B9013BA1
:10FDB00000EB431318B210BD52080130F6E71846A5
:10FDC000F9E7002310B51C465AB2914200DC10BD81
:10FDD00040F823400133F7E7000000000000000076
:10FDE000C3F10803DB0070B50133002403A500BF95
:10FDF0005B1920C940CAAD1B20C0184720C940CAA2
:10FE0000B54120C020C940CAB54120C020C940CA60
:10FE1000B54120C020C940CAB54120C020C940CA50
:10FE2000B54120C020C940CAB54120C020C940CA40
:10FE3000B54120C06441B4FA84F0400970BD00BFF0
:10FE4000C3F10803DB0070B50133002403A500BF34
:10FE50005B1920C940CAAD1920C0184720C940CA43
:10FE6000754120C020C940CA754120C020C940CA80
:10FE7000754120C020C940CA754120C020C940CA70
:10FE8000754120C020C940CA754120C020C940CA60
:10FE9000754120C06441204670BD00BFF0B5082206
:10FEA00089B00C460646FFF760FFCB6A03930B6BE5
:10FEB00004934B6B05938B6B0693CB6B07930027D7
:10FEC00008236A4669466846CDE901770097FFF73F
:10FED000B7FF082305466A4631463046FFF7B0FFB4
:10FEE000236B0393636B0493A36B0593E36B05444C
:10FEF000CDE906376A46082369466846FFF7A0FF42
:10FF0000082305446A4631463046FFF799FF236AC5
:10FF10000093636A0193A36A0293A36B0693E36B56
:10FF20000793054408236A4631463046CDE90477F5
:10FF30000397FFF785FF636A0093A36AA26B01939F
:10FF4000E36A02930492636BE26B0393CDE90523AA
:10FF5000236A0793054408236A4631463046FFF773
:10FF60006FFFE36A0093236B0193636B0293236A31
:10FF70000693A36A0793054408236A463146304630
:10FF8000CDE904770397FFF72BFF236B0093636B97
:10FF90000193A36B0293E36B0393636A0693E36A93
:10FFA00007932D1A08236A4631463046CDE9047777
:10FFB000FFF716FF636B0093A36B0193E36B029350
:10FFC000236A0393636A0493A36ACDE90537236B1D
:10FFD00007932D1A08236A4631463046FFF700FF83
:10FFE000A36B0093E36BCDE90137636A0393A36AC4
:10FFF0000493E36ACDE90537636B07932D1A082351
:020000022000DC
:100000006A4631463046FFF7EBFE2D1A0D4C0FD4F1
:1000100035B9082231462046FFF792FE01280FD05D
:100020000823224631463046FFF7DAFE2D1AEFE765
:100030000823224631463046FFF702FF2D18F7D439
:1000400009B0F0BD68B405002DE9F04391B00F464A
:100050001C220021804609A8FFF764FA01251C2212
:10006000002101A80895FFF75DFA394608AA11F9A1
:10007000046B009533461046FFF7E2FE314608A8B0
:10008000FFF77FFE013804B2012C07DC32466946D7
:100090004046FFF76AFE11B0BDE8F0833A46684675
:1000A0006946FFF71DFE10AB601103EB80001FFADD
:1000B00084F909F01F0350F8202C05FA03F31342CA
:1000C00005D03B46424669466846FFF7CCFD09F13C
:1000D000FF3424B2D8E770B5036813F00105064673
:1000E000144605D013460A460146FFF7A9FE054609
:1000F00021463046FFF717FE45B104F18042013A30
:1001000056F8223043F0004346F8223070BD70B5F7
:100110009DF910401E4623460546FFF761FE38B1A3
:100120002346324629462846BDE87040FFF788BE80
:1001300070BD2DE9F0438BB01446129D15F9046B88
:1001400000961F46804689462B460246214602A855
:10015000FFF7DDFF02A9129A0846FFF7C1FD129BC7
:1001600002AA41464046FFF77EFD129B02AA2146A5
:100170002046FFF778FD2B464A463946384600961A
:10018000FFF7C5FF129A394602A8FFF7A9FD02A999
:100190002B46424608460096FFF7B9FF02A92B46B8
:1001A000224608460096FFF7B2FF2B4642462146FC
:1001B00020460096FFF7ABFF129B22464946484671
:1001C000FFF751FD2B4602AA414620460096FFF755
:1001D0009EFF129B224639463846FFF744FD2B46C8
:1001E0004A46394638460096FFF791FF324602A943
:1001F0002046FFF7BAFD0BB0BDE8F08370B59DF95E
:1002000010401E4623460546FFF71AFE30B9224627
:1002100029463046FFF794FD012807D02346324691
:1002200029462846BDE87040FFF7DABD70BD2DE9CC
:10023000F0439BB01646229C14F9045B0095984647
:100240000746894623460246314612A8FFF75FFF5C
:1002500012A9229A0846FFF743FD229B12AA3946AB
:100260003846FFF700FD229B12AA31463046FFF7C1
:10027000FAFC23464A46414612A80095FFF7BEFF06
:1002800023464A46414640460095FFF740FF234635
:100290003A4631460AA80095FFF739FF229B0AAA81
:1002A00049464846FFF7DFFC2346324639460AA84E
:1002B0000095FFF7A3FF229A41463046FFF710FD55
:1002C00023460AAA314630460095FFF720FF234611
:1002D0003246394602A80095FFF719FF229B02AA71
:1002E00041464046FFF7BFFC23464A46414640464A
:1002F0000095FFF70CFF229A12A902A8FFF7F0FC65
:1003000002A923460AAA08460095FFF700FF2346E4
:100310003A4602A90AA80095FFF7F9FE0AA9229B0E
:1003200012AA0846FFF79FFC23464A460AA94846F8
:100330000095FFF7ECFE2A4602A93846FFF715FDA7
:100340001BB0BDE8F0832DE9F04115468AB00446A4
:1003500088461C22002103A8FFF7E4F82E1D95F91A
:10036000007003232A46414620460293FFF7B8FC5B
:10037000334602AA214620460097FFF7C8FE2B46C7
:10038000424621462046FFF76EFC0097334605F1B2
:10039000840221462046FFF731FF0AB0BDE8F08114
:1003A0000C4B1B78062B10D10B4B1B681A070CD17A
:1003B0000A4B186800F0F003302B08D000F0E00082
:1003C000A0F1400358425841704700207047012077
:1003D000704700BFE00F00F0E40F00F0E80F00F0FE
:1003E000094B1B78062B0CD1084B1B681A0708D148
:1003F000074B186800F0F000A0F130035842584154
:1004000070470020704700BFE00F00F0E40F00F0DD
:10041000E80F00F010B9024B01221A60704700BFCC
:100420000050004010B50C494A6E042A044611D011
:100430000B6E1344032B02F101024A6688BF043B92
:10044000182202FB031318460021FFF76BF8206007
:10045000012010BD0020FCE780C0002010B504463C
:1004600086B01422002101A8FFF75CF86088ADF87F
:100470000800FFF761F92378ADF80600092B0CD8C6
:10048000DFE803F005051014161B1D0E1F210723BE
:100490008DF8043008238DF80C3001A8FFF740FADE
:1004A00006B010BD0D238DF80430F6E70E23FAE7F1
:1004B00007238DF804300523EDE70F23F3E710231E
:1004C000F1E70523EFE706238DF80430A3680393D3
:1004D000A388ADF80630E0E708B5134644F2010200
:1004E000904203BF5A6819889868002218F00AFEE3
:1004F00030B50B4B1B68012293F8641021338A42FC
:1005000004DB405CB0FA80F0400930BD13F8014BC9
:10051000855CA54201D10132F1E70020F5E700BF7B
:100520002CBA002070B5244B0022C3F80025234AC2
:10053000516831B12249C3F8081322490420C1F897
:100540008000D3F80C55D3F81445D3F80815D3F828
:1005500010054FF0FF36B542C3F8146518BF05F516
:10056000E075C3F80C65C3F80865C3F810651EBFD5
:100570004FF0A043022643F82560651C1FBF4FF0D3
:10058000A04304F5E074022543F82450441C1FBF27
:1005900000F5E0704FF0A043022443F820404B1CCC
:1005A0001FBF4FF0A04301F5E071022043F8210086
:1005B0000023D376536070BD00200040D8BA0020DD
:1005C0008402020000E100E02DE9F04F85B08A4688
:1005D0000390039C257828462CF06BFF0746D8B97A
:1005E0002D2D1CD10134012303940193DDF80CB0AF
:1005F000BAF1000F01D0CAF800B00022114603A8DA
:100600002CF0FFFE8046002835D1614D00242046A5
:10061000294605B0BDE8F08F01340394D9E72B2DAE
:1006200004BF013403940190E0E7184602932CF0D4
:10063000D3FEB0F10009029B20DBC8451EDD404619
:100640003AF01AF922462B463AF080F904460D4654
:1006500048463AF011F922462B4639F0C1FF0136DF
:1006600004460D460396039E3378002BDDD1B8F186
:100670000A0F37D113E000240025F4E7B8F10A0F80
:1006800030D12E2B0BD10FF20019D9E90089013698
:100690000396039E30783038C3B2092B39D9039BB7
:1006A0001A7802F0DF02452A1CD15A1C03925A78AC
:1006B0002D2A01D02B2A05D12D3A574203F10203EE
:1006C000574103934FF000080A20039A1378303BF8
:1006D000D9B2092936D9002F39D12E4F0026B8F1C9
:1006E000000F46D1039BBAF1000F01D0CAF80030C9
:1006F0009B458AD09BF800202E2A03D10BF1010BD9
:100700005B4582D0019B002B81D005F100431D4643
:100710007DE73AF0B1F842464B463AF017F9024607
:100720000B462046294639F05BFF002204460D4661
:1007300040464946174B3AF033FA0136804689461F
:100740000396A6E7013200FB08380392BDE7114F7C
:10075000C8F100080026B8F1000FC3D02046294692
:1007600032463B463AF01CFA08F1010804460D46B1
:10077000F1E72046294632463B463AF0E7F808F1D1
:10078000FF3804460D46AAE79A9999999999B93F75
:100790000000F87F0000244070B58AB00C46014686
:1007A00068461D4631F0F8FB0022214605A831F0CD
:1007B000F3FB684631F0C9F8044605A831F0C5F8E6
:1007C0008442064621D0039850B1C389A3F5007333
:1007D0009BB2C381C38903F4F0530BB932F0A8F87C
:1007E000089850B1C389A3F500739BB2C381C38934
:1007F00003F4F0530BB932F09BF8002C01DB002E10
:1008000000DAF5B9A01B0AB070BD002C1BDA039802
:1008100050B1C389A3F500739BB2C381C38903F4AC
:10082000F0530BB932F084F8089850B1C389A3F59E
:1008300000739BB2C381C48914F4F05401D132F027
:1008400077F80020DFE7684631F028F905A831F095
:1008500025F9AEE7044A138A9BB223F0410343F023
:1008600040031382704700BF682D002030B587B069
:100870000A46014601A831F08FFB0025DDE901326F
:10088000934205F1010401D2013514D1049850B10D
:10089000C389A3F500739BB2C381C38903F4F053EA
:1008A0000BB932F045F8202029F0CEF814F1FF34CE
:1008B0000DD207B030BD059810B1C05C0A28E5D054
:1008C00029F0C2F801A8254631F0E8F8D6E708205B
:1008D000EAE730B587B00D46019009B100230B60FF
:1008E0000021102202A8FEF71DFE02A9019835F092
:1008F00083FEE0B10024029B039A23F07F4303337D
:1009000023F00303013203F110030AD11C44002237
:1009100002A901A835F0AAFE0028ECD1204607B0B4
:1009200030BD002DF3D02A6813442B60EFE7044656
:10093000F4E730B587B04FF4D8240021102202A884
:100940000194FEF7EFFD02A9204635F055FE70B187
:10095000002202A901A8DDE9015435F087FE002834
:10096000F6D124F07F4413352C4424F00304C4F55D
:10097000EC2007B030BD2DE9F04F89B0D51C0193B4
:1009800025F00305002382468B4617461035039356
:10099000984604AC039E86B3304635F031FE80465F
:1009A000039835F053FE064678B1039BC21A954270
:1009B0000BD9FB1A0344984507D9B5F5007F04D23B
:1009C000214635F019FE00B90396019B039947EAC9
:1009D000036710224FF0FF33204605930497CDE9BB
:1009E00006AB19F069FE129B23B194E80F00129C2C
:1009F00084E80F00039E103638E04FF4D8230393A9
:100A0000B1462146039835F0F7FD78B1059B0133D7
:100A100006D1DDE906235B4504BF5245DDF80C90A5
:100A20000122214603A835F021FEEEE7039835F0B8
:100A3000E7FD85421ED9039835F008FE0123039097
:100A40000398C8B9B9F1000F0BD02146484635F0DC
:100A5000D3FD0422002309EB020105A8059319F038
:100A60002BFE039878B9B8F1000F11D0304609B0C9
:100A7000BDE8F08F0023E3E7002BC2D135F0C0FDC5
:100A80008542BED8DEE735F0BBFD8742EBD881E773
:100A900035F012FF80460028E8D00023039379E761
:100AA0002DE9F04F8DB002AFB3F10009C7E90201A3
:100AB00092463E6D4FF0000519DBAE4217DB07F1A1
:100AC000100110463D6132F0F7FD804600BB5046F4
:100AD00033F0F6FF044638612BF098FC04F5807380
:100AE000834209D95A4901202CF014F800252846E0
:100AF0002C37BD46BDE8F08FE31D23F00703ADEBB7
:100B0000030D0DF1080822464146504633F0C8FF58
:100B100006B93E6907F1180B5A46D7E9020135F0CC
:100B2000D0FD044620B9B9F1000F2FD04949DAE7CA
:100B3000B9F1000F35D1BB691A0E05D1B34203D10B
:100B4000314635F017FE60BBBD6925F07F439E42FC
:100B50001CD12D0E1AD1D7F810A0564516D1331F2F
:100B600010E062597A619D428CBFAAEB0502042213
:100B700008EB050107F114007B603AF0EDFB28B9A2
:100B80007B680435AA45ECD80125B0E7CDF800B064
:100B900000233246D7E90201FFF7EDFE04460028A4
:100BA000C4D03969BB6909EB010223F07F439A4243
:100BB00001D9294997E74C44204635F0DBFD05462D
:100BC00020B9264901202BF0A5FF90E714F003007F
:100BD0001FD0A4EB0009C0F10406D9F800307B61F6
:100BE0003B699E4228BF1E4607F114031844324653
:100BF00041463AF0BFFB0422494607F1140019F0C0
:100C00005BFD3B69B3427FF672AFB04434449E1B38
:100C10003E613A6902F00306921B3A611AB121461D
:100C2000404619F049FD002E3FF461AF39690C448C
:100C3000324623687B61414407F114003AF09AFB85
:100C40000422214607F1140019F036FD4FE700BFDA
:100C500025B505004CB505006AB5050086B505004B
:100C60000C4A002330B41146184640F6CA0401EB82
:100C700003151032E8819D1C0133A34222F80C5C5D
:100C8000F5D148F694430122C852034B1A8030BC78
:100C900031F012BA882D0020862D002070B586B064
:100CA00015460C460022014601A831F075F92E4682
:100CB000DDE901239A4210D3049850B1C389A3F50A
:100CC00000739BB2C381C38903F4F0530BB931F0B5
:100CD0002FFE00232370AD1B0DE07EB9049850B1A8
:100CE000C389A3F500739BB2C381C38903F4F05396
:100CF0000BB931F01DFE284606B070BD059B03B14F
:100D00009B5C04F8013B01A830F0C8FE013ECFE730
:100D100037B50123009300231A460A49044632F0EE
:100D2000DFF805465CB1E389A3F500739BB2E3816C
:100D3000E38903F4F05313B9204631F0F9FD284656
:100D400003B030BD61B60500F8B5858907460C468D
:100D500095B31A4B013D03EB05152846EB8903F5C6
:100D600000739BB2EB8133F055FAEB89A3F5007366
:100D70009BB2EB81EB8903F4F053461C13B9284670
:100D800031F0D6FD304631F078FD214632F032FEAA
:100D9000044680B10146384633F000FBE389A3F5F1
:100DA00000739BB2E381E38903F4F05313B9204647
:100DB00031F0BEFD701CF8BD0126E3E7882D002050
:100DC00038B5074C25780023EDB20246194623704A
:100DD00034F0BEFF25700348BDE8384027F068BDF9
:100DE000842D0020A331060070B5044631F0AEFA20
:100DF0000546B0B120460022184933F0C5FC044630
:100E000031F064F878B900255CB1E389A3F500738B
:100E10009BB2E381E38903F4F05313B9204631F028
:100E200087FD284670BD00220D49204633F0ACFCFA
:100E300006460028E7D00B492BF04EFAF389A3F5BC
:100E400000739BB2F381F38903F4F0530546002B42
:100E5000DAD1304631F06CFDD6E700BF50B6050060
:100E6000A4FC05005AB60500002370B50B600546CA
:100E70000E4631F081FB044610B90025284670BDAE
:100E8000294632F053FC054668B9E389A3F500739F
:100E90009BB2E381E38903F4F053002BEDD12046AC
:100EA00031F046FDEAE7204631F06EF83060E38924
:100EB000A3F500739BB2E381E38903F4F053002BA5
:100EC000DCD1ECE72DE9F341002400F47F671546FF
:100ED0001470A7F54072502A0E4600F4704312D8E1
:100EE000484A11F0100F484908BF1146002B79D02D
:100EF000B3F5805F78D0B3F5005F444C18BF002491
:100F00004FF440784BE0A7F50072202A0DD8002B53
:100F10006CD0B3F5805F6BD0B3F5005F3C4C18BF6D
:100F200000244FF400783B4939E0A7F52072302ABD
:100F30000AD8002B5ED0B3F5805F374C18BF002471
:100F40004FF4207835492AE0B7F5C07F09D1002B4E
:100F500052D0B3F5805F324C18BF0024B8463149F7
:100F60001DE0A7F11002B2F5887F47D844F643028E
:100F7000ADF80020C3F302321B0402F1310248BF76
:100F80004E2329494CBF8DF804408DF803408DF85D
:100F9000022048BF8DF803306C464FF01008F00770
:100FA00003D50F2228463AF027FAB2070BD5284678
:100FB0003AF01AFAA7EB08073F11012229180A2371
:100FC000B8182BF057FB54B1330708D528463AF030
:100FD0000BFA2146C0F10F0228463AF00DFA02B092
:100FE000BDE8F081114C8BE7114C89E7114C98E773
:100FF000114C96E7114CA3E7114CAFE7A0461149FD
:10100000CDE700BFB6B50500AFB505009DFE0500F4
:10101000D5B50500D5F50500E1B50500DDB5050040
:10102000C0B50500C4B50500BCB505001AF505003E
:10103000C8B50500CBB50500D0B50500D9B505008C
:10104000E5B50500A4310600F0B54FF0805302204D
:10105000D3F85014D3F85424284BC3F80403284879
:10106000C3F80403274B93F800E093F801C09F787E
:10107000DE781D795C7998794EEA0C033B43334363
:101080002B4323430343204B2AD083F800E083F80B
:1010900001C09F701E715D719C71D8711D789C7824
:1010A0005A785E79586885EA0401514081F08801D8
:1010B000D970197971409E797140DE797140197249
:1010C00012020321597242EA05420C4B2243C3F833
:1010D000942500BA4422C3F89005C3F8A025F0BDBA
:1010E000080A1970090C9970110A1A715971110CBA
:1010F000120E58709971DA71D0E700BF00500040AD
:101100008000080054BF00203FBF002038B50022F7
:10111000054633F039FB044698B100231A460146D0
:10112000284627F069FAE389A3F500739BB2E381AF
:10113000E38903F4F05323B92046BDE8384031F089
:10114000F7BB38BD70B5EFF3108672B60D4A9468E0
:101150000123A4B993600C4B0C4DD3F880102940A7
:101160001160C3F88050D3F8841051604FF0FF3203
:10117000C3F88420047006B962B6002070BD037005
:10118000F9E700BF24C2002000E100E0FC06FFBC3C
:1011900038B50BF093FA0446D8B10F4DB5F90000FD
:1011A00031F06BFB0D490246204633F0B4FAB5F935
:1011B000020031F062FB0A490246204633F0ABFAE6
:1011C000B5F9040031F059FB06490246204633F0D8
:1011D000A2FA204638BD00BF14C200200208060053
:1011E000CB0806006C0A060010B588B012788DF89E
:1011F0000C20CDE90001FF22002102918DF80D2085
:1012000001214FF6FF72104C8DF81C10ADF80E2026
:101210008DF8103026F0C6FD70B12BF0EFF858B9FC
:1012200014F1FF34F6D2094904202BF073FC684610
:1012300026F0C8FD08B010BD002CF4D02BF0DEF86D
:101240000028F0D1F3E700BF80841E0037B6050008
:101250002DE9F341314C637E0546002B5BD12368B9
:101260000BB10123637695E80F002D4E86E80F0041
:10127000A27E637F2B4E23F00303FF2A63771EBFFA
:10128000012393404FF0A0424FF0000118BFC2F875
:101290000C35254B21770422C3F8082331603168CF
:1012A00000910099297939B32A681278C3F81C256E
:1012B0002A79012A22D92A685278C3F81C25256880
:1012C0000DBB194FDFF85480D7F80831002BFBD045
:1012D00035603368019341463846019BFEF750FB69
:1012E0000028F1D1A27EFF2A12D0012393404FF0B3
:1012F000A042C2F808350BE0E27ED7E72A7B012A3C
:10130000DDD9E27ED9E7084B0422C3F8042300208C
:1013100002B0BDE8F0811120FAE700BF1CBB00203D
:1013200024BB0020083100400030004037B50B01DD
:101330005BB249B2044643EA01008DF804001A4D3D
:1013400050B20343120152B28DF805302B7811438D
:1013500002438DF806108DF8072013B302AB03EBA0
:10136000941302AA13F8040CC4F30113134413F8E2
:10137000043C43EA002019F011F92B788BB102AA42
:10138000C4F3810304F003041344144413F8040C5D
:1013900014F8043C43EA002003B0BDE8304019F0E3
:1013A000FDB803B030BD00BF32C20020C30914BF76
:1013B00013020B0270B510F0400F0D460CBF29460A
:1013C0001146194306461220144619F071FAB10667
:1013D0004CBF23022B0216F0100F14BF21462946E2
:1013E0001943122019F064FA32074CBF23022B0272
:1013F00016F0040F14BF214629461943122019F094
:1014000057FAB3074CBF2102290216F0010F08BF9B
:101410002C4621431220BDE8704019F049BA000063
:1014200010B5074A002332F8024B8C4203D1184111
:1014300000F0010010BD0133082BF4D10020F9E7C2
:1014400034BA0020F0B5224B9F7C1C4600221D467A
:10145000D6B2B7420ED895F878701D4C0022D6B29D
:10146000B74216D895F8DE500022D4B2A54220D853
:1014700000200DE0B4F814C0844502F1010204F12B
:101480000A04E5D142F64D2301200B808870CE700E
:10149000F0BDB4F87AC0604502F1010204F10A041B
:1014A000DDD142F64D230B8002238B70CE700120DC
:1014B000EEE7B3F8E060B04202F1010203F10A0383
:1014C000D3D142F64D230B8003238B70CC70EEE713
:1014D000A8BC002010B50C4C226886B0034682B12F
:1014E00004208DF804000868D989ADF80C10123377
:1014F00033F8021C0290ADF80E10049301A92046A7
:10150000904706B010BD00BFA8BC00207FB54B8936
:10151000022B0FD1094A136863B1097B006802905E
:1015200011F0010F14BF022103218DF804101046A1
:1015300001A9984707B05DF804FB00BFA8BC0020D4
:1015400070B50D4D002435F8026B964210D1012282
:10155000A240D2B2D543EDB2014410F8014B2BB1F9
:101560001443884200F8014CF7D170BD2C40F8E7D5
:101570000134082CE7D1F8E734BA002070B5002315
:10158000084C1A4641FA02F5ED0706D504EB42066F
:1015900000EB4305B688AE8001330132082AF1D151
:1015A000036070BD30BA002010B586B0044600223A
:1015B000684616F079F82046009916F0A3F92046FF
:1015C00006B010BD38B501230B7004460D4630F04F
:1015D0007DFC88B100220B49204633F0D5F810B1CC
:1015E00033F07FFF287020460022074933F0CCF803
:1015F000BDE8384033F0B8BD2046BDE8384032F091
:1016000009BE00BF18B505001DB50500084B5A6E90
:10161000013A5A6622B907490A7822F002020A7092
:101620001A6E0132042A08BF00221A66704700BFF2
:1016300080C000209ABC002030B5044685B00D461D
:10164000102200216846FDF76DFF237A012B0AD096
:10165000022B0ED063680193236829469B68684675
:10166000984705B030BD23690293A38AADF80C30CA
:10167000F0E70123A2898DF80030E389ADF80A2054
:10168000D31AADF80830E5E728DF704729DF704747
:1016900038B51C4B5A6E19465AB31C6E182202FB01
:1016A00004331A7A012A07D0022A23D018460921C6
:1016B000BDE83840FFF7C0BF1825D88A9A8A05FBD5
:1016C0000414D4E90314121AB2F5806F4FEA8000B3
:1016D0000144B4BF92B24FF480622044FFF7D6FFBA
:1016E00011280BD1084A137823F0020343F00403B6
:1016F000137038BD9889FFF7C7FFF1E70028F8D0CD
:10170000D4E700BF80C000209ABC0020054A1378AF
:1017100013F0060F04D143F002031370FFF7B8BFB4
:10172000704700BF9ABC00202DE9F3411F4B1B7886
:101730001746DA07064688462BD51D4D1D4B9D42A0
:1017400029D31D4B9D4226D239B330B341EA000361
:101750009B0724D12B68984223D36A6800EB870348
:101760009A421ED3FFB101A8FEF75CFE78B1019B3F
:101770000024C3E90054019B01221A72C3E90386C5
:101780009F82FFF7C3FF204602B0BDE8F08107202B
:10179000FAE70120F8E70220F6E70320F4E7062045
:1017A000F2E70520F0E70420EEE700BF9ABC002036
:1017B000202D0020202D0020302D002038B5074B93
:1017C000074A5968948810684A880332032592B200
:1017D00000EB84001D70FFF7A7FF38BD9CBC002004
:1017E00024C1002010B501220C460649FFF79CFFDA
:1017F00028B9054901EB041101238B7310BD0E209C
:10180000FCE700BF80B60500E0BF002008B502225B
:101810000149FFF789FF08BD84B6050008B5034BF1
:10182000034918680222FFF77FFF08BD24C100208A
:101830008CB6050073B51B4B1B78DB0705462BD513
:10184000194E1A4B9E4229D3194B9E4226D238B3C9
:10185000C0F30B04D4B93368984219D3726800F509
:1018600080539A4214D301A8FEF7DCFD90B1019B8E
:10187000C3E90064019B02221A722D0B01229D8193
:101880001A82FFF743FF204602B070BD0620FBE737
:101890000520F9E70720F7E70120F5E70220F3E745
:1018A0000320F1E79ABC0020202D0020202D0020ED
:1018B000302D002010B50B4C0B4B628803EB02134C
:1018C0009A892AB95868FFF7B5FF0423237010BD21
:1018D00005232370054B022218689A80FFF7AAFFA0
:1018E000F5E700BF9CBC0020E0BF002024C1002021
:1018F00008B5074B191D5888FDF76CFE18B1BDE8F7
:101900000840FFF75BBFBDE80840FFF7D3BF00BF4B
:101910009CBC002060DF704710DF7047002208B5D4
:10192000114617F0EFFB00002DE9F347254B1B682C
:101930001BB1984730B3FFF7F1FF234B1B7803F03F
:10194000FF07FBB1214D224E2C68DFF88C90B4FAD2
:1019500084F46409B0463378A3B901A8FDF71EFEEC
:10196000052812D00028E6D1019B0BB9FDF7F2FF44
:10197000184B1B680BB1019898474CB10124EAE75A
:10198000002CFBD002B0BDE8F087002CFAD13C4619
:10199000DFF848A098F80030002BF3D1B9F80030F8
:1019A000ADF80430DAF8003001A91846FDF7F4FD6F
:1019B0000528E5D00028BED12A6818469047002C9B
:1019C000E8D1C8E788BC002021C1002068BA002007
:1019D00022C100202CC1002064BA00201CC20020BB
:1019E00010B5084B9A685AB150B9EFF3108172B62E
:1019F000054A1C6814605C685460986001B962B65E
:101A0000002010BD24C2002000E100E02DE9F341D8
:101A10001D4F7B6806460D469BB304292FD94369A9
:101A20007BB3437C0024012B0DF107000CBF8846DB
:101A3000A0468DF80740FFF785FB0DF10600FDF786
:101A400057FED0B101230370104B4660D3F8043524
:101A5000C0E90484C0E902359DF806307B709DF82A
:101A60000700FFF7BDFF24B9094B4FF48012C3F8FC
:101A70000021204602B0BDE8F0810424EFE70724EE
:101A8000F7E70824F5E700BF5CBF00200010014025
:101A900000E100E02DE9F341CE0801F007044FF02A
:101AA000010808FA04F4855DE4B22540074613D125
:101AB0000DF107008DF80750FFF744FBBB5D9DF863
:101AC00007001C4202BF1C43BC554546FFF788FF78
:101AD000284602B0BDE8F0810025F9E72DE9F3477B
:101AE0008146002701261FFA87F84FEAD80A08F036
:101AF000070406FA04F419F80A50E4B2254008D0A5
:101B00000137B7F5807FEED1B846404602B0BDE858
:101B1000F0870DF107008DF80750FFF713FB19F858
:101B20000A309DF807001C4202BF1C4309F80A4016
:101B30000125FFF755FF002DE2D0E6E773B5054616
:101B4000B8B1C1F3C70401F0070301269E40035D4D
:101B500033420ED000230DF107008DF80730FFF758
:101B6000F1FA2B5D9DF8070023EA06062E55FFF7D4
:101B700037FF02B070BD000038B50A4B1A687AB161
:101B80005D686DB1FF280BD084B221462846FDF771
:101B9000E9FD28B121462846BDE83840FFF7CEBF11
:101BA00038BD00BF64C100202DE9F74F9846531E91
:101BB000072B81460F46154600F2BB80FF2800F236
:101BC000B88001465E48FDF7CDFD0646002800F0CE
:101BD000B08039464846FDF717FE044600283ED03F
:101BE000C3689D4247D805D25FFA85F9E368207C37
:101BF000994543D394F81090B9F1FF0F40F09780C6
:101C0000504B1A689B46002A41D14FF6FF73238040
:101C1000A3700023C4E90133E360238A03F478430B
:101C200043F0FF032382112084E0237C1844C0B2D8
:101C3000FFF7A2FFE3685FFA8AF083420AF1010A24
:101C4000F3D84FF6FF732380A3700023C4E9013358
:101C5000E360238A03F4784343F0FF032382FF21E8
:101C60004FF6FF70FDF7D0FD04460028DBD0A0F84A
:101C700000908770BEE74FF0000ADBE74844C0B22F
:101C800009F10109FFF778FF5FFA89F9AEE75B68B0
:101C9000002BBAD00023DBF808205FFA83FA9245C4
:101CA00002D34FF0FF0912E0DBF8040060B35146A5
:101CB0000193FFF7EFFE019B30B3B9F1FF0F08BFAF
:101CC000D146AAEB090A0AF1010AAA4521D1B9F1C4
:101CD000FF0F84F8109098D0E560207CFDF752FD4E
:101CE00058B305EB85052D01ADB2AD0888F802703B
:101CF000C8F80400A8F8005026B1082F02D1AD00A2
:101D0000063D8580002015E0B9F1FF0F0CD14FF0A2
:101D1000FF090133BFE74846019309F10109FFF7C5
:101D20002BFF019B5FFA89F9D145F4D3EFE7002639
:101D3000D2E7072003B0BDE8F08F0320FAE700BF29
:101D400038C0002064C1002038B504460025E3688F
:101D5000AB420ED84FF6FF732380A3700023C4E973
:101D60000133E360238A03F4784343F0FF032382C3
:101D700038BD207C2844C0B2FFF7FEFE0135E6E7FF
:101D800037B5FDF741FD0546A0B144682CB10A4BBB
:101D900001941B789B0706D403242846FFF7D4FF41
:101DA000204603B030BD01A8FDF7FAFB0446002829
:101DB000F3D0F1E70524F3E799BC0020FF2810B524
:101DC000044609D801460548FFF7B8FE21460448F5
:101DD000BDE81040FFF7B2BE10BD00BF38C0002004
:101DE00058C0002013B50DF106010446FDF71AFC9A
:101DF00070B1BDF80620084B03EB02139A894AB173
:101E0000A17A39B1013A00209A81A07202B010BDC6
:101E10000A20FBE70620F9E7E0BF002037B50D46B2
:101E20000DF106010446FDF7FDFB88B1BDF8062063
:101E3000084B616803EB021300209A8901329A81F2
:101E4000296063680C336B600123A37203B030BD5B
:101E50000A20FBE7E0BF00202DE9F043DFF8848093
:101E6000D8F874E0BEF1030F0F46944635D81C4EE7
:101E7000756CC1F108039D422FD8D8F870407444A6
:101E80001C2304F00304814603FB0484B9E80F001B
:101E90000FC499E807000EF1010384E80700C8F8B1
:101EA0007430C7B1336C2B4403F0070306EBC30354
:101EB000002206F138040CEBC20103C9A34202F16F
:101EC000010283E8030014BF0833054B9742F2D1A7
:101ED000736C1F447764012000E00020BDE8F083AC
:101EE00060BB002064BF00202DE9F0411C46184B68
:101EF0001B789B0706460F46154627D5DFF8588006
:101F0000A3880BB10A201FE098F800302BB92146B6
:101F1000A088FDF75FFB20B92060A3880133A38070
:101F2000EEE723681EB1998832889142EFD11FB144
:101F300019883A889142EAD19B682B6023686B60CC
:101F4000044B1B892B810020BDE8F0810220FBE7B8
:101F500099BC00209CBC0020E0BF002030B587B0B9
:101F60004CF2070305460C46ADF8043003AA0F4BAC
:101F700001A90020FFF7B8FF10B1002007B030BD65
:101F800001A903A8FFF74AFF0028F6D10723A37091
:101F9000019B5A882280029A62609B8803F58043E5
:101FA0002B8003A8FFF71EFF0120E7E78CBC002071
:101FB0001FB50023A0F58040A1F58041CDE9023393
:101FC000ADF80400ADF8061002AB0DF1060101A852
:101FD000FFF78AFF002818BF052005B05DF804FB55
:101FE0002DE9F04102230B80164B00251C6800F5FB
:101FF000805E2F4608304FF6FF7870450AD305B152
:102000001C6002B11770BDE8F08101270EE0344674
:1020100001250BE006680136F1D086884645F4D0EC
:102020000688002EF1D08668A642F0D8468806F1D0
:10203000030C00EB8C00B1F800C00CF1030C6644FB
:102040000E80DAE724BE002070B5064D0646002457
:1020500055F8043B0BB1304698470134082CF7D1B2
:1020600070BD00BF3CBB00202DE9F047AA4C266F95
:102070001C2707FB06F586B0635D013B8046052BF8
:1020800000F22A81DFE813F00600640064001D01FD
:102090001D017E0130B1A14A137823F001031370B2
:1020A00001201FE025442B79032B15D8DFE803F02E
:1020B00002072C34FFF7B2FB01232B7109E0984D86
:1020C0002B78022B40F03C826868FFF79FFB0023CF
:1020D0002B70002800F0F080904A137823F0010361
:1020E00013700E201C237343E218E35C0290023B42
:1020F000012B00F232818B4B907D196C5A6C01449C
:10210000121A19645A6428E1874F3868FFF792FB66
:102110000223BB800023D0E7834FDFF804823868B6
:10212000FFF774FB814BD7F800E05B88B7F804C079
:102130001B0108EB03025168A2F808C0C2F804E0D2
:102140000222BA800022396008F803202A71C0E711
:1021500007FB0647724BB7F812A04FEA0A1A03EBC7
:102160000A029946118960B1FB8803F1030888448B
:10217000C3F57F435189A2F80880FD330B44538196
:102180008EE7536803EB81083B7C062B00F29780B7
:10219000DFE803F02D733C4D1F84040041F61D5011
:1021A0001C2303FB0643D144DB88B9F80810DA1C72
:1021B0000A44A9F80820C3F57F43B9F80A20FD3383
:1021C0001344A9F80A3041F61D53984200F0C38029
:1021D00088E757485749002343601C2303FB064305
:1021E0009B690360FDF71EFA002800F04C81291D51
:1021F000012221444046FFF797FA1C2303FB0643C4
:1022000002221A74002857D00E20C9E705F10C01EC
:102210000122214408F10800FFF786FA1C2303FB82
:1022200006439A7D002A14BF03220122E9E73D4BB1
:102230005A6C002A00F08C81196C1C2505FB0645A0
:10224000481C00F0070003EBC1071864A88A53F884
:102250003110013A5A6408EB8000BA88FFF764FA3B
:10226000AB8ABA881344AB82AB7D013BDBB2AB7562
:10227000002BC7D101232B74C4E705F1080101220B
:10228000214408F10400FFF74FFA1C237343E25C7A
:10229000032A0CBF052206222344B2E7254B1988E6
:1022A000234B5868FFF79EFA1C2303FB06430622C4
:1022B0001A7400287FF474AF06B0BDE8F0870F20D1
:1022C0006EE700287FF4ECAE07FB06473B79012B55
:1022D00032D01BB1022B3ED00F2003E7CDE9020024
:1022E000FB6801930DF1020101A8FDF79BF980B194
:1022F0000298BDF802108388FB8003883B81FFF7BA
:1023000071FA1C2303FB064302221A710028D3D062
:1023100059E70A20F5E700BF64BF002099BC002000
:10232000E0BF002060BB002024C100209CBC002036
:102330005C2D002030C20020864FA81D3B4601AA1C
:1023400041462044FFF7D0FDB8B9B9880298FFF79D
:1023500049FA0A28DAD1002302931C2303FB06F270
:10236000A25C013A052A00F2B580DFE812F08E0087
:102370009200A000CB00D500E1000A28C7E9008840
:10238000E9D020E700287FF48BAE734BDA7AAAB14C
:10239000D8721A78013A062A9ED801A151F822F083
:1023A000512402004B240200612402006724020031
:1023B000D92202006D2402007D2402001A78072A27
:1023C000E7D801A151F822F0E9230200932302008B
:1023D000932302000524020019240200372402007E
:1023E00037240200012402001A8901321A810022D6
:1023F0005A80DA72594A1278B2FA82F252099A7203
:10240000012207E0564958688A884088033202440E
:102410008A8002221A70BCE75D88504A504902EB5C
:1024200005120868556850608888108102228A80E9
:102430000D600622EEE70722ECE7484900229A7277
:102440008A8942B9897B31B15A80FFF751FA5DE739
:102450009A7A002AF1D100221A705A805A607AE7DB
:10246000FFF7ACF952E7FFF725FA4FE75A883B4BE5
:1024700003EB02135868FFF7C9F947E700225A60D7
:10248000FFF7CCF942E70A202CE600238DF8043050
:1024900020E003FB064301228DF804201A89ADF8E1
:1024A00010209A88ADF81220DB68039312E003FB3A
:1024B000064302228DF804201A89ADF810209A886C
:1024C000ADF81220DA681B7C03929A1F53425341E5
:1024D0008DF8143001A8FFF7B7FD206F1C220021F2
:1024E00002FB0040FDF71EF8636F1BB3226F013241
:1024F00002F00302013B22676367DBB10020FFF7B4
:10250000B3FDD9E603FB064303228DF80420DA88E5
:10251000ADF810201A89C5E703FB06430422DB88C7
:10252000ADF8103000238DF80420ADF81230D1E75B
:102530000523ABE70B4A137823F004031370BBE6C3
:10254000084A137843F0020323F00103137002E7F3
:102550001368FFDE38C200209CBC0020E0BF0020D2
:1025600024C1002099BC00200846FFF77DBD000073
:10257000054A137813F0040004D143F004031370E8
:10258000FFF772BD704700BF99BC0020F0B51C4634
:102590003D4B1B789E0789B007460D466FD50988CD
:1025A0004FF6FF7399426CD06B88002B69D0696835
:1025B000B5F808C000239C4503D8BAB916460431C3
:1025C0000AE051F83300800757D10133F3E731F8BF
:1025D0003200304486B201329445F8D80DF1020140
:1025E0003046FDF767F828B109B0F0BD138856886A
:1025F000ADF8023000238DF81430BDF80230ADF88C
:1026000016300323ADF81830204B8DF804401A68BB
:1026100029898DF81A1001321A602B88ADF80C3018
:10262000032C6B88ADF8083004BF04238DF81430F8
:10263000049208BF3B686A6808BF0793002401A89A
:10264000ADF80A60ADF80E40FFF706FC50B9BDF8D2
:1026500002200F4B03EB021358890338801B58816B
:102660000820C1E7049B3B600A4B7C601B89BC725D
:102670003B81FFF77DFF2046B6E70320B4E7022049
:10268000B2E70420B0E700BF99BC002024BE0020C0
:10269000E0BF00209CBC002030B58BB0FF28044672
:1026A00001921D4645D88B781846FDF783F800281F
:1026B0003FD04A6802920A88ADF80C20A4F5804207
:1026C000ADF81C20A3F58042ADF81E2002AA0892A6
:1026D0000122ADF82420194604AA2046FFF768FC21
:1026E0000528019A0ED1022352B907A904A8FFF7C1
:1026F0004DFF07281FD010D8B0B103200BB030BD5C
:1027000001AAF2E732B10E4B1B789B0702D501A854
:10271000FCF746FF03230022E7E708280DD00E2828
:102720000CBF11200320E9E7002DE7D0049B2B60AC
:10273000E4E70720E2E78620E0E71120DEE700BFBC
:1027400099BC00201F4B204A1B6800BF00BF00BF80
:1027500000BF00BF00BF00BF00BF93422FD000BF2B
:1027600000BF00BF00BF00BF00BF00BF00BF00BF71
:1027700000BF00BF00BF00BF00BF00BF00BF00BF61
:1027800000BF00BF00BF00BF00BF00BF00BF00BF51
:1027900000BF00BF00BF00BF00BF00BF00BF00BF41
:1027A00000BF00BF00BF00BF00BF00BF00BF00BF31
:1027B00000BF00BF00BF00BF00BF00BF00BF0138A7
:1027C000C3D17047A42C00200024F40073B5154E2B
:1027D000736805461BB343690BB3002404740DF101
:1027E00007008DF80740FEF7ADFC0DF10600FCF781
:1027F0007FFF90B1022303709DF80630456073702F
:102800009DF80700FFF7ECF824B9074B4FF480124E
:10281000C3F80021204602B070BD0424F0E708246C
:10282000F8E700BF5CBF002000E100E02DE9F843BD
:102830002649274B0025C1F84051C1F84451C1F841
:102840004851C1F84C51C1F80051C1F804511B68FE
:10285000002B39D0D1F804451E49DFF88C80096877
:10286000641A24F07F442F461A68A24217D8A41A8B
:1028700015441A7CDE6982B1D8F800901F74D3E940
:102880000521B9F1000F06D01046C84728B1FFF75F
:1028900045F83346E8E708469047002EF9D10E4A3E
:1028A0000E4B11781B788B4205D10133DBB2022B22
:1028B00008BF002313701278094B43F82250094BCC
:1028C0004FF48012C3F80021BDE8F88300100140E6
:1028D00020C200203CC1002039C1002038C10020A6
:1028E00030C1002000E100E084BC00200D4B0E4907
:1028F0004FF4003210B5C3F8802001244FF4803328
:10290000C1F848332F20C1F808334C60FFF71AFF95
:10291000064B8C602F2000211960FFF713FF044B3A
:10292000197010BD00E100E0001001403CC1002022
:1029300019C100202DE9F04FB64AB749137809783C
:10294000B64D85B09942D5F80080019500F095808C
:102950000133DBB2022B08BF002313701278B04B97
:1029600053F82260019A08EB060323F07F431360BB
:102970000127AC4BAC4A18680290AC48117890F82B
:1029800000904FF0000CE2465078884278D1BCF1BC
:10299000000F02D0A54981F80090002F40F0BB80C5
:1029A0001F6802997F1A18BF012700201968029139
:1029B0009E49039191F800E000244FF0010800289F
:1029C00040F0AD8092F80190D2F804C092F802A0D5
:1029D0001178494540F0C1801B68029A9A4201D1A2
:1029E000002F44D0002B00F01281D3F80090904CBF
:1029F000019BD4F8046519688E4F751A3B7825F051
:102A00007F450335A3B94FF48033C4F84433C4F889
:102A10000433894B4FF400324FF00108C3F8802192
:102A20002F201A60C4F80080FFF78CFE87F8008022
:102A3000A9452CBF4944491921F07F41C4F84015EC
:102A4000D4F804359B1B23F07F43891B033321F00B
:102A50007F418B420BD9D4F80435C4F840352F2080
:102A6000FFF770FE744B4FF40032C3F80021039A55
:102A70000023137005B0BDE8F08F0026374678E7D5
:102A800001EB4104506892F802B000EBC40E013132
:102A900010F834401868C9B28B4508BF0021022CD9
:102AA00004D0032C7FF470AF002410E0DEF804B0F3
:102AB00004468646002C3FF467AFA34500F0C08073
:102AC000A646E469F6E780F810A0C0690124002852
:102AD000F9D1002C3FF458AF186055E7D4F80C90AA
:102AE000C4F800E0761A8C44E1691960B9F1000F6E
:102AF00007D008EB0C0121F07F41C4E90119E06126
:102B000020461C68002C3FF451AF2168B142E5D942
:102B10008E1B26604AE7002084468646F1E7014680
:102B2000C069019DD1F804A02E68444DD1F80890E9
:102B3000AAEB060C2CF07F4CAC4535D80CEB090603
:102B40000E60D3F800C081F81080C1E90144CC6167
:102B5000BCF1000F33D1196031E701EB410B0131BA
:102B6000C9B2514514BF117014701CF83B100129F3
:102B70000CEBCB067FF42CAF716891F810B0BBF171
:102B8000000F7FF425AFD6F808C0C1F804C0F5687F
:102B90008D603569CD6076698E61BEF1000F0CBF26
:102BA00066465E464E60BCE7A6EB0A0626F07F4608
:102BB0004E4502D2A9EB0606C2E70C60C1E7D1F888
:102BC0000090DCF80060B1451FD8A6EB0906CCF8F0
:102BD0000060C1F81CC0BEE7A9EB0A09D6F81CA02A
:102BE000B446BAF1000F0AD05646D6F800A0CA453E
:102BF000F2D3AAEB090AC6F800A0B2466646C1F8AD
:102C00000090C1F81CA0F161D9E66646EDE7FFF738
:102C10006DFE2CE738C1002039C100203CC10020E6
:102C200030C1002020C200205CBF002018C100205D
:102C30000010014019C1002000E100E0FEFF7F000C
:102C400074450FD1D0F81CB0C3F800B0BBF1000F31
:102C500008D10A4D0120A86001984FF0010CC0F87E
:102C600000B0E1462068E469CEF81C40002C3FF437
:102C70008BAE25682844206086E600BF0010014026
:102C800037B5074B054693E803006C46002384E8FC
:102C900003001A4621462846FFF7FEFC03B030BD6C
:102CA00040B40500FDF7DABB10B54FF6FF730446DC
:102CB0009C42084609D1FEF711FFB0F5807F04461B
:102CC00001D14FF6FF74204610BDFF2CF9D82146E4
:102CD000FEF7E0FE0028F6D1F3E710B5044601F058
:102CE000EFFC2046BDE8104000F02EBF1FB5037872
:102CF00093B90279072A0FD1448803932046CDE97E
:102D000001338DF80420FCF717FDADF8060001A88B
:102D1000ADF80840FFF7E1FF04B010BD1FB5002378
:102D2000CDE901330393ADF80600022301A88DF825
:102D300004308DF80810FFF7D0FF05B05DF804FBF4
:102D400086DF704738B504884CB9821C00F10A054B
:102D500012F8013B1BB99542FAD100200AE00B881A
:102D6000A342FAD108220231023038F0F5FAB0FA63
:102D700080F0400938BD08B570B171B103780A78A8
:102D8000534013F0FE0F08D106220131013038F014
:102D9000E3FAB0FA80F0400908BD0020FCE710B566
:102DA000044600F0BDFF2046BDE8104000F04ABFD9
:102DB00043DF70476FDF7047024B0022C3E90022F8
:102DC000704700BF8CBC0020F0B5FF2887B00446D8
:102DD0000E4615461F4629D80846FCF7EBFC28B3DB
:102DE00003AA2046FFF7E4F818B10524204607B0EF
:102DF000F0BD01A903A8FFF711F804460028F4D19B
:102E0000019BAE705A882A805FB13B6892009A425B
:102E10000AD30299686838F0ADFA03A8FEF7E2FF1A
:102E2000E4E7029B6B60F8E70424DFE70724DDE7B3
:102E30002DE9F041CEB020AE502380460CADB82233
:102E40000021304601930395FCF76CFB0DF19703CD
:102E500005930DF1AE0306930DF1C503079337AB50
:102E600008930DF1F30309930DF585730A931C4F35
:102E700004960DF221130B930024444507D1E2B2CE
:102E8000002104A8FFF796FF4EB0BDE8F081502264
:102E900000212846FCF746FB01AB02AA072137F8C0
:102EA000020BFFF791FF20F002000528ECD06B7CAD
:102EB000032B12D817230DF1310203FB04630DF12C
:102EC000450152F8040B43F8040B8A42F9D11188EA
:102ED000198092789A700134CFE743F20220D3E749
:102EE00042C100202DE9F04110220546A6B0002184
:102EF0002D48FCF717FB35B929462846FCF730FC6E
:102F000026B0BDE8F0816A0028492748DFF89C8098
:102F100004AE38F02FFA382200213046FCF702FBCD
:102F200000245023CDE9013412AF03975022002131
:102F30003846FCF7F7FA01AB02AA072138F8020B72
:102F4000FFF742FF20F002000528D9D09DF8593044
:102F5000032B26D8C4EBC402B318DDF85910B150C6
:102F60000134BDF85D209A80A5429DF85F209A71DA
:102F7000DCD10DF1170313930DF11E0314930DF122
:102F8000250315930BAB16930DF1330317930DF136
:102F90003A0318930DF1410312961993E9B238469A
:102FA000ACE743F20220ABE752C1002042C100204F
:102FB0002DE9F043037889B00546002B3FD1017914
:102FC00007293CD104AA4088FFF7FEFEB8BBFFF7F3
:102FD000F3FE02A90DF10600FEF7C0FF78B36E887C
:102FE000BDF80670BE42F4D0059C631C184611342F
:102FF00013F8012B12B9A342FAD1EAE7DDF80C80ED
:10300000102208F1010138F0A7F908F111018146F9
:103010002046FFF7B0FEB9F1000F01D00028D8D04C
:103020003046FCF789FB0023ADF81A0006A88DF89E
:103030001830ADF81C60ADF81E70FFF7B0FE09B097
:10304000BDE8F083CA1F012A73B5064654D800258F
:10305000CDE900558DF80210FCF7D6FB0446002898
:103060004CD0437CDB074BD4007CFCF78BFB10B9C6
:10307000032002B070BDE368019003EB83031B01E2
:103080009BB29B086846ADF80030FCF79BFB62687A
:1030900004F1080369463046FFF7FEFA637C03F04B
:1030A0000603062B01BF174A136803F1FF331360B1
:1030B00030B9637C23F0070343F001036374D8E75E
:1030C00011280BD10F4A136801331360637C23F07E
:1030D000060343F0040363740020CAE7862809D17D
:1030E000084A136801331360637C23F0060343F03E
:1030F0000203E3E70728BBD10720BAE70520B8E7BA
:103100002846B6E72CBE00202DE9FF4105461022D7
:1031100000216846FCF706FA68882979ADF80200B4
:103120008DF80410FCF770FB2B78454E092B5ED808
:10313000DFE803F00505684D4D6C7173757D00285F
:103140003FD0437CDC073CD5FEF7FEFD2B78581EB4
:1031500043424341002468468DF800408DF8083012
:10316000FCF744FB33684BB3364E002537464FF02F
:10317000140808FB05735B7C5A0703D49B0759D5D9
:10318000002C57D0B1783088FFF75CFF002851D071
:1031900014235D437B1986289B788DF804307A5B75
:1031A00016BF0290082309236846ADF802200CBF21
:1031B0008DF800308DF80030FCF718FB04B0BDE846
:1031C000F08101238DF80030AB68029316E080B1E6
:1031D0008268AB689A420CD1437CD90709D5326822
:1031E00023F00503013243F00403326043740024EA
:1031F000B8E702238DF80030EB6803936846FCF7CC
:10320000F5FAF4E703238DF80030F7E704238DF88F
:103210000030EB68D9E70523F5E70623F7E7072336
:1032200068468DF800300124FCF7E0FA9AE7EB6875
:103230000293DCE70135082D06F1140699D1BDE7AC
:103240002CBE002074C1002070B500238CB02D4925
:103250002C4E4FF6FF70CDE90033FCF747FB4FF6DD
:10326000FF750446AC420BD0A4F58043ADF8143092
:1032700002AA6B46002105A8FEF736FE0A2822D0D6
:10328000214B1A781846E2B94FF6FF718C4218D0DC
:103290001E4E367801251D70B607A4F580439BB2FB
:1032A0001DD58B422CD005218DF8141005A8114690
:1032B0008DF81850ADF81A30FEF7CEFD60B1FFF76B
:1032C00057F90CB070BD2046FEF778FD2046314618
:1032D000FCF70CFB0446C5E70D4B1D70F1E702231C
:1032E0000022092102708DF8141005A8FF21ADF805
:1032F00016408DF81810CDE90723FFF705FFE0E72A
:103300000423EDE758C00020F1BF002099BC002045
:10331000F2BF0020F0B5426805783D4C85B0B2FAA6
:1033200082F149090391691E0346042924D8DFE884
:1033300001F0030330496A009989DE8901F5804173
:1033400089B243F6FE77B94204D906F5804080B2CF
:10335000B84211D8012DADF802108DF8046013D1D8
:10336000002A14BF032100218DF8001003929B68EE
:1033700002936846FFF7C8FE23781BB10023237031
:10338000FFF762FF05B0F0BD002A14BF0421012140
:10339000EAE79989DD8901F5804189B243F6FE7635
:1033A000B14204D905F5804080B2B042E4D8002A89
:1033B0000CBF02220522ADF802108DF804508DF8E2
:1033C0000020D4E7988900F5804080B243F6FE7172
:1033D0008842D1D8DB89002BCED1FF23ADF8020083
:1033E0008DF804305AB906238DF80030FEF7E6FC5C
:1033F000084A002323701370FFF726FFB9E707235D
:103400008DF80030F4E708238DF80030B1E700BFF5
:10341000F2BF0020F1BF0020F8B50D490D4DFCF7BB
:1034200065FA4FF6FF760446A5F12007B44201D1B4
:103430002046F8BDFF2CFBD821462846FCF792F920
:103440000028F5D020463946FCF750FA0446EDE74F
:1034500038C0002058C0002073B5104B104C93E8C2
:1034600003006D46002385E803001A46294620889C
:10347000FFF712F94FF6FF762388B34201D01128E7
:1034800001D102B070BD1846FFF7C6FF00231A46EF
:1034900029462080FFF700F9EEE700BF48B4050099
:1034A00074BC00201FB50378012B044615D10179A7
:1034B000012912D1002302AA4088FFF785FC60B9D8
:1034C00002238DF800306388ADF80230039B684614
:1034D0001B788DF8043000F0B5FD054B1A884FF6C7
:1034E000FF739A4201D0FFF7B7FF04B010BD00BFD1
:1034F00074BC002070B504468AB0142200216846CE
:10350000FCF710F86588ADF804502846FCF714F96C
:103510002378ADF80200092B15D8DFE803F0051673
:103520003048525E8614A1A507238DF80030237918
:103530008DF808309DF80A3043F001038DF80A3009
:103540006846FCF7EDF90AB070BD07238DF800302E
:1035500023798DF808309DF80A30444AA168039118
:1035600043F001038DF80A301368002BE8D099422C
:10357000E6D1002313603E4A03931580E0E7082359
:103580008DF8003023798DF80830E3680493374BC9
:10359000A1681A680391002AD2D09142D0D135494E
:1035A00000221A600B680392013B0B60C8E70723F7
:1035B0008DF8003023798DF8083001238DF809301B
:1035C000BEE708238DF8003023798DF808300123F9
:1035D0008DF80930A3680493B2E7274D09238DF8CD
:1035E00000302B78002BABD04FF6FF70FFF714FFA5
:1035F0004FF6FF7398420646A2D12049FCF776F9B0
:10360000B04204469CD1142200210DEB0200297027
:10361000FBF788FF0B238DF81430ADF81840ADF898
:10362000164005A8FCF77CF98AE70A238DF80030DC
:10363000114BA4681A780294002A81D01422002128
:103640000DEB02001970FBF76DFF0C238DF81430A1
:103650004FF6FF73ADF81830ADF816300794E0E779
:1036600005238DF800306BE70623FAE734C000200D
:1036700020BE002070BC002076BC002058C0002076
:103680002DE9F047474B1B788AB00546002B00F028
:103690008780454B454F93E803003C7803AE86E8AE
:1036A0000300BCB94FF6FF70FFF7B6FE0123ADF87B
:1036B000143001AB06930423029305AA02AB062142
:1036C00080460194ADF81640FFF77EFB07284AD1EB
:1036D00001233B70364B1C689846002C5AD1354A62
:1036E000354F12883B68AA4241D1002B3FD01422AB
:1036F00021460DEB0200FBF715FF072328468DF846
:103700001430FCF719F80623ADF8160005A8ADF83B
:1037100018508DF81C30FCF703F920460AB0BDE8BC
:10372000F087CDF804A0019B4046A34224BFC146C8
:103730001C46FFF771FEBDF814309B00029305AAEA
:1037400002AB06218046FFF73FFB0028EBD005289F
:10375000E7D04FF6FF7398451CD1164BA3F80090A5
:10376000154B1C60B4E74FF6FF79A246EDE7013335
:103770003B6000220E4B31462846FEF78DFF0028A5
:10378000CCD00023C8F800303B68112803F1FF3388
:103790003B6001D11120C1E7862818BF0320BDE797
:1037A0000820BBE728BE002050B4050033C000202D
:1037B00034C0002020BE002070BC002063DF7047B2
:1037C000A6DF7047A2DF70472DE9F04391B098461D
:1037D00011238DF8043013788DF805300024164637
:1037E00001254FF0000365F34203074689461C227A
:1037F000214609A88DF80630FBF794FEB3788DF8C2
:103800000930C3F30302A24214BF1A2212228DF818
:10381000242001AA0E9203AB72788DF8082004933D
:10382000224602AB65F34202059308238DF80A2075
:10383000CDE9064404AAADF81C3009A943463888EE
:103840008DF80E50ADF80C900894FFF7BBFF11B047
:10385000BDE8F083A0DF7047044A0123116883406C
:103860000B401ABF1218507E1846704730BA00201D
:1038700070B4094D134601262A6806FA01F4144271
:1038800007D001F1190402463146281970BCFDF732
:1038900057BE70BC704700BF30BA00201FB5002370
:1038A000CDE9013303938DF80A201A46074BADF892
:1038B000081006241978ADF806008DF80440FFF7CB
:1038C000D7FF01A8FFF709FA04B010BDAF2C002004
:1038D00010B4084A012314688B40234006D00A44E0
:1038E0005DF8044B0146507EFDF79ABD18465DF821
:1038F000044B704730BA002010B50A4B19780446C3
:10390000FFF7E6FF58B1084B00205A88A24201D1C8
:10391000C0B210BD0130082803F10C03F5D1FF201F
:10392000F7E700BF04BC002006BC00202DE9F843E7
:103930000546FBF701FF234B07460022142098465B
:1039400000FB02F1CC5AAC422AD10B44002634468B
:103950004FF014095BB199782846FEF711FA10B1BF
:10396000052818BF032401363246072A1DD9A4B9F9
:10397000FF2D24D8144928464FF6FF75FFF794F918
:10398000FFF762FCAF4208D03846FFF7B5FFFF28CB
:1039900003D00C2343430D4AD5522046BDE8F8839B
:1039A0000132082ACCD10023D0E709FB02F338F812
:1039B0000310A94201D14344CCE70132D5E70724E3
:1039C000EBE700BF74C1002058C0002006BC0020F7
:1039D0002DE9F0411F46154B9DF818400E469046C4
:1039E00019780546FFF744FFB8F1000F17D0104BC8
:1039F0003A4619782846FFF73BFF0E4B22461978C6
:103A00002846FFF735FF44B12846FFF775FFFF282A
:103A100003D00C234343084AD652BDE8F081002C62
:103A2000FBD03046BDE8F041FFF780BFAF2C00204F
:103A3000B12C0020B02C002006BC002008B5FFF7F8
:103A40005BFFFF281DBF0C234343034A4FF6FF7063
:103A500018BFD05A08BD00BF06BC00202DE9F043B6
:103A600085B00546FFF7EAFF4FF6FF739842074619
:103A700041D001224FF0030901AB0821384602F181
:103A80000108FEF791F81FFA88F8064648BB02992C
:103A90000A46032342F8049B06312846FBF740FE02
:103AA000044660B908213846FFF7CCFA0446112CC9
:103AB0003FD01AD80CB30C2C2FD107231EE00C28B2
:103AC0000DD0052800D1344608213846FEF758F9B4
:103AD000002818BF03244246002ECDD1E7E7012677
:103AE000F2E70728E9D00446E1E7862C13D043F239
:103AF00002039C4211D100221CE0012328468DF8CC
:103B00000430ADF80850FFF799FFADF8060001A8A2
:103B1000FFF7C8F8EFE70823F0E7092328468DF8F8
:103B20000430FFF78BFFADF80850ADF806000394A2
:103B3000EDE70122034B28461978FFF799FE05B0FF
:103B4000BDE8F08396BC00200378072B02D14088A3
:103B5000FFF784BF704700002DE9F0434FF6FF7573
:103B6000A84285B0044668D0FFF768FFA84227D175
:103B700000260327B0464FF001093B463246414636
:103B80002046FBF7CFFD042805464DD0082847D036
:103B90000B282DD117F002031FD1B8F1000F20D14F
:103BA0001EBB032320468DF80430FFF747FFADF816
:103BB0000840ADF8060001A8FFF774F8002237E0CE
:103BC000002301AA0821FFF7FFF80028D0D1029BAB
:103BD00003F106089E881F68CDE701274FF0000912
:103BE000CBE703271E469846F8E703274646F5E746
:103BF000B9F1000FD5D0112819D043F20203984231
:103C0000DCD008B90223CDE7092320468DF8043023
:103C1000FFF714FFADF80840ADF806000395CAE7BA
:103C2000B9F1000FEED1BCE7B9F1000FB9D0012214
:103C3000034B20461978FFF71BFE05B0BDE8F08363
:103C400095BC002037B50578012D044614D1408875
:103C5000FFF782FF6088FFF7F1FE00236A462946DE
:103C6000FFF7B2F840B9019B1B782BB1034B60887A
:103C700019782A46FFF7FCFD03B030BD97BC002041
:103C8000F0B587B004460E461746FFF7D7FE4FF64D
:103C9000FF739842054624D01E4B20461978FFF743
:103CA00017FE80B30023CDE90033029304238DF87F
:103CB0000030194BADF802401978ADF80460204689
:103CC0008DF80670FFF704FE68B12846FFF72EFE58
:103CD000124B204600221978FFF7CAFD6846FEF70E
:103CE000FCFF07B0F0BD07212846FEF749F805287C
:103CF000EED10923049003A88DF80C30ADF80E40E6
:103D0000FEF7EBFFE4E73A4631462046FFF7C6FDF3
:103D1000E7E700BFB12C0020B02C0020AF2C002022
:103D200010B5027886B004461AB1012A09D006B04F
:103D300010BD0E4B1B78002BF9D0C088FFF7F6FDA5
:103D4000F5E70B4B40881978FFF792FD142200210C
:103D500001A8FBF7E7FB6088ADF80600FFF76EFEF1
:103D6000ADF8080001A8FBF7DBFDE0E728BE002066
:103D70006CBA002070B5044686B01422002101A858
:103D8000FBF7D0FB23786088ADF80600013B0B2BD6
:103D900000F29080DFE803F02106233A4E585C6879
:103DA000747A7C8C2679444B321C19784FF00105CB
:103DB00018BF01228DF80450FFF75AFD731B5A42B9
:103DC0005A413E4B60881978FFF752FD6088FFF733
:103DD00035FEADF80800002D42D106B070BD0223BB
:103DE0008DF804302379002B14BF012302238DF8B2
:103DF0000C30314B01221978FFF73AFD2F4B227915
:103E000019786088FFF734FD0125DFE703238DF87B
:103E100004302A4B1978FFF75BFD002814BF0123FB
:103E200002238DF80C30A3798DF81030A388ADF8FB
:103E30000E30E9E7204B1978FFF74AFD0028CCD176
:103E400002238DF80430DFE703238DF80430EAE71E
:103E50000723A2888DF80430ADF808208DF80C30C7
:103E600001A8FBF75DFDB8E708238DF80430A388AF
:103E7000ADF8083007238DF80C30A3680593EFE701
:103E800006238DF8043063680393BDE70523D8E764
:103E900003238DF80430094B1978FFF719FD00282A
:103EA00014BF012302238DF80C3041F20113BEE749
:103EB0000423C6E7002589E7F0BF00206CBA002084
:103EC0001FB50D294FF0000301930393ADF80600D1
:103ED000029108D10B2301A88DF80430FFF74AFFA7
:103EE00005B05DF804FB86290CBF0A230923F2E71D
:103EF00030B508490A680023012505FA03F4224277
:103F0000D8B202D122430A6030BD0133182BF4D15C
:103F10001846F9E730BA002010B50378182B04468C
:103F200002D1FFF7E5FF207010BD000010B5024B75
:103F3000197DFDF723FB10BD30BA00202DE9F04FAD
:103F40003D4D89B02878FFF787FC60B103A8FFF7E3
:103F5000EDFFDFF8E8A0DFF8E8B00DF11009002769
:103F6000039B9F4202D309B0BDE8F08F39F8024BA2
:103F700029782046FFF7ACFC064678B39AF8001083
:103F80002046FFF7A5FC804640BBBBF800304FF64B
:103F9000FF7219462046FBF7C7FB43F2030290422B
:103FA00029D10133ABF80030EFE7052320468DF827
:103FB0000030FFF743FDADF802006846ADF804405D
:103FC000FEF770FEB046324629782046FFF750FCD7
:103FD00042469AF800102046FFF74AFC0137BFE737
:103FE0002046FFF72BFDFEF74BFE0026EBE72046B1
:103FF000FFF7B2FDE7E70828F2D012D80028D4D0A6
:104000000628EDD00923029020468DF80030ADF847
:104010000440FFF713FDADF802006846FEF742FECC
:10402000D1E743F202039842CDD043F201439842D4
:10403000DDD01128E6D1C6E797BC002098BC00204F
:1040400034C200201FB5044640882378ADF806002E
:10405000012B10D05AB21AB1022B15D004B010BDEA
:1040600001A88DF80420FEF71DFE6088FBF764FBB5
:10407000FFF772FDF2E78DF8043001A8A388ADF8D0
:104080000830FEF70FFEE9E72379002BE6D0FBF7B7
:1040900053FB4FF6FF739842E0D0044B012219788E
:1040A000FFF7E6FBFFF74AFFD8E700BF97BC002009
:1040B00038B5074C0146207DFDF7B2F930B1A07D3F
:1040C000FDF7AEF9002814BF0220012038BD00BF63
:1040D00030BA00202DE9F0478CB08946164680465C
:1040E000FFF7E6FF20228246002104A8FBF71AFA18
:1040F000BAF1000F46D0B9F1000F17D099F800506F
:1041000015F001054FF6FF7415D04046FFF796FCF9
:10411000A042074639D14048FDF7E0FCB0F5807F6A
:1041200001D0B84275D10025032470E04D468526A4
:104130004FF6FF775FE02E4627465CE04A46314661
:104140004046FBF7F5FA0446B9F1000F5DD00028B0
:104150005DD199F8003013F0010F14BF0121022145
:104160004046FEF7DBFDB6F1850218BF01220024B0
:104170000095012339464046FFF72AFC20460CB043
:10418000BDE8F08743F20204F8E7002502AB012204
:1041900007213846FDF708FD0446002837D121469F
:1041A00050220398FBF7BEF9039B83F800A0039C01
:1041B000079604F13403049304F118030893631C75
:1041C00009934046154B0B93FFF796FBFF280CD045
:1041D000134A0C2101FB002050F8042FC4F81120D1
:1041E0008288A4F815208279E2753846FBF732FB05
:1041F000044660B90646BAF1020F04AB9ED1002214
:1042000031464046FBF794FA0446002CABD000221E
:10421000AEE707460125B9E738C00020F3BF00200C
:1042200006BC0020F0B585B00446FFF741FF324FD1
:10423000012806463D7831D12046FFF7FFFB4FF6B7
:10424000FF7398422AD0204632462946FFF710FBDA
:104250000023CDE90133039301A80C238DF804302A
:10426000ADF80640FFF786FD244B1B78E3B13978A3
:104270002046FFF72DFBB8B9214B22491A6820468A
:10428000FFF728FF8628054632D011280FD070B1DD
:1042900029462046FFF714FE05B0F0BD002229464E
:1042A0002046FFF7E5FADFE700221146E7E7A5F130
:1042B00011035E425E410022134B20461978FFF73E
:1042C000D7FA124B324619782046FFF7D1FA104B35
:1042D000002219782046FFF7CBFA0E4B00221978FE
:1042E0002046FFF7C5FA002DD6D0112DD4D0CFE748
:1042F00000260122E0E700BFAE2C00201FC10020F5
:10430000DCBF00201AC10020AD2C0020AC2C002006
:10431000AB2C0020AA2C0020F0B587B0074601A8DE
:10432000FFF704FE02AD0024019B9C4201D307B0BD
:10433000F0BD35F8026B39463046FFF7C9FA10B1C7
:104340003046FFF76FFF0134EEE700002DE9F04F34
:10435000054687B0904699460F4639B9A14B1B7860
:10436000F3B90524204607B0BDE8F08FFFF7A0FEA3
:104370000138C0B2012800F22D8100212846FBF748
:10438000D9F90446862C00F0B080112C00F09980F9
:10439000002C00F09680B9F1000F00F0BF80B9E06A
:1043A000FFF786FE012800F09E80022840F012816F
:1043B0008D490B78284613F001048B4614BF4FF04B
:1043C000010A4FF0020AFFF739FB4FF6FF739842DC
:1043D000064659463AD03B4602AA0721FEF7F4FCAE
:1043E0000446F0B9039B93F84420D10740F1C780FD
:1043F000B8F1000F40F0D68003F1340202F112014F
:104400002846FBF793F94FF0000A04460023009377
:10441000BAEB030318BF0123B4FA84F25209314600
:1044200045E00528F2D1BDE004AB0122072130466A
:10443000FDF7BAFB0446002840F0C1803046FBF788
:1044400009FA0446002800F0B280B8E0002C41D000
:104450006648FDF743FBB0F5807F834637D0B04216
:1044600036D004AB01220721FDF79EFB044650B96C
:104470005846FBF7EFF9044628B95B492846FBF795
:1044800059F9044638B107215846FDF779FC10B1B7
:10449000052818BF03244FF6FF73BBEB030318BFB7
:1044A0000123B4FA84F200935209012359462846A5
:1044B000FFF78EFA002C7FF465AF51462846FEF7D1
:1044C0002DFCA4F111035E425E4100220FE0B346D1
:1044D0000324E0E72846FBF72DF900970446012363
:1044E000B0FA80F29AE7404948E700260122404BA3
:1044F00028461978FFF7BCF93E4B32461978284612
:10450000FFF7B6F9B9F1000F08D0002C3FF42AAF3D
:10451000112C17D021462846FFF7D2FC0D2C3FF472
:1045200021AF06D8002C3FF41DAF082C18BF032480
:1045300018E7862C14D043F202039C423FF412AFDA
:10454000112C1AD12C4B3A4619782846FFF790F9CE
:104550002A4B424619782846FFF78AF9002401E7DA
:10456000254B3A4619782846FFF782F9234B4246F5
:1045700019782846FFF77CF9F4E60324F2E6B8F14F
:10458000000F0FD1598D03F1180200297FF436AFC7
:1045900003F12C01343311F8010B00287FF42EAF06
:1045A0008B42F8D19BF80030DA073FF53DAF0E495A
:1045B0002846FBF7BFF8044600283FF427AF072141
:1045C0003046FDF7DDFB00283FF420AF052818BF7B
:1045D00003241BE743F20204B9F1000F3FF4C2AE1B
:1045E00098E700BF1FC100201AC1002038C000207A
:1045F000AB2C0020AA2C0020A92C0020A82C0020E5
:104600002DE9F04786B00746FFF726F958B101A813
:10461000FFF78CFCDFF84880DFF8489002AE0025F9
:10462000019B9D4202D306B0BDE8F08736F8024BED
:1046300039462046FFF74CF980B198F80010204623
:10464000FFF746F999F8001082462046FFF740F937
:104650000123014652462046FFF778FE0135DFE789
:10466000A82C0020A92C002010B50378062B0ED909
:10467000072B1BD10E4B1C782046FFF7EDF810B12D
:104680002046FFF749FE0B4B1878FFF7B9FF0A4B9E
:104690001C782046FFF7E0F810B12046FFF73CFEFB
:1046A000064BBDE810401878FFF7AABF10BD00BF49
:1046B000AD2C0020AB2C0020AC2C0020AA2C00201C
:1046C0001FB503780446092B09D8DFE803F0050A73
:1046D00020202020202020204088FFF7A3FD04B0C8
:1046E00010BD144B197819B3134B00791B7803F0E4
:1046F0000102904206D86179C3F34003994294BF06
:1047000000210121012300226088FFF71FFE23788A
:104710008DF80430043434F8023CADF8063094E8E7
:10472000030004AB03E9030001A8FFF723FBD6E76E
:104730000121E7E71FC100201AC1002037B5174B40
:10474000174A5B881188174C174D994208D8528830
:104750009A4205D36369FBB900232B7003B030BDC7
:104760002B783BB16369002BF6D000228DF8042032
:1047700001A80FE00D490E480978D4E9012300296A
:104780000CBF11461946FDF741F90028E4D0A36992
:10479000002BE1D09847DFE70122E7E766BC002065
:1047A00078C00020C8BB00205CBB002040C10020B6
:1047B000E4BB00207BDF70477ADF704776DF70470D
:1047C00075DF704737B5164B18884FF6FF73984260
:1047D00010D0144A144D1378297B0133DBB299426F
:1047E00013702C4608D31149FFF7EAFF10B1AB69EB
:1047F00003B1984703B030BD002313702B7C33B155
:104800003B21FFF7DBFF10B1AB6903B19847636948
:10481000002BEFD000228DF8042001A8E9E700BFAB
:10482000C4BB002040C10020C8BB002078C00020CD
:1048300065DF70472DE9F74F0C9CBDF834B0278831
:10484000002580468A4691462E46B8F80020B2429E
:104850000BDC35B12288013AD21B92B2FF2A39D83B
:10486000DA55002003B0BDE8F08FD8F8042052F8E4
:104870002600019000220DF1030101A8FFF7D8FFE7
:104880000028EFD19DF803204A4521D12288002D30
:1048900014BF0020022002EB09010144594519DC34
:1048A0003DB9013292B2228003F802A0228801327F
:1048B000228022880DF103011A4401A8FFF7B8FFF6
:1048C0000028CFD121889DF803200A4422800125A9
:1048D0000136BAE70C20C5E72DE9F341089CBDF885
:1048E00024501746CDE9004502220646FFF7A2FFF5
:1048F00048B9102239463046CDE9084502B0BDE836
:10490000F041FFF797BF02B0BDE8F0812DE9FF4706
:104910000023138090F82D3006460D4614463BB315
:1049200002A8FBF715F8002840F0FB801388082246
:10493000CA54238801339BB21B222380CA54238884
:1049400001339BB2CA18DDF809102380E950BDF885
:104950000D30938023889DF8082006339BB212F017
:10496000FE0218BF01222380EA54238801332380EA
:10497000B378FBB1238804331F2B21D802A8FAF7A0
:10498000E5FF002840F0CD8023880322EA542388E5
:1049900001339BB219222380EA542388BDF80820F2
:1049A00001339BB2E9182380EA54120A4A70238823
:1049B00002332380F278AAB12388D91C1F2901D998
:1049C0000C20AEE00221E954238801339BB201217F
:1049D0002380E95423880B449BB22380EA54238824
:1049E0000B4423807268AAB12388D91C1F29E7D8F9
:1049F000022192F90020E954238801339BB20A2155
:104A00002380E954238801339BB22380EA5423880E
:104A1000013323803389002B76D1338A5BB11F2386
:104A2000CDE9004307222B46032106F11000FFF7D2
:104A300053FF002875D1338B5BB11F23CDE90043B1
:104A400015222B46142106F11800FFF745FF002818
:104A500067D1326A002A67D1776A4FB3BB88218851
:104A6000981C8A1C02441F2AAAD8FE28A8D80333FF
:104A70006B54238801339BB2FF222380EA5423889E
:104A800001339BB223803A88EA54E918120A4A702B
:104A90002088023080B22080BA884AB1B9680029E3
:104AA0004AD0284436F066FC2388BA881344238011
:104AB00096F82C30002B79D1307890B33388012BC5
:104AC0003AD023889F1C1F2F3FF67AAF012805D1CB
:104AD000727802321A441F2A3FF672AFC3F11D03E7
:104AE0009BB202A9E819ADF80830FAF72DFFC0B95A
:104AF0003278022A40F09880BDF808209A4240F2AD
:104B0000AE80ADF8083098E01F23CDE900430622BF
:104B10002B46022106F10800FFF7DEFE00283FF4D5
:104B20007CAF04B0BDE8F0872788BB1D1F2B3FF684
:104B300047AF1188052901D80720F2E76FF4486CC8
:104B400001EB0C039BB24FF27D3C6345F4D95388D3
:104B5000052BF1D96FF44860181880B26045EBD985
:104B60004FF6FF70814203D0834201D09942E3D8CF
:104B70000523EB55238801339BB212212380E9548E
:104B8000238801339BB223801188E954E818090A6D
:104B90004170238802339BB223805288EA54E9187B
:104BA000120A4A7023880233238055E7B36A002B28
:104BB000C2D04FF000084FF00C094FF0160A96F8DB
:104BC0002C305FFA88F293427FF676AFB16A09FB28
:104BD00002F28F18BB88981CFE283FF6F1AE2088A1
:104BE00003332B54238801339BB2238005F803A0A1
:104BF000238801339BB223808A5AEA54E918120AA7
:104C00004A702088023080B22080BA884AB1B968E0
:104C1000002991D0284436F0ADFB2388BA8813448C
:104C2000238008F10108CAE7012A7FF46AAF72788D
:104C30009342FFF466AFADF808200821BDF80830B4
:104C4000FE2B3FF6BDAE22880133AB5422880132E1
:104C500092B22280A95422881344238061E709215B
:104C6000ECE7000007B5144B1A686AB10020186021
:104C70001B6800934FF08042009B0123C2F8083369
:104C80000E4A5370FAF766FE0D4B1A688AB100227D
:104C90001A601B680193019B4FF080430222C3F806
:104CA0000823064B0120987003B05DF804EBFAF777
:104CB00051BE03B05DF804FB00010040A8BB00201A
:104CC0000401004013B5104B104C114800221A602B
:104CD0001B6801932146019BFAF752FE88B9A27E18
:104CE0000C48FF2A1FBF012393404FF0A042C2F897
:104CF0000835002363762371236802B0BDE81040B5
:104D0000184702B010BD00BF083100401CBB002096
:104D10000030004020BB002070B52D4C86B094F8C8
:104D20002130019394F820300093E36904F12602C6
:104D300004F123014FF04020FAF753FE2346E0B977
:104D400094F82360A56906BB217B8A1E012A1CD822
:104D5000E0692269904218D16269E37BE261C5F3A0
:104D60004015032984F8203084F8215007D100959C
:104D70004FF040212046FAF70BFF06B070BD4FF010
:104D800040212046FAF7A7FEF7E7124A07CA06AC09
:104D900004E90700C6B14FF04021D1F8C424C1F89E
:104DA000C42490070CD501228DF80820002283F836
:104DB00024206A07E1D4D3E9002102A89047DCE768
:104DC0005107F3D50222EFE78DF80860EEE700BF48
:104DD000F4BA002000BB0020F7B515464FF0FF32B3
:104DE000C1F8082390F8242004460F4602F0FF0E75
:104DF0002AB18368C1F80433112003B0F0BD012645
:104E000080F82460836100F10C0C95E807008CE8C1
:104E10000700AA7884F820206A68E2616A78C7F8F7
:104E200088252A78B24212D012B91E1C18BF01265A
:104E300084F821600096AB786A6839462046FAF714
:104E4000A7FE2368002BD8D184F82430D5E784F856
:104E500021E0AB786A6839462046FAF73CFEF0E775
:104E60000023435082B043580193019B02B0704726
:104E7000064A08B54FF492711046FFF7F1FF4FF460
:104E80008471FFF7EDFF0123136008BD002000408F
:104E900010B5CB7D0A464FF4847123B9FFF7E0FFCC
:104EA000D0F8183510BDFFF7DBFF537ED168D0F87E
:104EB0001805C854537E0133DBB25376F2E7000085
:104EC000F8B52C4C626822B12B4B4FF40171C3F83A
:104ED0000813E37D4BB1237E7BB322B1264B4FF405
:104EE0000172C3F80423112026E00122E275E0607C
:104EF0006376A27E237612B90BB9FFF7B9FF636818
:104F000073BB4FF4A2711C481B4E1A4FFFF7A8FF4A
:104F1000D6F82431D6F80821D6F8445182B90DB913
:104F2000002BF5D00022E27503BB0DBBA17E124B16
:104F3000012299B11A600020F8BD20610123D8E751
:104F4000002BEFD1002DEDD139463046FFF7A0FF01
:104F5000637EE27D9A42DBD82B46E3E75A60EAE7BC
:104F6000054B4FF40172C3F80423E4E70320E3E7A1
:104F70000F20E1E7D8BA0020002000400A4610B513
:104F80004FF48E71FFF76CFF938A91689BB2C95CF6
:104F9000938A01339BB29382C0F81C1510BD0000A8
:104FA00030B54A4AD2F8043313F4007F85B0154671
:104FB0004AD0D2F82431002B46D04FF492711046DB
:104FC000FFF74EFF4FF40173C2F80833404B997E50
:104FD00009B9012151603D4902228DF80020D1F824
:104FE0008024C1F880240392DA7D8DF80820DA68E5
:104FF00001920022DA751A766846D3E900129047CA
:105000003248D0F81C313BB1314A938A917D9942A4
:1050100047D91146FFF7B2FF2C4AD2F844318BB181
:105020004FF4A2711046FFF71BFF294B997E09B17F
:1050300001211160DA7D2AB10022DA75587ED96823
:10504000FAF798FA05B030BDD5F804335B07D7D529
:10505000D5F80831002BD3D01D4C1C482146FFF752
:1050600017FF637EE27D9A422346C9D1227E52B168
:105070002369E168E3600023607EE275237663764E
:10508000FAF778FABCE7A27E0AB901226A600F4AF1
:105090004FF40171C2F808130022DA75587ED968FE
:1050A000EEE74FF48E71FFF7DBFE917D0029B3D060
:1050B00000238DF8081091688DF8003001919375E8
:1050C0006846D2E900139847A6E700BF00200040D9
:1050D000D8BA0020800000F1A040D0F8003723F4B7
:1050E0004033C0F80037D0F8003743EA0141C0F838
:1050F0000017704700F1804000F5C040002382B0E7
:10510000036003680193019B02B070472DE9F04FE3
:1051100085B00024594D01944FF48072012102F1B1
:10512000804303F5C04390B21B68012B06D1D5F82C
:1051300004330B4202D0FFF7DDFF0C430432B2F51B
:10514000907F4FEA4101EAD14D4B1B68012B0AD1F8
:105150004FF4BE70FFF7CEFF4FF0A04344F0004481
:10516000D3F81035019314F0FF0F1AD0454F0126E4
:105170000025344210D0AB0003F1804303F5C04357
:10518000D3F81005D3F8101557F8253023B1C1F323
:105190000141C0F3042098470135082D4FEA460627
:1051A000E7D1002C63DA4FF0FF330022CDE9023261
:1051B000344D354E0024A24601274FF0A04816F981
:1051C000012B531C46D0D2B222F0C0094FEAD901BC
:1051D00004A8084402F0070310F808CC07FA03F308
:1051E0001CEA030F36D005EB090C92099CF930C07C
:1051F00055F82CB0BBF1000F0AD1032A2AD10DF1CA
:105200000C0E1EF801C04CEA030C0EF801C001E0C0
:10521000032AF4D009F5E07110F80C0C58F82110AD
:105220001842C1F3014105D0022913D1032A0BD141
:10523000114604E003290DD1032A05D10221484675
:10524000FFF748FF0134E4B2BBF1000F02D0114672
:105250004846D8470AF1010ABAF1040FAFD134B178
:105260004FF0A043019AD3F81035934202D105B014
:10527000BDE8F08F0193039B02939AE70060004022
:105280007C61004080BA0020D0BA00200028C3B260
:10529000A8BF00F160424FEA501010B5BABF0D4AE6
:1052A00003F00F0402F561424FEA41114FEA80001A
:1052B000C9B200F16040B4BF115582F8001300F587
:1052C000614003F01F0201239340C0F88031036066
:1052D00010BD00BF14ED00E02DE9F8430446C2798B
:1052E000C17A0E2023F0ACFC237B644A0BB35378C5
:1052F00043F0100353702568EB175906604B41EAE1
:10530000D51168064FF0FF328B4208BF82420AD3A4
:105310005C4A002335F062FE00F5006020F47F66F1
:1053200026F00F064EB929465748BDE8F84327F046
:1053300023BF537803F0EF03DCE7207923F0F4FB7D
:1053400040B9607923F0F0FB20B95048BDE8F8433C
:1053500027F012BF4E4F3B781BB100233B70FBF789
:10536000E1F825794B4B002228461A7023F0DCFB2C
:1053700020B14FF44071284615F0C0FD65792846EC
:1053800023F0D2FB20B14FF49851284615F0B6FD1A
:10539000637A2579002B284614BF4FF00E094FF091
:1053A000000923F0C1FB00285AD03B4B05EB8505D3
:1053B0001D4495F801806479204623F0B5FB002850
:1053C00051D0354B04EB84041C446378334CE27EAB
:1053D000002A4BD15A1C0AD04FF0A04101229A401A
:1053E000C1F8082503F5E072032041F82200B8F166
:1053F000FF3F2B4D1FBF4FF0A04108F5E07200208A
:1054000041F82200C5F82465C5F86C950026C5F85A
:105410001485C5F80C35234B636028464FF48E7114
:105420002660FFF71DFD4FF4A271FFF719FD1E4B1B
:10543000C5F8043302210846FFF728FF0423C5F806
:105440000035B8F1FF3F4FF48073E6822676638320
:1054500010D0FFF70DFD0123A37615F06DFA09E0DA
:105460004FF0FF38A7E74FF0FF33AFE708210F48B1
:1054700027F062FE01233B70BDE8F88328BA0020C4
:1054800047E8010048E80100E9B50500FEB5050060
:1054900041C2002042C2002094B60500D8BA0020C4
:1054A0000020004071A903008000020014B605002E
:1054B00010B50D4C00226260A2602261E2600B4ACE
:1054C000106810F0010002D10621FFF7DFFE084B43
:1054D0001B7823B94FF080430122C3F8182501231C
:1054E0002370002010BD00BFA8BB002000E100E039
:1054F00021C10020F8B50E46D11C48BF911D1446AD
:1055000041F387010546671EFAF75BFC00214AB2AA
:10551000A24201F1010100DBF8BDBB1A23F0030038
:10552000B25C03F00303DB0002FA03F32A581A43C8
:105530002A50ECE7F0B500254F1E6CB28C4205F105
:10554000010500DBF0BD3B1B23F0030603F0030362
:105550009659DB0026FA03F30355EEE72DE9F041F7
:10556000B3F9024014F11F0548BF04F13E050F4690
:1055700003F1240645F34715904601462B46324673
:105580003846FAF75DFCB8B9B4EB451F16DA62117C
:10559000012304F01F0403FA04F457F822301C42DC
:1055A00014BF012400242B46324639464046FAF700
:1055B00047FC2046BDE8F0810124F4E70446F2E709
:1055C00010B500231A465CB2A14203DCB2FA82F0A5
:1055D000400910BD50F8234001332243F3E7000097
:1055E0002DE9F04F8A46234F8BB0064611465046B0
:1055F0001446FAF7C6FB3B68FBB10425C0EB441028
:1056000014FB05FB00B205FB04654FF0FF38043DB9
:1056100028FA00F84FF040093B6859463046984751
:1056200058B12B6803EA08032B6021463046FFF788
:10563000C7FF20B1B9F10109EED1002017E02346E0
:105640003246514602A8FAF7CBFB2146019002A848
:10565000FFF7B6FF019B003318BF01235B00002852
:1056600014BF5842C3F10100C0B20128E2D10BB00F
:10567000BDE8F08F802D00202DE9F04FD1B0CDE9AD
:1056800005015B9D95F9004048A8914622461F46BA
:10569000FAF76BFBA3000793069BA200134419467D
:1056A000224638A80293FAF760FB95F90060002FB4
:1056B00000F08C803246394628A8FAF756FB0DF5E3
:1056C000807A324630AF48A95046FAF74EFB38A9E7
:1056D0003846FAF74AFB2B4628AA38A948A8FAF711
:1056E00003FB2B4628AA38A948A8D5F8A460B047E0
:1056F0002B4628AA39465046FAF7F6FABDF9683122
:105700000497023B1BB2002B67DCD9F800300095F0
:1057100003F001084FEA481840AADB4302EB080AED
:1057200003F0010330AA90445B0140AA1A4403929B
:1057300030AAD3184146039A0493504605F1040950
:10574000FAF775FD4B4640AA48A908A80094FAF755
:10575000DEFC08A908462B464246FAF784FA08A957
:1057600008462B46069AFAF77EFA214608A8FFF764
:1057700027FF00285DD008A8FAF723FB08A92B46CD
:10578000029A0846FAF76FFA08A92B4652460846CD
:10579000FAF769FADDE90301434652460095FAF744
:1057A000C8FC2B4608AA30A940A8FAF79DFA224661
:1057B00040A90598FAF7D9FA059B079C234430A91C
:1057C0001846FAF7D2FA51B0BDE8F08F314628A852
:1057D000FAF7F7FA0123289371E71FFA83F85B11B0
:1057E00008F01F0259F823300095012101FA02F256
:1057F0001A42049B13BF20270027202600260AEB0D
:10580000070B1F440AEB06030393049B039A1E44F1
:10581000334639465846FAF70AFD08F1FF383B4649
:1058200000955A4631460398FAF783FC0FFA88F33D
:1058300069E710AF224608A938460DF1600BFAF768
:1058400094FA20AE49465846FAF78FFA3046214678
:10585000FAF7B7FA012328A82093FAF7B2FA2246FA
:1058600059463846FAF76CFA28B9224620A908A802
:10587000FAF77BFA82E73B68DA0709D42146384613
:10588000FAF751FA224649463046FAF724FCE6E791
:10589000189BDB0707D421465846FAF744FA2246FC
:1058A000494628A8F1E7002823461CDD5A46394618
:1058B0003846FAF795FA21463846FAF734FA22467E
:1058C00028A93046FAF73CFA002805DA23464A466A
:1058D00031463046FAF7B4FA234628AA3146304614
:1058E000FAF77EFACEE73A4659465846FAF778FA7A
:1058F00021465846FAF717FA2246314628A8FAF701
:105900001FFA002805DA28A923464A460846FAF76E
:1059100097FA28A9234632460846FAF761FABEE705
:105920002DE9F04793F9006092B00446894610468D
:10593000314615469846FFF743FE002840F0918017
:10594000424649460AA8FAF7CBF943460AAA214635
:1059500002A8FAF788F90AA908464246FAF7C0F9F8
:1059600043462A4649464846FAF77DF908F10407B6
:10597000424629462846FAF7B3F93B462A462146CD
:1059800020460096FAF73AFC3B462A462946284626
:105990000096FAF733FC3B462A46214628460096F5
:1059A000FAF7B5FB43462A4621462046FAF75BF94B
:1059B0003B462246214628460096FAF71FFC3B4606
:1059C00000962A4621462046FAF718FC2368DB0792
:1059D0004AD533463A4621462046FAF731FA31464F
:1059E00082462046FAF79FF906F18043013B54F8BE
:1059F000230040EACA7044F8230042462146284664
:105A0000FAF76EF93B4602AA294628460096FAF7AD
:105A10007EFB3B4602AA294628460096FAF777FB0A
:105A200002A908463B462A460096FAF770FB434611
:105A300002AA21462046FAF716F90AAA3B46104662
:105A400021460096FAF763FB324629462046FAF7CC
:105A50008CF949462846FAF788F90AA94846FAF720
:105A600084F912B0BDE8F08731462046FAF75BF9B9
:105A7000C3E7000073B500230DF102008DF802307A
:105A8000FBF760FB264B1B7803F0FF04002B41D192
:105A9000244B1A68002A3DD0234AD2F80813C907BC
:105AA00038D51C601B68214D01930DF10300019B4B
:105AB000D2F808658DF80340FBF744FB6A68296853
:105AC0001F2A98BF541CA142F6B26C6004D1202C4E
:105AD00014BF611C0021296015499DF803008E54F4
:105AE0002A6894423ABFC2F121021319A31AAA6884
:105AF0009A4238BFAB60FBF773FF6B682A681F2BB5
:105B000094BF013300239A4201BF074A0123C2F820
:105B1000083353609DF80200FBF762FF02B070BDCE
:105B200021C1002000D1004000D000400CC1002065
:105B3000E8C0002030DF70472DE9F74F3B4F0646A5
:105B40008846B8F1000F03D1012003B0BDE8F08F03
:105B50004546202D28BF20255FFA85FB0024002321
:105B60000DF102008DF80230FBF7ECFA304B1B7898
:105B700003F0FF0993BB0DF103008DF80390FBF7D1
:105B8000E1FAD7E900148C4204D3641AA54207D97C
:105B9000052414E02134641AA542F9D8C1F1210486
:105BA000244BA542194431D82A46304635F0E2FB51
:105BB0003B682B44212B28BF00233B6000249DF829
:105BC0000300FBF70DFF1C4B00221A601B680193BA
:105BD000019B1A4B0122C3F804231A609DF80200AE
:105BE000FBF7FEFEB9F1000F08D059463046FFF72B
:105BF000A1FF42F2070398420446ADD0022CAED07A
:105C0000002CA9D1A8EB05082E449AE7224630467D
:105C100035F0B0FB074BA5EB040A52461946301984
:105C200035F0A8FBC7F800A0C8E700BF0CC10020F2
:105C300021C10020E8C0002000D1004000D0004079
:105C400017B4314A314B116889B90021304A1068C4
:105C500020BB00205A79D40740D408B9002949D084
:105C60001C68DA88234603B05DF8044B184700210E
:105C700011601268D9680092009A0029E5D0254A7F
:105C8000D2F84005814204BFD88801EB8001C2F8F8
:105C900040155A7942F004025A71D7E7002010608B
:105CA000126898680192019A0028D2D0194AD2F855
:105CB0003845A04204BFDC8800EB8400C2F83805F8
:105CC0005A7942F0020214075A71C3D512F0010446
:105CD00002BF64F3C3025A712046BBE702F006011B
:105CE000062907D122F0060211075A7106D56FF373
:105CF000C3025A7103B05DF8044B7047054AD2F8ED
:105D00003805D2F84015ABE71451024070BA0020B4
:105D10000451024000500240A5DF7047A4DF7047E5
:105D2000A3DF70472DE9F0470E4690B016F010053E
:105D3000814692469846189C0CD011238DF8083065
:105D400023788DF8093001224FF0000362F34203FB
:105D50008DF80A301C22002109A8F9F7E3FB8DF821
:105D6000246005B102AD42F64D23ADF80C306378E6
:105D70009DF864108DF804300022A3788DF805306A
:105D8000134661F3C303DBB243F00303CDE90622FC
:105D90000E95012701AD8DF80630089203AE1A9BCF
:105DA000B9F800008DF80E7004AA09A9CDE90465C0
:105DB000ADF81CA0FDF706FD58BB42F60813ADF880
:105DC0000C3063788DF80430A3788DF805300346E5
:105DD00067F342038DF806301A9A98F800308DF870
:105DE000003098F80130CDF81A00ADF81E008DF89B
:105DF000013032F8080B8DF80E70022304A9CDE9AA
:105E00000465ADF81830ADF81C30CDF820D0FFF7A0
:105E100087FF10B0BDE8F087A1DF7047BFF34F8F59
:105E20000549064BCA6802F4E0621343CB60BFF336
:105E30004F8F00BFFDE700BF00ED00E00400FA0552
:105E400008B5FAF7CDFA10B1664B674A1A60FAF74F
:105E5000A7FA28B1654B664A1B68C3F34233136047
:105E6000FAF7BEFA20B1634AD36823F08073D36097
:105E7000FAF796FA40B14FF080430022C3F80C21A4
:105E8000C3F81021C3F83825FAF7AAFA10B15A4B13
:105E900003221A60FAF7A4FA40B1584B05221A609F
:105EA00001229A6700229A603F225A60544B1B7865
:105EB000062B50D1534B1B681B074CD1524B1B6810
:105EC00003F0F003502B46D14FF080524F4BD2F8E5
:105ED0000414C3F82015D2F80814C3F82415D2F816
:105EE0000C14C3F82815D2F81014C3F82C15D2F8E6
:105EF0001414C3F83015D2F81814C3F83415D2F8B6
:105F00001C14C3F84015D2F82014C3F84415D2F875
:105F10002414C3F84815D2F82814C3F84C15D2F845
:105F20002C14C3F85015D2F83014C3F85415D2F815
:105F30003414C3F86015D2F83814C3F86415D2F8D5
:105F40003C14C3F86815D2F84014C3F86C15D2F8A5
:105F50004424C3F87025FAF723FA28B12C4B2D4AB4
:105F60001B6803F04F0313602B4AD2F8883043F4C8
:105F70007003C2F88830BFF34F8FBFF36F8F4FF0BD
:105F80001023D3F80022002A03DBD3F80432002BBD
:105F900024DA224B0122C3F80425D3F80024002A76
:105FA000FBD04FF010221521C2F80012D3F80024C4
:105FB000002AFBD04FF010231522C3F80422174B00
:105FC0001A46D3F800140029FBD00021C3F80415A9
:105FD000D2F80034002BFBD0FFF720FF104B114A02
:105FE0001A6008BD74C007400DF0ADBA440200103D
:105FF0003C050040F0ED00E0A005004010560040D8
:10600000E00F00F0E40F00F0E80F00F000C00040E7
:1060100058020010E40E004000ED00E000E00140F6
:10602000A42C00200090D003002382B003600368FA
:106030000193019B02B070472DE9F341844BD3F8E3
:10604000042162B3D3F800339F0728D5814D8248DD
:10605000FFF7EAFF2B7803F0FF08F3B97F4F804E7C
:106060007B783C4603F0FF02002B00F0AF807368A2
:106070004046984701A88DF80480FBF763F87B68D9
:106080009DF8040001337B60FBF7AAFC754B0122ED
:10609000DA601A60744B00221A6001232B706C4B7B
:1060A000D3F81821D2B1D3F80023560616D5D3F869
:1060B00024356E48DB08C3F3080113F4FF7F18BFD3
:1060C0000239FFF7B1FF624B4FF48052C3F8082545
:1060D0004A1EFE2A40F2A4800122DA615C4AD2F80C
:1060E0001031D3B1D2F80033DD0616D56048FFF782
:1060F0009BFF1023C2F808335E4BC2F81035FF2314
:10610000C2F814350123D3615B4B1C682CB15B488A
:1061100000231A4603210068A0474D4AD2F84C31AB
:1061200033B3D2F800331C0322D55548FFF77CFF68
:106130004E48FFF779FF5348FFF776FF4D4BC2F803
:106140001035FF23C2F814350123D3614FF488635F
:10615000C2F804330D23C2F80C34C2F80434464BA1
:106160001C682CB1454800231A4619460068A04710
:10617000374AD2F828315BB1D2F80033580507D539
:106180004048D2F80C34FFF74FFF0D23C2F80C340F
:106190002F4AD2F81C31B3B1D2F80033190612D508
:1061A0003948D2F80414FFF73FFFCB0707D5374B28
:1061B000197821B10121C2F8041400221A70244B6D
:1061C0000D22C3F8042402B0BDE8F0810DF10300F4
:1061D0008DF80320FAF7B6FFBA68134683B9326028
:1061E000A660636833B92A4B1B7803F0FF025BB1EA
:1061F000F9F7C4FB63689DF803000133636043E76C
:10620000B342EED01B68E9E7224B1A601B6801938A
:10621000019B4FF080430122C3F804231A60E9E791
:10622000144A1078502803D1184901220A7054E703
:1062300011480468002C3FF451AF4FF6FF70C3F8CB
:1062400008050E480B4600680221A04746E700BF3C
:106250000050004094BC002004510040A8BB002026
:10626000BCBB002000B001407C2D00201851004034
:106270001051004040BE00204CBF002050BF002005
:106280004C510040285100401C51004020C10020CA
:1062900021C100200001004013B5284B2849D3F844
:1062A0003C3413F0030345D10A680132072A0A601F
:1062B0002CD9244A012414610DF107008DF8073010
:1062C000FAF740FF204B5A68013A5A605A6822B9DF
:1062D0001E4A127802B3F9F74FFB9DF80700FBF74F
:1062E0007FFBBFF35F8F1A4A00231360BFF35F8FFA
:1062F00001211160174A14681CB117481A4600683A
:10630000A047164B00221A70FAF79EFE0D4B002292
:10631000C3F8402102B010BD114A4FF08041146013
:10632000D1F80C2402F00112B2F1011FF8D00022C2
:106330005A70D2E700230B60E8E700BF005000402E
:106340007C2D002000B00140A8BB002021C100200E
:10635000FC5F00404CBF002050BF002094BC0020D8
:10636000040000408DDF704777DF704701381F2839
:106370009DBF034B23FA00F000F00100002070479E
:106380008B80808030B551EC100B85B053EC112B15
:106390008DED000B55EC124B8DED021B34F048FDDA
:1063A0009DED000B28B19DED021BB0EE410AF0EE11
:1063B000610A53EC102B204629468DED000B34F07A
:1063C00037FD9DED000B08B145EC104B05B030BD1D
:1063D00038B555EC104B0022002310EE100A294668
:1063E00034F026FD10B105F100431D4645EC104B7D
:1063F00038BD436833B1013B436003685A1C0260F7
:10640000187870474FF0FF3070470B685A1C0A60CD
:10641000187070472DE9F04F89B00E4600AF002389
:10642000044607F1140130467B612DF045F905461D
:1064300018BB30462EF044FB8046786125F0E6FF1D
:1064400008F5807383420CD9A649012026F062FB2F
:106450003246A549012026F05DFB2437BD46BDE844
:10646000F08F08F1070323F00703ADEB030D6D4632
:106470004246294630462EF013FB7E6926B99B49D9
:10648000012026F047FBE8E74FF00308B6FBF8F3DE
:1064900003EB43039E4201D09549F1E7204622F0E9
:1064A00043FB08B99349EBE7934BC7F808D004EBDB
:1064B00084041C446178914C2079002840F00981C3
:1064C0008F4A0123C2F80405FF29C2F82405C2F847
:1064D0002005C2F81C35C2F82805C2F818054FF08F
:1064E000C050C2F81405C2F8103518BF01F5E070AD
:1064F0004FF0A04308BF4FF0FF31C3F85887C3F8EF
:10650000FC8A18BF43F820801623C2F86435FF23A5
:10651000C2F868354FF0FF33C2F860352520C2F865
:106520007015C2F86C350221764B2360FEF7AEFE83
:10653000012323710323B6FBF3F39BB203EB430860
:1065400008F1010828F001029100ADEB010D684649
:10655000FA606D4A3A6041184FF0000C796082F899
:1065600000C0E91C4FF0EE09851C4FF0880A4FF07F
:106570008E0B63455FDC0C2202FB0303002279686B
:10658000994200F29E802679012E40F0A28000F010
:106590006043B3F1005F40F0A280FB68C3F34E029A
:1065A000574B0021C3F85025C3F83815C3F8081518
:1065B000C3F84005C3F80C656579E28025F009054C
:1065C00045F008056571C4E90210C3F800650223AF
:1065D00023710D46002977D04FF6FE7208EA0202B9
:1065E000F8F7A0FF494B00221A601B68FB61FB69AA
:1065F000474B1A601B68BB61BB69414B2222C3F841
:10660000042301221A603A681278042AFBD941490E
:10661000002222250120C3F808530860C3F8002592
:10662000C3F808530860C3F800253B4B2021C3F88A
:106630008410227150E011F8026C11F8032C36021C
:1066400046EA024611F8012C05F10C0E164306F439
:106650004012B2F5001F1ED0B2F5401F20D0B2F597
:10666000801F20D105F802BC06F44002B2F5000FED
:106670001CD0B2F5400F1ED0B2F5800F1ED105F828
:1066800001BC0235AE454FEA0616E0D10CF1010C13
:10669000033175466DE76FF0170205F8022CE3E74A
:1066A00005F8029CE0E705F802ACDDE76FF01702A1
:1066B00005F8012CE5E705F8019CE2E705F801ACD7
:1066C000DFE703F8012B5AE701462368284698477D
:1066D00088E70820FBF722F9D7F808D0BDE610209C
:1066E000F8E700BF25B505006FD305009BD3050073
:1066F000BBD30500E6D3050094B6050070BA0020B0
:1067000000500240AD81030055C2002004510240F8
:10671000145102400450024000E100E010F5A24F85
:106720000FD006DC10F5A34F0ED04142084826F0EA
:1067300023BD10F5A14F09D010F1220FF5D1054965
:1067400000E005490548F2E70549FBE70549F9E797
:1067500057D0050033D0050048D005003BCF0500D9
:106760000DD005001FD00500024B034958680022D8
:106770002EF00AB8682D0020F12306002DE9F04F15
:10678000ADF51B7D00AF144605461022884607F183
:10679000180000219B46F8F7C5FE20462BF096FB1B
:1067A0000646002859D00022BE4920462DF0ECFFB5
:1067B000064680B1102207F118012EF071F9F38915
:1067C000A3F500739BB2F381F38903F4F05313B97B
:1067D00030462CF0ADF820460022B3492DF0D4FF0E
:1067E0000446002843D0B1492CF008FC002840F0B2
:1067F0005582AF4920462CF001FC002840F0518220
:10680000AC4920462CF0FAFB002840F04D82AA4902
:1068100020462CF0F3FB002840F04982A74920468F
:106820002CF0ECFB0646002840F044822246A449A6
:10683000012026F06FF9B146E389A3F500739BB2FE
:10684000E381E38903F4F05313B920462CF070F888
:10685000B9F1000F0DD1002603E044B1994826F0AC
:106860008BFC304607F51B77BD46BDE8F08F4FF037
:1068700001094FF48C72002107F13800F8F752FE3D
:10688000002307F1140128467B612CF015FF044614
:10689000D0B928462EF014F90646786125F0B6FDE9
:1068A00006F58073834204D98749012026F032F926
:1068B000D1E7F31D23F00703ADEB030D6C46324621
:1068C000214628462EF0ECF8002307F1100140463F
:1068D0003B612CF0F1FE0546A8B940462EF0F0F8D9
:1068E0000646386125F092FD06F580738342DBD8B9
:1068F000F31D23F00703ADEB030D6D463246294629
:1069000040462EF0CDF83E69F600BBF1000F3DD1B8
:106910004FF48C72594607F5A870F8F703FE07F19B
:1069200040033246294607F5A870FB631BF0B0F818
:106930008046F8B9D7F85011D7F85401B9630B0164
:10694000C218C3583B6453687B649368BB64D368C4
:10695000FB645E4E4B1E7B60103A07F15003796872
:10696000002921DC116819605168596091689960AB
:10697000D268DA60002340F21912184607F5A871B0
:1069800019440133934208D00870F7E7324629468C
:1069900007F138001BF07CF88046B8F1000F2ED0CC
:1069A0004046FFF7BBFE56E7A2F1040E03F1100AC2
:1069B0005EF8040F4649C5B216F805C0050E51F839
:1069C0002CC0755D434951F8255043498CEA050CAC
:1069D000C0F30725C0F30740755D305C51F82550C2
:1069E0003E4951F820008CEA0505454043F8045B18
:1069F0005345DDD1796801397960103AAFE707F185
:106A00000C017869C7F80C80FAF72EFAFD68064683
:106A10001DB9334826F0B0FB1DE709F1FF39B9F184
:106A2000040F00F23381DFE819F00500AF00E30046
:106A300031012F01D7F814A01AF00F0F40F029816F
:106A4000BBF1000F4ED0013D0F3405F10109BAF141
:106A5000000F4FD007F11801A4F1100328468B4610
:106A600013F801CF11F8012B9C4282EA0C0200F8C6
:106A7000012FF5D14A46494607F138001AF0ACFE1D
:106A80004A465B4605F1110E106851689C46ACE819
:106A90000300083272456346F6D1AAF1100A103598
:106AA0001034D2E798CF0500580306009BCF0500AD
:106AB0009FCF0500A3CF0500A7CF0500ABCF0500F2
:106AC000AFCF0500C6CF050025B5050057B70500B7
:106AD0003CB905003CC505003CBD05003CC10500B6
:106AE000F0CF05000F35A24407F5A8795445A5F16C
:106AF0000F0222D1002340F21912184607F1380183
:106B000019440133934240F0C780B8F1000F3FF4BD
:106B1000A8AE4046FFF702FE002E3FF49CAEF3897C
:106B2000A3F500739BB2F381F38913F4F0547FF45F
:106B300092AE30462BF0FCFE8DE62346CE4604F1A5
:106B4000100B18685968F446ACE8030008335B453D
:106B5000E646F6D1214607F138001AF0DFFC07F1CE
:106B60001801A5F110038C4613F8010F11F8012B41
:106B70009D4282EA00021A70F6D199E80F001034A3
:106B80008CE80F001035B1E77B69E3187B6007F5EF
:106B9000A87A07F118097B68A342ABD099E80F00E7
:106BA0008AE80F004A46494607F138001AF014FEF9
:106BB000BBF1000F02D123788AF8103099F8003029
:106BC00014F8012B534005F8013BBBF1000F01D035
:106BD0008AF8103007F25113CC4607F2611E18688C
:106BE0005968624603C2083373459446F7D1D2E729
:106BF00007F5A87B10220021584607F1280AF8F76C
:106C000091FC102200215046F8F78CFC7A694FF075
:106C10000009A3189C423FF46DAFB9F1000F0BD0EF
:106C20001AF8092014F8011B09F101094A4005F876
:106C3000012B09F00F09EDE75946524607F13800DC
:106C40007B601AF0C9FD7B6807F5B07111F8012D62
:106C50000132D2B20A70002AE2D18B45F6D1DFE7C9
:106C6000FA6861192A4407F13800BBF1000F08D017
:106C70001AF0B2FD10357A6905F10F039A42EFD888
:106C800038E71AF04BFCF5E70025F4E7DFF82C8035
:106C900030E76FF021082DE708702FE74FF001096A
:106CA000CAE54FF00209C7E54FF00309C4E54FF00C
:106CB0000409C1E54FF00509BEE500BF80AFFFFF45
:106CC0000023FFF75BBD0123FFF758BD70B500221D
:106CD000164905462DF058FD2EF046FA144B15497D
:106CE0000646032258682DF04FFD044678B1002275
:106CF000B1B22DF07BFCE389A3F500739BB2E38175
:106D0000E38903F4F05313B920462BF011FE0A4B2C
:106D10001C6824B1E38903F500739BB2E381284624
:106D2000002112F0B3FE204670BD00BFE5C905008A
:106D3000682D0020F2C9050044C2002008B540B209
:106D4000FFF712FBBDE8084012F0F6BA38B5054669
:106D500008460C462BF0D2F8002808BF0024224633
:106D60000E4928462DF0B6FC0D4B4FF6FF721988E0
:106D700074B18A4204D10020BDE8384012F0DCBA78
:106D800000221888114613F0DBFB0828F4D1F2E743
:106D90008A42F0D0188813F0D1FBF6E7C0C905008D
:106DA000B42C0020014B188812F0E0BAB42C00205B
:106DB000014B188812F0DABAB62C002008B5074B40
:106DC0001A884FF6FF71914207D018881321FDF7FA
:106DD000F5FCBDE8084012F0AFBA08BDB62C0020A3
:106DE00007B500230846072269460093CDF8033013
:106DF0002EF0ACFD094B1A884FF6FF71914209D075
:106E000018886A46012113F0C7FB12F095FA03B007
:106E10005DF804FB43F20200F7E700BFB42C00204A
:106E200038B500220E4905462DF0AEFC0446A8B93F
:106E30000C4925F099FF0A490446024628462DF0E0
:106E400049FC2A46084920462DF044FC00202BF03E
:106E50000CFD0649024620462DF05DFC204638BD5B
:106E60009AC905009FC90500B9C90500DBC905001D
:106E700010B504462BF02AF8224630B92CB1074948
:106E80000320BDE8104025F045BE054B0549586874
:106E90002EF0ACFABDE8104012F0F2BC47CE05006F
:106EA000682D002070CE0500F8B5044628B9214AA7
:106EB000136823F480431360F8BD1F492CF09EF83B
:106EC0000028F4D120462BF03DF8054690B1194A30
:106ED0001368204643F4804313602EF0CBFD53EC3F
:106EE000102B10EE100A194616F01EFBBDE8F840F4
:106EF00012F022BA20462AF0E9FF0028DCD00D4A21
:106F00000E49136843F48043136020462A462DF04F
:106F10003BFC2FF0CDF82A4606460F46204608498E
:106F20002DF032FC2FF0C4F802460B4630463946AD
:106F3000DAE700BF48C2002013CD050018CD0500D8
:106F400024CD0500084B1A6818B142F400521A60AB
:106F5000704722F400521A60044B1860044B01225F
:106F60001A7011F061BF00BF48C2002058C2002053
:106F700057C20020F0B583B0044600AF28B90146DF
:106F800011F08EFF0C37BD46F0BD2BF098F928B1FB
:106F900020462DF03FF90421C0B2F1E77860391D99
:106FA00020462CF089FB0546F0B920462DF088FDDF
:106FB0000646786025F02AFA06F58073834208D9E0
:106FC0000D49012025F0A6FD0C49012025F0A2FD68
:106FD000D8E7F31D23F00703ADEB030D6D463246F2
:106FE000294620462DF05CFD79680029ECD0284622
:106FF00011F088FFC6E700BF25B5050048D505009C
:1070000008B5044B044958682EF0D6F9BDE808408D
:1070100011F0B0BF682D002088D50500F0B583B011
:10702000044600AF11F0A6FF002C69D00023391DE3
:1070300020467B602CF040FB054610BB20462DF01F
:107040003FFD0646786025F0E1F906F5807383423E
:107050000CD93A49012025F05DFD3949012025F080
:1070600059FD002420460C37BD46F0BDF31D23F02A
:107070000703ADEB030D6D463246294620462DF041
:107080000FFD78680028E8D02BF076FA044608B99E
:107090002C49E3E72C4B2D49024658682DF01AFB8A
:1070A000E389A3F500739BB2E381E38903F4F05312
:1070B00013B920462BF03CFC20462AF065FF7A6885
:1070C000294634F057F920462AF05EFF054620464F
:1070D0002CF0C9FA0146284611F05CFF0023391D47
:1070E0000A207B60F9F7C0FE7B680446002BB9D00C
:1070F000174A116819605168596012891A81B1E7FD
:1071000020462BF039FA044620B90E49012025F01B
:1071100001FDA7E70C4B0D49024658682DF0DAFA3D
:10712000E389A3F500739BB2E381E38903F4F05391
:10713000002BC8D120462BF0FBFBC4E725B505008A
:1071400048D505005FD50500682D002088D50500CD
:107150003FBF0020F0B583B0054600AF48B9424BB1
:10716000424958682EF028F9FFF74AFF0C37BD4610
:10717000F0BD0023391D7B602CF09EFA0646F0B965
:1071800028462DF09DFC0446786025F03FF904F573
:107190008073834208D93649012025F0BBFC35496C
:1071A000012025F0B7FCE1E7E31D23F00703ADEB79
:1071B000030D6E462246314628462DF071FC786854
:1071C0000028ECD013302BF0D7F9054608B92A492E
:1071D000E6E7254B2549024658682DF07BFA2846FC
:1071E0002AF0D2FEEB89A3F500739BB2EB81EB8909
:1071F00003F4F053044613B928462BF099FB1F4BB8
:10720000224603F1100153F8040B42F8040B8B42A1
:10721000F9D11B8813807D6831462A4604F112009B
:1072200034F0A8F865742544FE23AB740020FFF702
:10723000F5FE394605462CF03FFA28B10368236075
:107240004368636003892381002D8FD0EB89A3F508
:1072500000739BB2EB81EB8903F4F053002B85D1D3
:1072600028462BF065FB81E7682D002040D50500FE
:1072700025B5050048D505005FD505003CB70500DC
:107280002DE9F04182B0054600AF50B9594B5A493B
:1072900058682EF091F8FFF7B3FE0837BD46BDE8F9
:1072A000F0812AF03DFF28B92A465449032025F0F1
:1072B00031FCF2E70023391D28467B602CF0FCF9F5
:1072C0000446F0B928462DF0FBFB0646786025F011
:1072D0009DF806F58073834208D94949012025F0BD
:1072E00019FC4849012025F015FCD6E7F31D23F0D1
:1072F0000703ADEB030D6C463246214628462DF0C0
:10730000CFFB7D68002DECD007223F49204634F0AA
:1073100023F860B9073D07347D604FF003087868B3
:107320001B302BF029F9064680B93849DAE70822E4
:107330003749204634F010F828B9083D08347D60FC
:107340004FF00408EBE74FF00008E8E7294B2A4923
:10735000024658682DF0BEF930462AF015FEF38932
:10736000A3F500739BB2F381F38903F4F053054650
:1073700013B930462BF0DCFA264B2A4603F11801EC
:1073800053F8040B42F8040B8B42F9D11B8813808D
:107390007E6885F819802146324605F11A0033F0DF
:1073A000E9FFF3B203F108022E440133EB75FE232B
:1073B0006A740020B376FFF731FE394604462CF09C
:1073C0007BF928B103682B6043686B6003892B81CC
:1073D000002C3FF462AFE389A3F500739BB2E38115
:1073E000E38903F4F053002B7FF457AF20462BF0D2
:1073F0009FFA52E7682D002040D50500D4D405003F
:1074000025B50500EFD4050006D5050017D5050004
:107410000ED505003CB7050010B504462AF06EFDF8
:10742000084B0949002808BF0024224618682DF09F
:1074300051F9201C18BF012013F084F8BDE810405A
:1074400011F07ABF682D0020C0C905002DE9F74F63
:10745000504B51490546032258682DF095F90646D0
:10746000002845D000224D49DFF8308128462DF014
:107470008BF93146814668462AF0A7FA009CECB1A8
:1074800020462CF08FFE0022414607462DF07CF965
:107490000123002249468246F9F77EF958BBFB8951
:1074A00003F500739BB2FB813C46504639462CF0F5
:1074B0009DFD68462AF074FA002CDFD0009850B188
:1074C000C389A3F500739BB2C381C38903F4F0534E
:1074D0000BB92BF02DFA2946002C57D001A82AF021
:1074E00074FA019D4DB93246494620462CF052FDB2
:1074F00003B0BDE8F08F0024D7E7EB8903F50073F4
:107500009BB2EB8128462CF04DFE0122294607460E
:1075100020462DF037FC2249804628462BF06EFD90
:107520002049824628462BF069FDBAF1000F00D1B0
:10753000D0B140462CF036FE834610B3BAF1000FAE
:107540001BD0012239462FF010FFBBF80E20A2F508
:10755000007292B2ABF80E20BBF80E2002F4F0528B
:1075600012B958462BF0E4F940463A4629462CF029
:1075700011FD01A82AF014FAB3E739462DF05FFC9B
:10758000E3E7394640462CF037FCEDE730462CF077
:10759000B3FFA8E7682D0020C7CA050021CC05006D
:1075A000CECA0500D7CA0500F8B5064608460C46FF
:1075B0002AF08CFC074620B30022394920462DF0E2
:1075C000E3F82DF08EFF00220746364920462DF0C5
:1075D000DBF80446E0B12AF071FCC8B9E389A3F5F1
:1075E00000739BB2E381E38903F4F05313B920469F
:1075F0002BF09EF922462C490320BDE8F84025F0E7
:1076000089BA2CB122462949032025F083FA3C4649
:1076100030462AF073FC00283AD0002E38D048F2C9
:10762000480123482BF00AF90546D0B12246002133
:107630002DF0CEFC32461F4928462DF04BF81E4B4C
:107640001E4918682A462DF045F8EB89A3F500730A
:107650009BB2EB81EB8903F4F05313B928462BF06E
:1076600067F9301C18BF0120394611F013FD11F0E5
:1076700063FEA4B1E389A3F500739BB2E381E389C0
:1076800003F4F0535BB92046BDE8F8402BF050B945
:10769000094B0A4918682DF08FFE0026E1E7F8BD76
:1076A0003ACD0500E3CB050041CD050075CD0500C1
:1076B000797802008ECD0500682D002093CD05005D
:1076C0002DE9F84380460C462AF018FC30B93849B9
:1076D00042460120BDE8F84325F01CBA20462AF0B6
:1076E00031FC05462046C5B12EF0C4F957EC106BAD
:1076F000002432463B463046394633F0C1FB30B9B0
:1077000000222C4B3046394633F092FBC8B12A494F
:107710000120BDE8F84325F0FDB92AF0D7FB50B1B0
:107720002A46264920462DF02FF840B12EF0C0FC05
:1077300006460F46DDE714B122462149C9E7214F2D
:107740000026214DD5F804902BF082F81F490246FF
:1077500048462CF0E0FF42461D4968682CF0BAFF0D
:1077600008211C482BF06AF8054670B12146FFF746
:107770001BFFEB89A3F500739BB2EB81EB8903F44C
:10778000F05313B928462BF0D3F8002112482BF000
:1077900055F8044648B1002147EC106B0CF0FCFA98
:1077A0002146BDE8F8432CF021BCBDE8F88300BFBA
:1077B0005DCA050000002440AECA0500B6CA050037
:1077C0008BCA050000409F40682D0020C7CA0500F5
:1077D000BECA05004D740200DD77020037B5144CB7
:1077E00000210846FFF7E0FE0322124960682CF0F2
:1077F000CBFF00220190104960682CF0C5FF0D49B5
:10780000054660682DF0D8FD0B4960682DF0D4FD69
:10781000019B33B12DB1012301AA2946002020F09C
:10782000BBFF294601982CF0E1FB03B030BD00BF3F
:10783000682D0020C7CA0500BECA05001FB54FF05D
:107840008052D2F8A430D2F8A820D8B20290C3F364
:1078500007200190C2F30721C3F3074000901B0EDD
:10786000D2B241F0C00103482BF0AEFD05B05DF887
:1078700004FB00BFE3CA05002DE9F04F8BB000AF59
:10788000C7E902011446002A76D09E49002025F05F
:107890006BFA0022054638619B4920462CF074FFA4
:1078A0009949024628462CF036FF002297493D6947
:1078B00020462CF069FF9549024628462CF02BFF04
:1078C0002AF0C6FF804604F0F9FE00228346904964
:1078D00020462CF059FF8146E8B102468C493869B0
:1078E0002CF0F8FE002307F1240148467B622BF0C0
:1078F000E3FE044600284ED148462DF0E1F8054647
:10790000786224F083FD05F58073834238D981497C
:10791000012025F0FFF8B8F1000F07D0D8F80030AB
:1079200023B142467C4938692CF0D4FE58462BF0EE
:107930009AFE20B15A46794938692CF0CBFE5A4656
:10794000414648462CF026FBFB68002B40F0C080E7
:1079500007F1100301220021B86827F0BBF938694C
:1079600050B1C389A3F500739BB2C381C38903F4EB
:10797000F0530BB92AF0DCFF2C37BD46BDE8F08F81
:10798000EB1D23F00703ADEB030D6C462A462146A1
:1079900048462DF085F87B6A002BBCD0B8F1000F6B
:1079A000C4D0BBF1000FB6D0002514E0092A09D1DC
:1079B000A91C2144701ED7F810A02CF04BF958498F
:1079C000024619E0911E012927D89A4602239E42B9
:1079D00016DA013635447B6AAB429CD96319665D81
:1079E0005A78082AE2D1A91C2144701ED7F810A0A9
:1079F0002CF030F94B49024650462CF08CFEE8E75B
:107A00003AF8021F48487B602BF0DEFC01464046F6
:107A10002CF094FD7B680233D9E7911F012908D827
:107A2000A81C20441AF028FD014640462CF086FD93
:107A3000CFE7162A33D159883B482BF0C5FC2EF0EE
:107A40008CFD82460028C4D00122014658462DF004
:107A500099F9291D78602144F01E2BF003F87B680A
:107A600002463BB130B10146386018462CF0C4F9EB
:107A7000D7E90023184611462CF0B8FABAF80E30B0
:107A8000A3F500739BB2AAF80E30BAF80E3003F4D7
:107A9000F053002B9DD150462AF04AFF99E7FF2A68
:107AA00097D1D8789B78D7F810A043EA00202AF025
:107AB000E4FE1E49024650462CF02DFE291D2144AD
:107AC000F01ED7F810A02AF0CDFF1949024693E71F
:107AD000D7E9031607F1140029F077FF786948BB4E
:107AE0000446786950B1C389A3F500739BB2C38182
:107AF000C38903F4F0530BB92AF01AFF002C7FF46A
:107B000027AF2CE704CE050021CC0500C6C905002F
:107B10005AD5050025B50500CECA0500D7CA05000F
:107B2000B0D5050014CE0500572206001ECE050074
:107B30002BCE05002CF036FB0022BA4905462CF06E
:107B400023FE8046002800F00F810022B549304610
:107B50002CF01AFE4146814607F1180029F035FF46
:107B60000124B869002840F0CC80494640462CF0FA
:107B70003DFA0022AC4928462CF006FE8046E0B1D2
:107B80000022A94930462CF0FFFD814640462AF0EC
:107B90000EFB002800F0EA8048462AF008FB002887
:107BA00000F0E480494640462BF082FE002849461A
:107BB000404608BF00242CF019FA00229B492846B1
:107BC0002CF0E2FD804610B30022974930462CF09D
:107BD000DBFD814640462AF0A3FA98B148462AF0D8
:107BE0009FFA78B140462BF00AFD824648462BF0BA
:107BF00006FD824506D80123002249464046F8F793
:107C0000CBFD00B10024494640462CF0EFF900229C
:107C1000874928462CF0B8FD804680B1002284496F
:107C200030462CF0B1FD0146814640462BF040FE27
:107C300049460028404608BF00242CF0D7F900220E
:107C40007C4928462CF0A0FD8046F0B12AF03EF990
:107C500060B1414607F1240029F0B7FEDFF8D4A156
:107C6000D7F824B0BBF1000F40F09480B8F80E3084
:107C7000A3F500739BB2A8F80E30B8F80E3003F4E9
:107C8000F05313B940462AF053FE00226A492846B1
:107C90002CF07AFD8046F0B12AF018F960B1414627
:107CA00007F1240029F091FEDFF894A1D7F8249081
:107CB000B9F1000F40F09980B8F80E30A3F50073C9
:107CC0009BB2A8F80E30B8F80E3003F4F05313B995
:107CD00040462AF02DFE5DB1EB89A3F500739BB2FF
:107CE000EB81EB8903F4F05313B928462AF020FE08
:107CF00007F1140029F054FE002C3FF4EFAE0124EC
:107D0000EFE6B9F1000F12D02CF04CFA014607F162
:107D10001C001AF02DFB494607F1200029F055FE02
:107D20004FF0000A386A40B9BAF1000F00D10024C0
:107D300007F1180029F034FE13E72CF033FA01465E
:107D400007F124001AF014FBBA7F97F826309A4204
:107D500005D1BA8BBB8C9A4208BF4FF0010A07F1DC
:107D6000200029F01DFEDDE7012402E7334BA8EBDC
:107D700003000011013082B2B9F1000F08D0A9EB65
:107D800003000011013080B2131A584258410DE728
:107D90004846F9E7BBF80E3003F500739BB2ABF829
:107DA0000E300022514630462CF0EEFC814648B998
:107DB0000024584649462CF019F907F1240029F00F
:107DC000EFFD4DE7002259462CF0DCFF0028EFD0F4
:107DD000C389A3F500739BB2C381C38903F4F05335
:107DE000002BE6D12AF0A4FDE3E7B9F80E3003F545
:107DF00000739BB2A9F80E300022514630462CF099
:107E0000C3FC8346014648462BF052FD59460028E4
:107E1000484608BF00242CF0E9F807F1240029F0B7
:107E2000BFFD43E7CECA0500B0D505003CCE050036
:107E300021CC0500D7CA05002BCE0500882D0020D7
:107E40001ECE05002DE9F04186B000AF0023884624
:107E5000391D06467B602BF02FFC0546E0B9304605
:107E60002CF02EFE0446786024F0D0FA04F58073DE
:107E7000834206D93F49012024F04CFE32463E4958
:107E800038E0E31D23F00703ADEB030D6D462246FA
:107E9000294630462CF004FE7B68002BEED040468D
:107EA0002AF02CF828B1354B3549186842462CF099
:107EB00011FC344B1A6812F0400F1E4607D13249AC
:107EC000012024F027FE1837BD46BDE8F0812F4A77
:107ED00012884FF6FF71914201D12D49F0E71A68DF
:107EE00012F0800201D02B49EAE77C68102C05DDF6
:107EF00029491022012024F00DFEE4E7274B93F8D6
:107F000000C0274BA4B2BCF1000F23D19A7C62B30E
:107F1000B3F8760188422AD09B8A7C80C7F80AC0D1
:107F2000A7F80EC03B810123BB7207F10801BB1CFF
:107F3000C7E90435FBF744FC18B97B88A34218BF96
:107F40000C2011F0F9F90028BDD1336843F080030B
:107F50003360B8E7B3F87601884208D07C80C7F870
:107F60000A20FA81B3F84E31DCE70720E9E7082060
:107F7000E7E700BF25B505008ACC0500682D002085
:107F80001ACC050048C2002024CC0500B62C0020E5
:107F900038CC050047CC05005FCC050056C2002058
:107FA000A8BC00202DE9F04FB04B91B01B681B0717
:107FB00000AF044607D5AE49012024F0ABFD44379D
:107FC000BD46BDE8F08F15F029FB204629F07EFF65
:107FD0008046002800F05E81214607F1140029F058
:107FE000F4FCDFF8ACA2796981B10023BB61CB89D5
:107FF00003F500739BB2CB8107F118001AF0B8F9B2
:10800000024698B19B49012024F084FD786900283C
:10801000D5D0C389A3F500739BB2C381C38903F490
:10802000F053002BCBD12AF083FCC8E77D691DB14A
:1080300028462CF0B7F80546294607F11C0029F020
:10804000C4FCF969B8F1000F0FD071B1CB8903F509
:1080500000739BB2CB8107F120001AF089F9024628
:1080600010B38549012024F055FDF86950B1C3894A
:10807000A3F500739BB2C381C38903F4F0530BB91A
:108080002AF056FC5DB1EB89A3F500739BB2EB813E
:10809000EB8903F4F05313B928462AF049FC07F1A1
:1080A000140029F07DFC9EE707F128003C8C97F82E
:1080B00022601AF021FA08B1F9F730FC4FF00009FC
:1080C000002207F13001388DC7F830901AF012FA0B
:1080D000052810D043F2030290420CD0A8B93B8E81
:1080E000A34214D197F83230B34210D1B7F8289098
:1080F000B9F1000F0FD1386A1AF0D4F95F4904467C
:108100000246012024F006FD48E0F9F707FC3B8D0C
:1081100001333B85D4E7FC691CB120462CF042F8C2
:1081200004460022564920462CF02EFB00225549D9
:10813000064620462CF028FB2DF0D3F90022B8602B
:10814000514920462CF020FB2DF0CBF9F8602EB3DE
:10815000002307F1240130467B622BF0ADFA834601
:10816000002837D130462CF0ABFC7862786024F0E0
:108170004DF97A6802F58073834221D94349012081
:1081800024F0C8FCF389A3F500739BB2F381F38953
:1081900003F4F05313B930462AF0CAFB5CB1E3890B
:1081A000A3F500739BB2E381E38903F4F05313B9A1
:1081B00020462AF0BDFB07F11C0029F0F1FB40E747
:1081C000D31D23F00703ADEB030DEB4659463046B4
:1081D0002CF066FC7A6A002AD4D0002179853A8591
:1081E000494607F12802BAF80000C7F82CB0FDF79D
:1081F00095FD11F0A1F8BB6880F001005FFA80F8EE
:1082000013B9FB68002BBDD0BAF800204FF6FF7100
:108210009142B7D0FB68BAF80000A7F8309000226E
:10822000002BC7F83220FA867A6A7A8214BF0222BB
:10823000012287F8322007F1300107F11202C7E965
:108240000E2BFBF7BDFA30F008029BD043F204027C
:10825000904297D043F20142904293D011F06CF8D3
:10826000002818BF4FF000088CE700BF48C200206C
:10827000DDCE050005CF05001ECF05004ECF050061
:108280007AF605003ECF050045CF050025B505006F
:10829000B62C0020002C3FF492AE22460249032067
:1082A00024F038FC8BE600BF72CF05002DE9F04FBB
:1082B0009BB000AF0D4604463C22002107F12C0084
:1082C000F7F730F9022387F82C302846062387F881
:1082D0002F3029F0FBFD002800F08D8000228E4910
:1082E00028462CF051FA38B12DF0FBF8002814BFC5
:1082F0000223002387F82C300022884928462CF0DE
:1083000043FA38B12DF0EDF8002814BF06230523F9
:1083100087F82F300022824928462CF035FA06468D
:1083200018B3002307F10C01FB602BF0C5F9804660
:1083300000284ED130462CF0C3FB8146F86024F073
:1083400065F809F58073834237D97649012024F016
:10835000E1FBF389A3F500739BB2F381F38903F486
:10836000F05313B930462AF0E3FA284600226E494A
:108370002CF00AFA054690B13B6D002B36D02BF05D
:1083800049FF3B6D1880EB89A3F500739BB2EB812D
:10839000EB8903F4F05313B928462AF0C9FA2046B2
:1083A00029F08CFD80B3E38903F500739BB2E38170
:1083B00020466C37BD46BDE8F08F09F1070323F076
:1083C0000703ADEB030DE8464A46414630462CF024
:1083D00067FBFA68002ABCD084B06B464FF6FF7189
:1083E0003B6519809A80C3F80880B2E74F490320A3
:1083F00024F090FBC7E7002DD1D04D492A46032039
:1084000024F088FB0024D3E7204629F03BFD0646F4
:108410000028C8D1204629F059FD002876D02046F2
:108420002AF03EFD0C235843073020F00700ADEB47
:10843000000D214607F1080029F0C7FAE946DFF8E8
:10844000E4B04D46B246B868C0B987F85860C7F87E
:1084500054901F2307F1080207F10C0107F12C00CB
:108460003B81FCF753FA10F067FF0028CAD107F1EF
:108470000C0138892AF0F6FA044699E72BF092FEAF
:1084800007F10C010446C7F80CA02BF015F9804643
:1084900078B920462CF014FBF860786023F0B6FF22
:1084A0007A6802F58073834225D95946012024F069
:1084B00031FB5CB1E389A3F500739BB2E381E389EF
:1084C00003F4F05313B920462AF032FAB86820B109
:1084D000C38903F500739BB2C3812CF045FEFB6892
:1084E0002880AB80C5F8088007F1080029F058FA09
:1084F00001360C35A7E7D31D23F00703ADEB030DC1
:10850000E846414620462CF0CBFAD2E7002CA0D01A
:108510002246084973E700BF01CB05000ACB0500DE
:108520002BCE050025B505001ECE050017CB050096
:108530004BCB050081CB050008B5054A136823F431
:108540000073136010F08AFFBDE8084010F0F4BE1D
:1085500048C2002008B5054A136843F4007313604D
:1085600010F0C2FDBDE80840FEF728BC48C200205C
:1085700008B512F031F841EC100B08BD08B50C4BF2
:108580001B884FF6FF729BB2934203D1094A1288AF
:10859000934208D0084820F08BF9084A136843F04A
:1085A0000803136008BDBDE8084014F09BBD00BF80
:1085B000B42C0020B62C0020EBCB050048C20020D4
:1085C00038B50F4C0F490022054660682CF0DCF8E6
:1085D0002CF0CAFDC3B27DB143F0010098420ED029
:1085E00064682AF04AF90749024620462CF093F8BD
:1085F000BDE83840FFF7C2BF03F0FE00EEE738BD2C
:10860000682D002030CD05002DE9F0418CB00646E4
:108610000F4629F05BFC40B93EB132465249032077
:1086200024F078FA0CB0BDE8F081002302930193A6
:108630004E4B039302AB05934D4B06934FF003084B
:108640000B23ADF81C300DEB080301220893494BB6
:108650008DF803200993424601AB03A93846ADF8D3
:108660001080ADF828800B932DF0C2FA0028D9D0E5
:108670000298414D414C29F07EFD48B1029A404993
:1086800068682CF027F8236843F00803236009E0AA
:10869000029B002B4AD13A4968682CF08DFE236872
:1086A0005906F0D4029850B1C389A3F500739BB268
:1086B000C381C38903F4F0530BB92AF039F99DF84B
:1086C0000330002B37D023682E4968689A065EBFB6
:1086D000236843F0080323602CF06EFE32462A49DB
:1086E00068682CF083FE3A46284968682CF07EFEC4
:1086F000019A1AB1236843F008032360244968688B
:108700002CF074FE019850B1C389A3F500739BB29D
:10871000C381C38903F4F0530BB92AF009F9236824
:1087200013F0180F1BD0FFF729FF7BE719494046CC
:1087300024F0F0F9B6E72368D5F804809B0648BF1B
:1087400023684FF0000044BF43F0080323602AF081
:108750008CF80C49024640462BF0DDFFBEE7304660
:1087600014F0E2FC5EE700BF72CF050020CC0500EC
:1087700078CE05007DCE0500682D002048C200207F
:1087800087CE0500B6CE0500BFCE0500C9CE0500D8
:10879000D3CE050091CE050013B56946044619F005
:1087A000FBFD28B90749012024F0B4F902B010BD3F
:1087B000054B0649586822462BF08CFFFFF7DEFE7A
:1087C000F4E700BFA2CC0500682D0020D8CC05003E
:1087D00070B50D4D2A7806460C462AB101200B498A
:1087E00024F098F9002070BD08F0EEFF084B2E70C1
:1087F000186024B1E38903F500739BB2E381054B54
:1088000001201C60EFE700BF4CC2002077C90500C3
:1088100044C2002050C2002037B505460021052083
:108820008DF80610FFF7D4FF70B1084B1C6824B117
:10883000E38903F500739BB2E3810199284610F0A8
:10884000F3FC204603B030BD0446FAE744C20020E2
:1088500037B505460C4605200021FFF7B9FFD0B11A
:10886000214601A819F0C4FC024638B10B49012089
:1088700024F050F90024204603B030BD084B1C689A
:1088800024B1E38903F500739BB2E3810199284683
:1088900010F0CAFCEFE70446EDE700BF3BCF050050
:1088A00044C2002013B5002104208DF80610FFF704
:1088B0008FFF68B1074B1C6824B1E38903F500738F
:1088C0009BB2E381019810F0FFFC204602B010BD7E
:1088D0000446FAE744C2002013B50C4604200021E8
:1088E000FFF776FFC8B1214601A819F081FC0246C6
:1088F00038B10B49012024F00DF90024204602B0C4
:1089000010BD084B1C6824B1E38903F500739BB2CA
:10891000E381019810F0D8FCF0E70446EEE700BFD1
:108920003BCF050044C2002038B5124D2A880146CD
:108930004FF6FF70904215D00320FFF749FF78B142
:108940000D4B1C6824B1E38903F500739BB2E381EE
:1089500013212888FBF732FF10F0EEFC204638BDCB
:108960000446F5E7FDF7FEFCBDE83840084608F090
:108970009FBF00BFB42C002044C200202DE9FF415E
:1089800000220F46314980462BF0FEFE002230497E
:1089900006462BF0F9FE6946054619F0FDFC044633
:1089A00058B9294630462BF021FB2A49032024F0F0
:1089B000B1F8204604B0BDE8F0815EB1F389A3F5BB
:1089C00000739BB2F381F38903F4F05313B930467B
:1089D00029F0AEFF41460220FFF7FAFE80B90024DD
:1089E000002DE6D0EB89A3F500739BB2EB81EB89F8
:1089F00003F4F053002BDCD1284629F099FFD8E787
:108A00004821154829F01AFF04460028E7D0022320
:108A1000014602AA0020CDE902571FF0BDFEE389FE
:108A2000A3F500739BB2E381E38903F4F05313B918
:108A3000204629F07DFF094B1C68002CD0D0E3892B
:108A400003F500739BB2E381CAE700BFB9C9050013
:108A500021CC050019CA050039B7020044C2002024
:108A600070B504460E460020184924F07DF90546ED
:108A700010B90025284670BD224615492BF02AFE64
:108A80002846FEF7CDF9EB89A3F500739BB2EB8185
:108A9000EB8903F4F053044613B9284629F048FF44
:108AA000002CE6D031462046FFF768FFE389A3F5A6
:108AB00000739BB2E381E38903F4F0530546002B76
:108AC000D8D1204629F034FFD4E700BF04CE0500FA
:108AD00021CC05002DE97043064658B129F0F6F97E
:108AE000044638B932464E49032024F013F8204694
:108AF000BDE8708300224B4930462BF045FE04460A
:108B000029F0DCF998B95CB1E389A3F500739BB255
:108B1000E381E38903F4F05313B9204629F008FFF9
:108B200022464149032023F0F5FF0024DFE75CB132
:108B3000E389A3F500739BB2E381E38903F4F05367
:108B400013B9204629F0F4FE0022384930462BF0B4
:108B50001BFE2DF0ADFA02460B468046894632F0E8
:108B60008FF930B9002200234046494632F06AF9B5
:108B700018B1DFF8C8904FF0000800212C4829F008
:108B80005DFE0446002846D0002149EC108B0BF016
:108B900003F9E389A3F500739BB2E381E38903F44E
:108BA000F053054613B9204629F0C2FE294601209C
:108BB000FFF70EFE002830D008211E4829F03EFEA7
:108BC000044670B13146FEF7EFFCE389A3F500736C
:108BD0009BB2E381E38903F4F05313B9204629F0F3
:108BE000A7FE154B1C6824B1E38903F500739BB203
:108BF000E381002D3FF47BAFEB89A3F500739BB2BB
:108C0000EB81EB8903F4F053002B7FF470AF28461F
:108C100029F08EFE6BE70546C8E70446E9E700BF8A
:108C2000AECB0500E3CB050041CD0500B6CA05007B
:108C30004DB30200A5B8020044C2002000409F408E
:108C400030B500218FB0044609202BF003F8154DF4
:108C50000190024680B114496868FF23CDE90213F0
:108C6000002312498DF810302BF055FD01A81AF0A1
:108C70006BFC01A81AF06EFC01A81AF065FC01A8B3
:108C80001AF054FC22460A4968682BF023FD094B70
:108C900002221A70E38903F500739BB22046E38138
:108CA0000FB030BD682D00200300FFFFF126060045
:108CB000D0D405005CC2002019F00CBD19F01EBC18
:108CC00038B5054609B119F0A7FC0022124928461B
:108CD0002BF05AFD2CF005FC10B110482BF020F8B9
:108CE00004460146284619F097FC5CB1E389A3F5D8
:108CF00000739BB2E381E38903F4F05313B9204678
:108D000029F016FE012029F0B0FD0549024628464B
:108D1000BDE838402BF0FFBC61B60500A431060069
:108D200063D3050008B519F077FC002008BD0000EA
:108D300070B58EB0044601A80E4615461AF064FCC4
:108D4000D8B1204600220E492BF01EFD0446A0B1EA
:108D500032460C492BF0BEFC2A460B4920462BF02C
:108D6000B9FCE389A3F500739BB2E381E38903F4C3
:108D7000F05313B9204629F0DBFD0EB070BD00BFE3
:108D800074D0050078D0050087D0050010B58EB0EE
:108D9000044601A81AF038FC30B101A8214619F0A8
:108DA000AFFE01A81AF0C2FB0EB010BD38B50546E3
:108DB0002BF0F8F9044629F0A1F8A0B9214618488B
:108DC00024F0DAF914B90024204638BDE389A3F56C
:108DD00000739BB2E381E38913F4F055F3D120468D
:108DE00029F0A6FDEFE75CB1E389A3F500739BB220
:108DF000E381E38903F4F05313B9204629F098FD89
:108E00000849002023F0B0FF04460028DCD00021F0
:108E100019F006FF2A46044920462BF05BFCD3E7F5
:108E20005AD40500B2C9050081D4050038B50546FD
:108E30002BF0B8F9044629F061F8A0B9214618488A
:108E400024F09AF914B90024204638BDE389A3F52B
:108E500000739BB2E381E38913F4F055F3D120460C
:108E600029F066FDEFE75CB1E389A3F500739BB2DF
:108E7000E381E38903F4F05313B9204629F058FD48
:108E80000849002023F070FF04460028DCD00121AF
:108E900019F0C6FE2A46044920462BF01BFCD3E7F6
:108EA0005AD4050067D3050081D4050030B591B0D0
:108EB000044603A80D461AF0A7FB48B1002303A8F7
:108EC00000932A46214619F0B5FC03A81AF02EFBA0
:108ED000002011B030BD30B58FB0044601A80D465A
:108EE0001AF092FB58B11DB129462046FFF7DEFF6C
:108EF00001A8214619F004FE01A81AF017FB0FB0D3
:108F000030BD000030B58FB0054601A81AF07CFBDB
:108F100078B300211A4819F091FE044630B329466F
:108F200001A819F045FE2946012220462EF0FAF943
:108F3000054600B3014620462CF066F9EB89A3F5FF
:108F400000739BB2EB81EB8903F4F05313B928460D
:108F500029F0EEFCE389A3F500739BB2E381E3897A
:108F600003F4F05313B9204629F0E2FC01A81AF0EB
:108F7000DDFA0FB030BD034824F0DEF8EAE700BFA9
:108F80008CD4050092D405002DE9F04391B08146C0
:108F900003A8884616461F461AF036FBB8B10021D2
:108FA00018982BF027F9044628F0CCFF80B3304600
:108FB0002BF030F9064638462BF02CF907461B20DB
:108FC00029F060FB054628B903A81AF0AFFA11B0E2
:108FD000BDE8F0833B46324641462AF0A1F9012123
:108FE00018982BF007F92646074630462BF012F961
:108FF00080B200903B462A46494603A819F01AFC65
:109000004545E1D03A46314628462AF0C3FFDBE722
:109010000CB94546E9E7E389A3F500739BB2E38108
:10902000E38903F4F053002BF3D1204629F080FCB0
:10903000EFE700002DE9F04F8BB08246019129F057
:109040006FF820B9002630460BB0BDE8F08F03F072
:1090500035FB06460028F5D04FF000094FF0FF35EC
:109060000022514605A828F097FFCB462C46A8467B
:109070002F464A464946DDE905308342C0F0D78095
:10908000089850B1C289A2F5007292B2C281C28919
:1090900002F4F0520AB929F04BFCB4F1FF3F08BFCB
:1090A0005C46B8F1FF3F08BFA046002F09DD7A1EDD
:1090B000002150462AF077F9BB49024630462BF092
:1090C0002AFBBA482AF02CFEB949024630462BF05A
:1090D00022FB791CA8EB010250462AF064F9B5493D
:1090E000024630462BF017FB6FF0004221465046F7
:1090F0002AF059F907462AF082FA18B9AE493846DB
:109100002AF0DBF93A46AD4930462BF004FB691CE6
:1091100014BF2A1B6FF00042214650462AF043F943
:1091200004462AF06CFA18B9A34920462AF0C5F97A
:109130002246A34930462BF0EEFA6A1C00F0B980B3
:109140006FF00042294650462AF02DF902469D490B
:1091500030462BF0E0FA09F1FF324FF6FE739A42E7
:1091600040F2AB80022029F08DFA02469649304643
:109170002BF0D1FA6B1C00F0A4806FF00042691C48
:1091800050462AF010F9019B0446002B49D028F0E4
:1091900063FE0546002844D10246214605A828F072
:1091A000FBFE03F08BFA81461B2029F06BFA074681
:1091B0001B2029F067FA8046DDE905239A42C0F0BA
:1091C0008480089850B1C389A3F500739BB2C38112
:1091D000C38903F4F0530BB929F0AAFB5CB1E3890E
:1091E000A3F500739BB2E381E38903F4F05313B951
:1091F000204629F09DFB38462AF001FA002800F0AD
:10920000978038462DF0A9F9414607462AF0F2FB2F
:10921000394648462BF0C2F8414638462AF0E6FE69
:109220004C462246694930462BF075FA0BE70998FF
:1092300088B1C05C2F2812D1B4F1FF3F08BF5C4653
:10924000012A01F1010106D1022904D17B1C02D1BE
:109250003D463C465F46B8F1FF3F0DD119E03A2844
:1092600007D17B1C02F10102F5D0631CF3D1D84673
:109270000FE0B8F1FF3F16D0D84514DA631C40F078
:1092800090802F2805D9392803D830380A2303FBCA
:10929000090905A8CDE902210BF1010B28F0FEFB1D
:1092A000DDE90221E7E63F28F3D1601CF1D05D46FD
:1092B000EFE7022029F0E6F948E7484629F0DDFA11
:1092C00053E7022029F0DEF95DE7099B002B53D01C
:1092D0009B5C262B25D138462AF091F9C0B138463F
:1092E0002DF03BF9414605462AF084FB29464846C5
:1092F0002BF054F8414628462AF078FE1B2029F02E
:10930000C1F907461B2029F0BDF98046002504E07D
:1093100040462AF074F90028E1D105A828F0BEFBE8
:109320004AE765B93D2B31D1019DF6E7824611E050
:1093300040462AF064F900287FF463AF6CE7252BE0
:109340001BD105A828F0AAFB09980028EED0059BA0
:1093500010F803A005A828F0A1FB504624F03CF823
:1093600000014FFA80FA099808B1059BC05C24F00F
:1093700033F84AEA0000C3B255B101220DF11301DE
:1093800040468DF813302AF075F8CDE7252BD8D05C
:1093900001220DF1130138468DF813302AF06AF8D6
:1093A000B4E73F2883D074E793D505009CD505002A
:1093B000A0D50500FA2606000CD50500A7D50500A6
:1093C000ACD50500B5D50500BCD50500C1D5050057
:1093D0002DE9F04F93B0014604A81AF031FC28B9EA
:1093E0004FF0000B584613B0BDE8F08F9DF81B807E
:1093F000B8F1010F07D0B8F1180F04D04B49012084
:1094000023F088FBECE7BDF81530BDF81950BDF826
:109410001760DB0642BF2B4635461E4606FB08F3A7
:109420001F33B8F1010F4FEA63134FEA83030CBFF8
:1094300020271A2703FB05794846009329F09CF85A
:1094400083460028CCD028F09FFD422303704D2393
:1094500043700C238373331280F80290C3744FEA75
:1094600029292B12877280F8039043750123B8F1E4
:10947000010F83759DF81B300376009A867401BF37
:10948000FF238376C37603776B1E0446057502FBC4
:1094900003774FF000084545A4D09DF81B30012B01
:1094A0003BD04FF000090FFA88FAB14530D0524650
:1094B0000FFA89F104A81AF055FB9DF81B30DB0860
:1094C00009FB0373020AE0542344000C5A7098709D
:1094D00009F10109E9E700235B000FFA89F1019A1C
:1094E000039304A81AF03EFB09F10109039B00F065
:1094F0000100CA4543EA0003EED1029A02EBEA02F8
:109500000AF1080A02F8013CAAF10809B145E2DBB8
:10951000009B08F10108FF1ABDE70FFA88F30193D9
:10952000E3194FF0080A0293EEE700BF93D005005D
:1095300038B5FFF74DFF054610B90025284638BD60
:109540000AF0C4FEEB89A3F500739BB2EB81EB89B3
:1095500003F4F053044613B9284629F0E9F9002C26
:10956000EBD02146084829F02FFFE389A3F50073CB
:109570009BB2E381E38903F4F0530546002BDDD170
:10958000204629F0D5F9D9E7C1D0050010B5FFF77D
:10959000CFFF044668B120F0F3FFE389A3F5007321
:1095A0009BB2E381E38903F4F05313B9204629F019
:1095B000BFF90248BDE8104020F04EBAA3310600C2
:1095C00030B58FB00C460146684615461AF038FB98
:1095D00020B12AB221B268461AF0C4FA0FB030BDE9
:1095E00030B58FB00D46014668461AF029FB0028B9
:1095F0004CD0BDF91B20BDF91F309A4244DC03F06A
:109600005DF8044618B3BDF91B0029F036F920496E
:10961000024620462BF07FF8BDF91D0029F02DF9F8
:109620001C49024620462BF076F8BDF91F0029F0B0
:1096300024F91949024620462BF06DF8BDF92100A6
:1096400029F01BF91549024620462BF064F8C5B1F4
:1096500000226FF07F038DF81F208DF820308DF8E9
:1096600021208DF822304FF0FF327F2368468DF89D
:109670001B208DF81C308DF81D208DF81E301AF03F
:10968000A5FA20460FB030BD0024E0E70446F8E715
:10969000D0D20500D3D20500D6D20500D9D205001C
:1096A00070B58EB004460D460146684616461AF05F
:1096B000C7FA50B3BDF80530022D23F070039BB2FA
:1096C0001DD0032D1ED0012D08BF43F03003ADF88F
:1096D00005304EB1BDF80530DA064CBF83F04003CB
:1096E00083F02003ADF8053068461AF06FFAE3897D
:1096F00003F500739BB2E38120460EB070BD43F0CA
:109700006003E4E743F05003E1E70446F4E770B593
:109710008EB004460E460146684615461AF090FA89
:1097200070B16846ADF81660ADF818501AF04EFAF0
:10973000E38903F500739BB2E38120460EB070BD50
:109740000446FAE7F0B58FB004460E460146684677
:1097500015461F461AF074FA00B3012E9DF81A1030
:10976000A8BF0126012DA8BF012546EAE67666F3CB
:10977000010145EAE57565F3830187F3020767F3A5
:10978000051168468DF81A101AF020FAE38903F5DE
:1097900000739BB2E38120460FB0F0BD0446FAE7A8
:1097A0002DE9F0438FB004468846014668461646C8
:1097B0001D46169F1AF044FA002846D0404628F06D
:1097C000AFFC40B92249012023F0A4F9002420462F
:1097D0000FB0BDE8F083FF2E01D91E49F3E72846FC
:1097E00028F09EFC28B9284628F069FD08B91A49D6
:1097F000E9E77B1EFE2B01D91849E4E742461849E8
:1098000020462AF067FF2A46164920462AF062FFC2
:10981000384629F032F81449024620462AF07BFFE8
:10982000304629F02AF81149024620462AF073FFF3
:109830004FF6FE736846ADF814301AF0C7F9E389A5
:1098400003F500739BB2E381C1E70446BFE700BFA5
:10985000DCD20500F9D2050016D3050040D305007F
:109860004FD3050054D3050059D305005ED305003E
:109870002DE9F04317461D46421E47F6FE739A42F5
:109880008FB08146884602D84A1E9A4208D93D497F
:10989000012023F03FF9002420460FB0BDE8F083FB
:1098A0003846FCF763FD044620B93749012023F010
:1098B00031F9F1E7284628F009FBD8B100223349F5
:1098C00028462AF061FF00220446314928462AF042
:1098D0005BFF25460646284628F010FB044680B963
:1098E0002A462C49012023F015F9314628462AF052
:1098F0007DFBD1E7EB8903F500739BB2EB81064654
:10990000E9E736B1304628F0F9FA044608B932469C
:10991000E7E72149002023F027FA04460028BBD0BE
:1099200000234FF0FF32CDE903238DF805308DF889
:1099300006304FF6FF730593069B1849009003F419
:10994000400343F07F4343F470230693144B079383
:109950008023ADF820308DF822302A4601238DF87F
:109960000430ADF80790ADF809808DF80B702AF03F
:10997000B1FE32460B4900982AF0ACFE68461AF058
:1099800025F9B2E7ADD10500BAD10500C6D1050071
:10999000CFD10500D8D10500B8D005000CD2050004
:1099A0007FFF7F0016D205002DE9F04192B00646F8
:1099B0000D46014604A814461AF042F94FF000087B
:1099C000002869D00DF10A0202A904A8ADF80C50D4
:1099D000ADF80E40ADF80880ADF80A8019F020FF10
:1099E0000DF10E0203A904A819F01AFFBDF9083001
:1099F000BDF90A20BDF90C50BDF90E40ED1AA41AAC
:109A0000119B2246294604A89847DDE9077345457E
:109A1000079326DDBDF81920013A12B26B1E0092A1
:109A20001BB24246414604A80F9DA847002C26DDE4
:109A3000BDF81730013C013B24B200941BB2002258
:109A4000002104A80F9CA04704A807971AF0BEF8AD
:109A5000F38903F500739BB2F381304612B0BDE881
:109A6000F081E3D0BDF81920BDF81710013A4B1E64
:109A700012B2294400921BB2424609B2D3E7E3D0A6
:109A8000BDF81910BDF817300A190139013B09B2A8
:109A900000911BB212B2D3E70646DEE7F0B58FB0F5
:109AA00004460E460146684615461F461AF0C8F899
:109AB000E0B1B7B9039B36B22DB22A4631466846AB
:109AC0001AF070F86846ADF81660ADF818501AF044
:109AD0007DF8E38903F500739BB2E38120460FB064
:109AE000F0BD38462AF096FB0346E4E70446F5E766
:109AF0002DE9F04F9DB004460D4601460EA8CDE974
:109B000005231AF09DF820B9002420461DB0BDE8B9
:109B1000F08F284628F0DAF920B97649012022F0A2
:109B2000F9FFF1E70022744928462AF02DFE2BF0B8
:109B30001BFB00227149029028462AF025FE2BF0DB
:109B400013FB00226E49009028462AF01DFE2BF0E0
:109B50000BFB002201906B4928462AF015FE804637
:109B60002AF058FB0390B8F1000F0ED0B8F80E3071
:109B7000A3F500739BB2A8F80E30B8F80E3003F4CA
:109B8000F05313B9404628F0D3FE284600225E4920
:109B90002AF0FAFD054628F075F9A8B1029B002BC2
:109BA00018DC5A49012022F0B5FF002DACD0EB891A
:109BB000A3F500739BB2EB81EC8914F4F054A3D1AC
:109BC000284628F0B5FEA0E7284628F0A9FA002884
:109BD000E4D1E6E7009B002BE3DD019B202BE0DCDA
:109BE000284629F031FA07465DB1EB89A3F50073E9
:109BF0009BB2EB81EB8903F4F05313B9284628F0AC
:109C000097FE019B012BB8BF01239B4609AB0022A5
:109C10001846394628F0C0F9012202FA0BF2531E09
:109C20000025049309AB2E46A946AA4607935E4534
:109C30005BDADDE909239A4202D2009B994522DBD7
:109C40000C9850B1C389A3F500739BB2C381C3893B
:109C500003F4F0530BB928F06BFE5FB1FB89A3F559
:109C600000739BB2FB81FB8903F4F05313B93846B0
:109C700028F05EFE0EA819F0A9FFE38903F5007332
:109C80009BB2E38141E72B020D9D0DB1099AAD5CBA
:109C9000079808361D4327F001FFB345F3DCA6EB18
:109CA0000B06049A25FA06F31340B8F1000F02D010
:109CB000039A9A420DD0019A012A01DC9BB1119BB3
:109CC000069A05994A44514412B209B20EA819F0F5
:109CD00069FF029B0AF1010A5345DCBF09F1010942
:109CE0004FF0000AA3E7129BEAE7009B9945D6DBF9
:109CF000A6E700BF33D205005CD2050048D30500BB
:109D000062D2050066D20500C3F9050072D20500D3
:109D1000F0B5DBB004460D4601460CA819F090FFE3
:109D200018B9002420465BB0F0BD284628F023FA7D
:109D30000028F6D02946012201A829F0F0F91AAE30
:109D40000025374601A823F0E0FC08B1802D16D18C
:109D500001A823F087FC802D03D140210D4823F07A
:109D6000EBF93A4669100CA819F07AFD0CA819F025
:109D70002DFFE38903F500739BB2E381D2E701A8CD
:109D80002BF006FA26F8020B01A8013523F097FC08
:109D9000D8E700BF9CD205002DE9F04F9FB00446E4
:109DA0000E46014610A8039219F04AFF20B900247C
:109DB00020461FB0BDE8F08F304628F0DCF90028BF
:109DC000F5D03146012205A829F0A9F9002605A8F9
:109DD00023F09BFCC0B905A823F044FC039B53B1BE
:109DE0002DB200950FFA8AF3BDF95820BDF956102F
:109DF00010A819F03BFE10A819F0E8FEE38903F55E
:109E000000739BB2E381D3E705A82BF0C1F9F307F8
:109E1000834616D5012E0FFA87F90FFA80F816D06F
:109E2000CDF800804B46BDF95820BDF9561010A85A
:109E300019F01CFEAB465D46ADF85690ADF8588063
:109E4000BB4605A8013623F03AFC5F46BFE7BA4699
:109E5000F1E770B590B004460E46014602A81546DB
:109E600019F0EEFEC8B136B22DB23346BDF920204E
:109E7000BDF91E10009502A819F0F8FD02A8ADF872
:109E80001E60ADF8205019F0A1FEE38903F50073C0
:109E90009BB2E381204610B070BD0446FAE7F0B5EE
:109EA00091B004460D46014602A816461F4619F019
:109EB000C7FE98B1BDF95830009332B23BB229B217
:109EC00002A819F0D3FD02A819F080FEE38903F57A
:109ED00000739BB2E381204611B0F0BD0446FAE75F
:109EE0002DE9F04F95B004460D46014606A819F03D
:109EF000A7FE002839D0BDF92C30023338D100221A
:109F0000374920462AF040FC0022364906462046C2
:109F10002AF03AFC2BF028F9804628462BF03CFB2F
:109F200000220146814601A828F036F80027DFF814
:109F3000B8A03C464FF0C00BDDE9013293421BD381
:109F4000049850B1C389A3F500739BB2C381C38940
:109F500003F4F0530BB928F0EBFC484631462AF0E5
:109F600045F8BC422046B8BF384615B0BDE8F08F72
:109F70004FF000084646D0E7059D35B1ED5C0A2D4F
:109F800003D1A742B8BF27460024BDF92C20002AE0
:109F90000FDD203DEBB25E2B97BF1AF81530002382
:109FA00013FB02F3B3FBFBF31C4401A827F076FD7F
:109FB000C2E7531C01D10434F7E70232F5D1304631
:109FC00028F0AEF840B14545EFDBA5EB080130467F
:109FD00029F085F90444E8E730462AF01BF9F9E74F
:109FE00054D305005ED3050058EA05002DE9F04F73
:109FF000A5B000AF0D46F862014607F15800BA62FD
:10A000001C4619F01DFE002800F06082B7F96C3084
:10A01000002B05DD7B624FF0000BC7E907BB21E099
:10A020005E1C00F08380023340F085800022A0494E
:10A03000F86A2AF0A9FB0022F8619E49F86A2AF022
:10A04000A3FB00229C493862F86A2AF09DFB2BF0A2
:10A050008BF8002278629949F86A2AF095FB2BF078
:10A0600083F8834697F87220B7F85D303B8102F0A1
:10A07000300110299BB263D183F03003A7F85D3023
:10A08000BB6AB7F85F10BC620133CC1A02F003025E
:10A09000012A0FD82946F86AFFF722FF97F8723095
:10A0A00003F0030303FB0000BB6A00EBD070A3EBDB
:10A0B0006003BB6297F87230C3F38102012A08D8AB
:10A0C0007A6A03F0030303FB022303EBD373A4EBCD
:10A0D0006304B7F85F307B61B7F86130BB61B7F8F4
:10A0E0005D30D80648BFD7E90523284648BFC7E9F1
:10A0F00005322BF051FA0022F860014607F13000DA
:10A1000027F04AFFBE6AD7E90C239A4280F0A38069
:10A110003B6C9BB313F80290B9F10A0F2FD17B6A05
:10A1200007F130001C4427F0B9FCEBE706234FF0A1
:10A13000000B7B6271E74FF0000BC7F824B06CE7AF
:10A1400020290ED183F06003A7F85D30BB6AB7F811
:10A150005F100133CB1ABB62B7F8613001341C1BAE
:10A1600094E7302992D183F05003B7F86110A7F833
:10A170005D30631CCB1ABC6ABB6287E79946B7F9AE
:10A180006C80B8F1000F40F38C80A9F120095FFAD0
:10A1900089F25E2A9BBF4A4B13F81930002313FB48
:10A1A00008F39CBFC021B3FBF1F33B613B695B4209
:10A1B000B34249DA7B699E4246DAC8F10003A34202
:10A1C00042DABB699C423FDA5E2A3DD800233C4A12
:10A1D0001D4699455BDC02EB4902C7F800D0537875
:10A1E0007B60384B88B000201D44EA4681466023DE
:10A1F0007A68914526DA2A7895F801C04FF0300E3A
:10A2000002F07F0218FB02E2B2FBF3F232442AF8BA
:10A2100010200AEB40010CF07F0218FB02E21CF058
:10A22000800FB2FBF3F222444A8000F1020034D0E6
:10A230004110524607F1580019F012FB22F0DEF8E7
:10A24000602350B3D7F800D03B691E4422F0D6F803
:10A25000002800F02881F86B002840F02981D7E918
:10A260000712F86829F096FE3B89A7F85D3007F1E0
:10A27000580019F0ABFCFB6AFA6ADB8903F500733E
:10A280009BB2D381F86A9437BD46BDE8F08F02EBEC
:10A290004301013349780D449BE709F10209023576
:10A2A000A6E7B8F1FF3F5FD1F11C0DDA0436CDE728
:10A2B0004FD3050054D3050059D305005ED30500E4
:10A2C00058EA05003CD605007B699E42EEDA621D25
:10A2D000ECDBBB699C42E9DAA9F12109B9F15E0F17
:10A2E000E4D8052399FBF3F303EB8302A9EB0209FE
:10A2F00009EB49023A614FF00609754A09FB03F37D
:10A3000002EB430906F1010A33B200257B600FFA24
:10A310008AFA39F8028B3B6948FA03F818F0040FFF
:10A3200007D062197B6E796812B207F1580019F0F4
:10A3300039FC18F0020F07D02A197B6E12B2514671
:10A3400007F1580019F02EFC18F0010F08D02A1957
:10A35000B11C7B6E12B209B207F1580019F022FC51
:10A360000135062DD5D1A1E718F1020F7FF46EAFAC
:10A37000386A27F0D5FE00285DD0CB4500F39180E8
:10A3800007F144050022396A284627F005FE4FF000
:10A390000008A9EB0B09796CBB6C7A6D994203D26A
:10A3A000FB6C0B444B453DDB002A42D0555C386DBD
:10A3B00050B1C389A3F500739BB2C381C38903F471
:10A3C000F0530BB928F0B4FA6B42B3423DDA7B6923
:10A3D0009E423ADA7B6A5B42A34236DABB699C4210
:10A3E00033DA7B6AF96908FB03F807F1440A4FEA9C
:10A3F000D802504627F0D0FD08F007084FF00009BA
:10A40000C7F804A0A94545DB386DF0B1C389A3F5B1
:10A4100000739BB2C381C38903F4F053ABB928F036
:10A4200087FA12E002B1525C2846904427F036FBCE
:10A43000B1E71546BBE7386A29F0ECFEA9EB0B083B
:10A44000CB45054600FB08F8BEDD2E44FEE67B6DDD
:10A4500073B17A6C9B5C03FA08F31B0608D504EB16
:10A460000A027B6E396912B207F1580019F09AFBA3
:10A4700008F10108B8F1080F04D1786827F00EFB45
:10A480004FF000080AF1010A7B6A5345DFDC09F14D
:10A490000109B7E706EB09031BB24FF0000A3B6165
:10A4A000F2E70025D1E707F1300027F0F7FA2AE6B6
:10A4B000C389A3F500739BB2C381C38903F4F0532E
:10A4C000002B7FF4CCAE28F033FAC8E6F862D9E668
:10A4D00058B805002DE9F04F99B00AAC81460F46F7
:10A4E0000146204616461D4619F0AAFB002800F03A
:10A4F0008980229BADF826300DF1220208A9204662
:10A50000ADF82070ADF82260ADF8245019F088F94C
:10A510000DF1260209A9204619F082F9BDF92000A3
:10A52000BDF92420BDF92210BDF926308518121A74
:10A53000CE1802EBD27A5B1A4FEA6A0A013203EBB9
:10A54000D378B8BFCAF1000A4FEA68080133B8BF30
:10A55000C8F1000808FB08F30393039A0AFB0AF307
:10A5600005EBD57506EBD6766D1076100493534344
:10A570000793009605EB0A033246A5EB0A01204635
:10A5800019F05CF80023CDE905340127B8450DDA50
:10A590000AA819F01BFBB9F80E3003F500739BB243
:10A5A000A9F80E30484619B0BDE8F08F059B049A13
:10A5B0005C1E07FB07F3AAEB04045343002C17DCD3
:10A5C000F21BAAEB040305EB040BA5EB040A5146AE
:10A5D000059300925B46069819F030F8F21951463F
:10A5E00000925B46069819F029F80137A246CDE79C
:10A5F000039904FB04F201FB023207999142DFDA6E
:10A60000013CDBE78146CDE737B505461C461344E0
:10A610000093121B0B19091BFFF75CFFEB8903F575
:10A6200000739BB22846EB8103B030BDF0B593B008
:10A6300004460F46014604A816461D4619F000FBC5
:10A64000002849D0189BADF80E300DF10A0202A97E
:10A6500004A8ADF80870ADF80A60ADF80C5019F018
:10A66000DFF80DF10E0203A904A819F0D9F8BDF91D
:10A670000A200092BDF90C30BDF9081004A818F0AA
:10A68000DDFFBDF90C30BDF90E2000921946BDF971
:10A690000A2004A818F0D2FFBDF90E200092BDF9DF
:10A6A0000C30BDF9081004A818F0C8FFBDF9083037
:10A6B000BDF90A2000921946BDF90E2004A818F031
:10A6C000BDFF04A819F082FAE38903F500739BB279
:10A6D000E381204613B0F0BD0446FAE7F0B593B02D
:10A6E00004460F46014604A816461D4619F0A8FA6E
:10A6F00058B3189BADF80E300DF10A0202A904A858
:10A70000ADF80870ADF80A60ADF80C5019F088F893
:10A710000DF10E0203A904A819F082F8BDF90E305C
:10A720000093BDF90A20BDF90C30BDF9081004A84A
:10A7300018F084FF04A819F049FAE38903F50073BF
:10A740009BB2E381204613B0F0BD0446FAE730B572
:10A7500091B004460D46014602A819F071FA78B38B
:10A760008DB100234FF0FF32CDE90523ADF8203045
:10A770009DF8223023F03F034FF6FF7243F00F03A2
:10A7800007928DF82230DDE90553BDF811200593BD
:10A79000013ABDF80F3012B20092013B00221BB209
:10A7A000114602A818F04AFF02A8059519F00EFA02
:10A7B000E38903F500739BB2E381204611B030BDFD
:10A7C0000446FAE72DE9F04F9DB00EAD03900F4619
:10A7D0000146284616461C4619F032FA002800F0B9
:10A7E000C680269BADF836300DF132020CA9284602
:10A7F000ADF83070ADF83440ADF8326019F010F8B3
:10A800000DF136020DA9284619F00AF8BDF93040BD
:10A81000BDF93420BDF93200A31803EBD3734FEA1E
:10A82000630ABDF93630C118121B01EBD1711B1A36
:10A83000491002EBD27464100491013203EBD3711E
:10A84000B8BF64424FEA610B0133B8BFCBF1000BD4
:10A850000BFB0BF30793079A04FB04F30893534392
:10A860000B93049A119BAAEB0401284618F033FFBE
:10A87000119B049A0AEB0401284618F02CFF0023D0
:10A8800001270993BB450DDA0EA819F09FF9039B28
:10A89000039ADB8903F500739BB2D38103981DB043
:10A8A000BDE8F08F099B089A5E1E07FB07F3A61B05
:10A8B0005343002E2BDCA31B0993AAEB060305933D
:10A8C000049BA3EB07090AEB06030693049B03EB27
:10A8D0000708A31B012B24DC119B05994A46284637
:10A8E00018F0F9FE119B06994A46284618F0F3FE27
:10A8F000119B05994246284618F0EDFE119B0699DA
:10A900004246284618F0E7FE01373446BAE7079971
:10A9100006FB06F201FB02320B999142CBDA013EB3
:10A92000C7E7AAEB0403544401334A460599CDF81E
:10A9300000902846013C0A9318F080FE23464A46C0
:10A940000699CDF80090284618F078FE0A9B0599E4
:10A95000CDF800804246284618F070FECDF8008001
:10A96000234642460699284618F068FECCE7039035
:10A9700094E737B505461C4613440093121B0B1988
:10A98000091BFFF71FFFEB8903F500739BB22846F5
:10A99000EB8103B030BD00002DE9F0478AB080465E
:10A9A00027F0BEFB044638B96149032022F0B2F813
:10A9B00020460AB0BDE8F08700224146684627F0ED
:10A9C000EBFA00273C463E46B9463D46DDE90032FB
:10A9D000934212D3039850B1C389A3F500739BB27D
:10A9E000C381C38903F4F0530BB927F0A1FF01F031
:10A9F00065FE0546D8B90024DAE7049A6AB1D35C4B
:10AA00000A2B0AD155EA090308BF012709F10109F8
:10AA10000025684627F042F8D8E7A14505F1010571
:10AA2000A8BF09F10104AE42B8BF2E46F1E7304697
:10AA300027F023FF3F490246284629F06CFE2046B6
:10AA400027F01BFF3C490246284629F064FE04FB20
:10AA500006F007300021C01029F0FCF8044668B960
:10AA6000EB89A3F500739BB2EB81EB8903F4F05300
:10AA7000002BC0D1284627F05BFF99E73A464146B4
:10AA8000684627F089FA4FF0000847464FF08009E2
:10AA9000DDE90032934213D3039850B1C389A3F583
:10AAA00000739BB2C381C38903F4F0530BB927F041
:10AAB0003FFF22462149284629F02DFE2C4677E704
:10AAC000049A5AB1D35C0A2B06D108F10108002779
:10AAD000684626F0E3FFDBE7202B26D0204627F050
:10AAE0001FFB10B306FB087A21464FEADA0205A8DD
:10AAF00027F052FA099909B1059BC95C0AF0070AC7
:10AB000049FA0AFA41EA0A0105A8C9B226F00EFF7D
:10AB1000089850B1C389A3F500739BB2C381C38960
:10AB200003F4F0530BB927F003FF0137D0E700BF60
:10AB300020D205005CD2050048D30500C3F905000A
:10AB40002DE9F04316461D46421E47F6FE739A4213
:10AB50008FB080460F4602D84A1E9A4205D97749DF
:10AB6000012021F0D7FF002408E03046FBF7FEFB70
:10AB7000044638B97249012021F0CCFF20460FB0BD
:10AB8000BDE8F0836F49002022F0EEF8044600286B
:10AB9000F4D04FF000094FF0FF33CDE903394FF601
:10ABA000FF730593069B009003F4400343F07F433B
:10ABB00043F470230693644B0793284680238DF853
:10ABC00005908DF80690ADF820308DF822308DF884
:10ABD0000490ADF80780ADF809708DF80B6027F090
:10ABE00075F9002865D04A465849284629F0CCFD19
:10ABF0002AF077FC28B1BDF8053043F00103ADF829
:10AC0000053000225249284629F0BEFD2AF069FC91
:10AC100028B1BDF8053043F00403ADF8053000223B
:10AC20004C49284629F0B0FD2AF05BFC28B1BDF85C
:10AC3000053043F00803ADF80530002246492846A8
:10AC400029F0A2FD2AF04DFC88B19DF80B000128E7
:10AC50000BD1BDF8053043F00203ADF80530BDF867
:10AC600009305B0703D03D497BE73D4978E728463B
:10AC700000223C4929F088FD0546D0B13A4928F028
:10AC8000BDF950B93949284628F0B8F950BBBDF88C
:10AC9000053043F08003ADF80530EB89A3F5007370
:10ACA0009BB2EB81EB8903F4F05313B9284627F0EC
:10ACB0003FFEBDF80900BDF8073043439DF80B0087
:10ACC00058430730C0100AF013FC294A05460146D4
:10ACD000009829F010FF294629F088F9684618F0F5
:10ACE00075FF4BE72349284628F088F920B9BDF8BD
:10ACF000053043F48073CEE71F49284628F07EF9DB
:10AD000020B9BDF8053043F4C073C4E71B49284699
:10AD100028F074F920B9BDF8053043F40073BAE7A0
:10AD20001749284628F06AF920B9BDF8053043F4E0
:10AD30002073B0E7134822F0FFF9AEE7ADD105006C
:10AD4000BAD10500B8D005007FFF7F00DAD005003A
:10AD5000E1D00500E5D00500F1D005002FD10500B8
:10AD6000FFD0050068D1050074D1050078D1050039
:10AD7000C3F905007CD1050080D1050084D1050010
:10AD800088D105008CD1050008B500222DED028B7D
:10AD9000B0EE408AF0EE608A002351EC100B30F0E8
:10ADA0005BF898B1B0EE480AF0EE680A2DF01CFE90
:10ADB0000B4B51EC100B00222FF0C8FDBDEC028BA9
:10ADC00041EC100BBDE808402DF08ABDBDEC028BB4
:10ADD0009FED010B08BD00BF000000000000F87FE0
:10ADE0000000E03F00000000F8B555EC104B25F0E6
:10ADF00000474FF0FF32284B2046394630F040F8EC
:10AE000060B94FF0FF32244B2046394630F02EF81F
:10AE100020B9B5F1004F08BF002C05D145EC104B0F
:10AE2000BDE8F84027F017BD002200232046294640
:10AE30002FF0FEFFC8B912A1D1E900012B4622462E
:10AE40002FF0CEFB06460F4630F0E0F804460D46E4
:10AE500054EA05030DD100220023304639462FF075
:10AE6000E7FF30B19FED080BDAE709A1D1E9000156
:10AE7000E4E720462946BDE8F84027F012BD00BFB0
:10AE80002083E4FFFFFFDF3F0000000000000080A0
:10AE90002083E4FFFFFFDFBFFFFFEF7F2DF01CBD2E
:10AEA0002DF0FEB92DF0B8BCF0B585B000AF002391
:10AEB000391D06467B6028F0FFFB0446F0B930469A
:10AEC00029F0FEFD0546786021F0A0FA05F58073B3
:10AED000834208D91949012021F01CFE2546284645
:10AEE0001437BD46F0BDEB1D23F00703ADEB030D9A
:10AEF0006C462A462146304629F0D2FD7B68104830
:10AF0000FB60002207F10801BC6018F023FF00235A
:10AF100039463B60F5F7A8FF3E68054626B9094863
:10AF200022F02AF93546DAE77B680548BC603246EC
:10AF300007F10801FB6018F00DFFD0E725B505000B
:10AF4000F3630200F0CF0500F0B583B000AF00233B
:10AF5000391D06467B6028F0AFFB0446F0B9304649
:10AF600029F0AEFD0546786021F050FA05F58073B2
:10AF7000834208D91649012021F0CCFD25462846F8
:10AF80000C37BD46F0BDEB1D23F00703ADEB030D01
:10AF90006C462A462146304629F082FD00231A4697
:10AFA0007968204618F0C9FF002339463B60F5F761
:10AFB0005BFF3E68054626B9064822F0DDF83546B7
:10AFC000DDE73B46044A7968204618F0B6FFD6E72D
:10AFD00025B50500F0CF05000B64020013B5002273
:10AFE0001B49044629F0D0FB2AF07BFA28B91949FD
:10AFF000012021F08FFD02B010BD00222046114635
:10B0000005F0AAFD044600B3134BC31A1B1101330C
:10B010009BB20DF106011148ADF806301CF06EFE32
:10B0200018B90F49012021F075FD5CB1E389A3F542
:10B0300000739BB2E381E38903F4F05313B9204614
:10B0400027F076FC05F01EFFD5E70346E1E700BFD9
:10B05000D7D50500C7D50500882D0020F35E040074
:10B06000DFD5050007B50123CDE9002353EC102BF4
:10B0700005F0A6FD03B05DF804FB2DE9F34105469C
:10B0800008460C46904657EC106B10F047FB002228
:10B09000002351EC100B2FF0CBFE38B9CDE9008026
:10B0A00032463B462146284605F08AFD02B0BDE8FF
:10B0B000F08100002DE9F0439DB000AF00230E4663
:10B0C00007F108018046BB6028F0F6FA0546F8B99A
:10B0D000404629F0F5FC0446B86021F097F904F5E4
:10B0E0008073834209D96149012021F013FDA846EC
:10B0F00040467437BD46BDE8F083E31D23F00703E7
:10B10000ADEB030D6D4622462946404629F0C8FCAA
:10B11000012E01D1142000E0F0104FF00009391D7C
:10B12000C7F80490F5F7A0FE7C68804624B9504823
:10B1300022F022F8A046DBE7012E78D15C224946B6
:10B1400007F11400BE68F4F7EDF94A4BFB6103F117
:10B1500088333B6203F12943A3F59613A3F68B636F
:10B160007B62A3F18833BB62434BFB622EB1324654
:10B17000294607F1140016F0BFFF7A69B969530F29
:10B1800043EAC1031BBAFB60D30002F03F02372A37
:10B190001BBA94BFC2F13802C2F1780237493B6151
:10B1A00007F1140016F0A8FF082207F10C0107F1BF
:10B1B000140016F0A1FFFB7F2370FB8B6370FB690B
:10B1C0001B0AA370FB69E37097F8233023717B8C13
:10B1D00063713B6A1B0AA3713B6AE37197F82730DE
:10B1E0002372FB8C63727B6A1B0AA3727B6AE37215
:10B1F00097F82B3023737B8D6373BB6A1B0AA37391
:10B20000BB6AE37397F82F302374FB8D6374FB6A7A
:10B210001B0AA374FB6AE37400231A4607F11401A6
:10B22000194401335D2B3FF463AF0A70F6E7E02E5B
:10B2300006D101232246B968284616F093FE57E747
:10B24000B6F5807F01D14B46F4E7B6F5C07F06D155
:10B2500001232246B968284616F0F2FC48E7B6F505
:10B26000007F7FF445AF4B46F3E700BF25B50500EF
:10B27000F0CF050001234567F0E1D2C3FCD50500FE
:10B28000024B03495868002229F07EBA682D00203D
:10B290006DC9050010B51D4C2378834206D00246C7
:10B2A0001B490420BDE8104021F034BC002323706A
:10B2B000184C206890B129B3114603F03BFC20687C
:10B2C00050B1C389A3F500739BB2C381C38903F452
:10B2D000F0530BB927F02CFB002323600E4C2068A1
:10B2E00050B1C389A3F500739BB2C381C38903F432
:10B2F000F0530BB927F01CFB00232360074B0122FE
:10B300001A7010BD114603F075FCD8E74CC200203E
:10B310003CC9050044C2002050C2002054C2002095
:10B3200010B50A460C460021FFF7B4FF6CB1E38963
:10B33000A3F500739BB2E381E38903F4F05323B9CF
:10B340002046BDE8104027F0F3BA10BD10B5094BF8
:10B350001C78012C0CD100210846FCF725F9064881
:10B3600028F0DEFC01462046BDE81040FFF7D8BFBC
:10B3700010BD00BF4CC20020CACB05000A46002108
:10B38000FFF788BF73B500224149054629F0FCF953
:10B3900029F0EAFE3F4B404906460322586829F04F
:10B3A000F3F9044678B12A46B1B229F01FF9E389CE
:10B3B000A3F500739BB2E381E38903F4F05313B95F
:10B3C000204627F0B5FA00223449284629F0DCF956
:10B3D00029F0CAFE80B2002846D129460820FDF790
:10B3E000F7F918B90024204602B070BD2C4B1C6838
:10B3F00024B1E38903F500739BB2E381294E3388BE
:10B400004FF6FF729A4207D1274828F089FC01467F
:10B410000820FFF785FFE6E700221D49284629F0AE
:10B42000B3F929F0A1FE013080B2ADF80400ADF807
:10B43000060001A930880FF07DF80DF097FE054653
:10B440000028D0D001460820FFF798FFEB89A3F52C
:10B4500000739BB2EB81EB8903F4F053002BC2D154
:10B46000284627F065FABEE700210920FDF7B0F96C
:10B470000028B7D00A4B1C6824B1E38903F5007398
:10B480009BB2E381012128460EF000FBABE700BF31
:10B49000E5C90500682D0020F2C90500CBC90500EB
:10B4A00044C20020B42C0020D7C9050070B5014665
:10B4B00006460720FDF78CF900283AD01E4B1C6881
:10B4C00024B1E38903F500739BB2E3811B4D2B8804
:10B4D0004FF6FF729A4208D1194828F021FC014624
:10B4E0000720FFF71DFF204670BD0022154930469A
:10B4F00029F04AF929F038FE2B8881B2002218463B
:10B500000FF016F80DF032FE05460028EBD001468C
:10B510000720FFF733FFEB89A3F500739BB2EB81A4
:10B52000EB8903F4F053002BDDD1284627F000FA15
:10B53000D9E70446D7E700BF44C20020B42C00205E
:10B54000D7C90500E5C905002DE9F04F85B088464B
:10B5500000AF00230646394640463B6028F0ACF871
:10B560000546F8B9404629F0ABFA0446386020F0A9
:10B570004DFF04F58073834209D94249012021F02F
:10B58000C9FA2C4620461437BD46BDE8F08FE31DAE
:10B5900023F00703ADEB030D6D46224629464046D6
:10B5A00029F07EFA00210620FDF712F908B90446B9
:10B5B000E8E7354B1C6824B1E38903F500739BB2BF
:10B5C000E381324B1A884FF6FF719142984607D1BA
:10B5D0002F4828F0A5FB01460620FFF7A1FED1E782
:10B5E00000222C49D7F80090304629F0CDF829F0F8
:10B5F000BBFD00221FFA80FA2749304629F0C4F823
:10B60000064600283CD00022244929F0BDF829F044
:10B6100068FFF389A3F500739BB2F381F38903F408
:10B62000F053834613B9304627F082F900239B4537
:10B630003B8114BF022301233B71391D0123B8F85C
:10B6400000007B71FD60A7F806A0A7F80A900EF035
:10B650001BFA0DF08BFD0546002893D0014606200D
:10B66000FFF78CFEEB89A3F500739BB2EB81EB89AE
:10B6700003F4F053002B85D1284627F059F981E7D0
:10B680008346D3E725B5050044C20020B42C002032
:10B69000D7C90500E5C90500F9C9050004CA0500B8
:10B6A00038B50D4601460A20FDF792F8002839D03A
:10B6B0001D4B1C6824B1E38903F500739BB2E38141
:10B6C0001A4B1A884FF6FF71914208D1184828F09A
:10B6D00027FB01460A20FFF723FE204638BD1888C5
:10B6E000144B1B7880B2DBB100232A461946F8F7C9
:10B6F0002DFE0DF03BFD05460028EED001460A2048
:10B70000FFF73CFEEB89A3F500739BB2EB81EB895D
:10B7100003F4F053002BE0D1284627F009F9DCE7C9
:10B720000820E6E70446D8E744C20020B42C0020F5
:10B73000D7C9050028BE0020F0B58BB06D460C4679
:10B74000294616F029FE002800F08D8000220123F2
:10B7500095E80300ADF818208DF81830A023ADF857
:10B760001A30454BADF80C10CDE90732434B02902F
:10B77000090C58688DF80E104149099229F004F817
:10B7800029F0F2FCC3074CBF3E4B3F4B08932046C9
:10B790004FF0C873099326F099FB002841D000228E
:10B7A0003A49204628F0F0FF2AF082FC02460B4678
:10B7B00006460F462FF064FB90B90022344B30460A
:10B7C00039462FF0C3F82AA3D3E900232FF0E8F974
:10B7D0000022304B2EF004FF2FF090FBADF820003C
:10B7E00000222D49204628F0CFFF2AF061FC0246B6
:10B7F0000B4604460D462FF043FB90B90022244B24
:10B80000204629462FF0A2F819A3D3E900232FF0F0
:10B81000C7F900221F4B2EF0E3FE2FF06FFBADF8AF
:10B82000220002AB93E80300ADF81410090C049059
:10B830008DF8161008AA06A904A80EF07DFE0DF0DA
:10B8400095FC044678B101460220FFF797FDE38995
:10B85000A3F500739BB2E381E38903F4F05313B9BA
:10B86000204627F065F80BB0F0BD00BFAFF30080B5
:10B87000000000000088934090000400682D002024
:10B8800030CD0500900120031000A00018CD050068
:10B8900000408F400000E03F24CD05000A46012112
:10B8A000FFF7F8BC38B5124B1C78012C05461DD1AA
:10B8B00000210846FBF778FE21460E4828F083FE5B
:10B8C000044608F0B5F95CB1E389A3F500739BB2B7
:10B8D000E381E38903F4F05313B9204627F028F8F5
:10B8E00029460120BDE83840FFF7D8BF38BD00BF6A
:10B8F0004CC2002050C200207CDF70472DE9F04F81
:10B90000AC4D85B02B6800AF044603F00403084635
:10B910000E463B6026F0DAFA002800F0BC800022D8
:10B92000A549304628F030FFB0B129F01DFC4FF496
:10B930007A73584340F2712390FBF3F080B2B0F574
:10B94000804F9E4B28BF4FF4804020281A8838BF74
:10B950002020824218BF188000229949304628F0E2
:10B9600013FF38B129F0BDFD2B68002875D023F4F2
:10B9700000632B6000229349304628F005FF38B160
:10B9800029F0AFFD2B6800286AD023F480532B6088
:10B9900000228D49304628F0F7FE8146002800F04D
:10B9A0008480002307F10C01FB6027F085FE8046B0
:10B9B000002864D1484629F083F88246F86020F0D8
:10B9C00025FD0AF5807383424DD98049012021F07D
:10B9D000A1F8B9F80E30A3F500739BB2A9F80E30A8
:10B9E000B9F80E3003F4F05313B9484626F0A0FF1F
:10B9F000204626F06BFA824608B9002C58D1314611
:10BA00002046FCF753FC002C40F0D2800024704DFF
:10BA100070496868224629F0E9FC32466E49686838
:10BA200029F0E4FC5CB1E389A3F500739BB2E381E8
:10BA3000E38903F4F05313B9204626F079FF3B68FD
:10BA40000BB10DF051FB40460DF076FC3B6843B363
:10BA50000DF004FD0DF070FC23E043F4006388E773
:10BA600043F4805393E70AF1070323F00703ADEB98
:10BA7000030DE84652464146484629F011F8112385
:10BA80004146BA893B7207F10800FFF735FF80464F
:10BA90000DF052FC9DE746B132465049032021F09B
:10BAA00039F81437BD46BDE8F08F4FF000089FE726
:10BAB000204626F003FA7860002868D0E38903F571
:10BAC00000739BB2E3812B6823F47F0323F40043CC
:10BAD000214607F10C002B6025F077FFD346F8686C
:10BAE00050B9BAF1000F92D0BBF1010F8FDD2B6876
:10BAF00043F400432B608AE728F054FB814626F08C
:10BB0000E5F910B9B9F1000F1ED131464846FCF7EE
:10BB1000CDFB8246F86810B1514628F06DF9BAF1B4
:10BB2000000F0ED0BAF80E30A3F500739BB2AAF83E
:10BB30000E30BAF80E3003F4F05313B9504626F025
:10BB4000F7FED7F804A009E0484626F0B7F9002828
:10BB5000F7D1484626F096F90028F2D10BF1010BF7
:10BB6000B9F1000F0ED0B9F80E30A3F500739BB2F7
:10BB7000A9F80E30B9F80E3003F4F05313B9484663
:10BB800026F0D6FE07F10C0025F00AFFA7E72046B5
:10BB900026F078F900283FF439AFE38903F5007304
:10BBA0009BB2E3812B6823F47F0323F40043A1E7D6
:10BBB00004462CE748C20020E0CC0500B22C00204F
:10BBC000E9CC0500F5CC0500B0D5050025B505008C
:10BBD000682D0020FFCC050009CD05004BCB0500EA
:10BBE00072DF7047F0B5264B264983B0044600AF9C
:10BBF0000246586829F0FAFB204626F05FF9E8B1C2
:10BC00000023391D20467B6027F056FD054668BBA2
:10BC1000204628F055FF0646786020F0F7FB06F531
:10BC20008073834217D91849012020F073FF174908
:10BC3000032020F06FFF0C37BD46F0BD204626F0F4
:10BC400021F90028DCD1002CF5D022461049032030
:10BC500020F060FFEFE7F31D23F00703ADEB030DCA
:10BC60006D4632462946204628F01AFF00213B79CE
:10BC70002A460846FFF7B4FF0DF05EFBDBE700BF86
:10BC8000682D00209ECD050025B50500A7CD050037
:10BC9000D3CD050070B5384C38492068002228F013
:10BCA00073FD054678B1002101200DF0F3F9EB8911
:10BCB000A3F500739BB2EB81EB8903F4F05313B946
:10BCC000284626F035FE00222D49206828F05CFD2C
:10BCD000054670B101200EF035FCEB89A3F5007329
:10BCE0009BB2EB81EB8903F4F05313B9284626F09D
:10BCF0001FFE00222349606828F046FD0022054609
:10BD00002149606828F040FD064605B918B1314662
:10BD10002846FFF7F3FD2846314628F067F9002250
:10BD20001A49606828F030FD054668B111F0FCF949
:10BD3000EB89A3F500739BB2EB81EB8903F4F0531D
:10BD400013B9284626F0F4FD60681149002228F056
:10BD50001BFD044678B1FFF745FFE389A3F50073A7
:10BD60009BB2E381E38903F4F05323B92046BDE895
:10BD7000704026F0DDBD70BD682D002093CD05001C
:10BD8000C0C90500FFCC050009CD0500BFCE0500E8
:10BD90009ECD05002DE9F043C38903F5007391B0F2
:10BDA0009BB20446C38103A88846154617F02CFCB5
:10BDB00090B301212E4816F041FF064648B31FFA02
:10BDC00088F026F05AFD2B490246204628F0A3FCB5
:10BDD00000222949204628F0D7FCDDF82690009063
:10BDE00007461FFA88F30022294603A8C8470028FF
:10BDF00016DA2249042020F08DFE012026F035FDC0
:10BE00001F490246204628F086FC3146384628F075
:10BE1000EDF803A817F08AFB204611B0BDE8F083C7
:10BE2000013026F02AFD17490246204628F073FC0F
:10BE3000022D17D10121144816F000FF05460028F5
:10BE4000E3D0214628F058FBEB89A3F500739BB2A1
:10BE5000EB81EB8903F4F053002BD6D1284626F072
:10BE600067FDD2E72146304628F046FBCDE700BF0C
:10BE70008CD40500BCD5050074D00500A4D4050001
:10BE8000BDD40500C4D40500C9D4050013B5C389C9
:10BE9000019003F500739BB20C46C3810E4928F054
:10BEA00019FC022221460198FFF774FF50B1C389A3
:10BEB000A3F500739BB2C381C38903F4F0530BB99C
:10BEC00026F036FD01980449012301AA1CF0B2FCBA
:10BED000019802B010BD00BF6CD005002DE9F047FD
:10BEE0008EB005468A46174626F01AF9814620B1DB
:10BEF00028460021FDF79EF80546284625F0E6FF76
:10BF0000044638B95748294621F036F920460EB084
:10BF1000BDE8F087BAF1000F07D0504625F0EEFFDC
:10BF2000044610B951465048EEE7022F16D101A839
:10BF300017F010FB90B100224C49284628F024FC51
:10BF400029F012F9DDF80D30834204DACDF80D0046
:10BF500001A817F0F9FA01A817F0E8FA01214448FE
:10BF600016F06CFE064600287AD0012F6DD14149AB
:10BF7000002020F0F9FE044690B9F389A3F5007380
:10BF80009BB2F381F38903F4F05313B9304626F0E2
:10BF9000CFFCB9F1000FB9D0002D39D12C46B5E74F
:10BFA0003549002020F0E0FEA046044644B339465F
:10BFB000204616F035FEBAF1000F10D02F4A514638
:10BFC000204628F098FD50B1C389A3F500739BB2B9
:10BFD000C381C38903F4F0530BB926F0A9FC2146B1
:10BFE000304628F089FAB8F1000F04D042462449BF
:10BFF000204628F06FFB2A462249204628F06AFB9B
:10C000003146404627F0F2FFB9F1000F0CD05DB188
:10C01000EB89A3F500739BB2EB81EB8903F4F0533A
:10C0200013B9284626F084FC002F7FF46FAF01A8D7
:10C0300017F0EAFA00283FF469AF01A8214616F08C
:10C040006BFB01A817F072FA60E7022F0CBF0E49D4
:10C050000E49002020F088FE4FF000080446A5E7B6
:10C060000446D1E7F8D305005AD4050028D40500CA
:10C0700037D405003ED4050046D4050081D4050020
:10C08000DBF3050074D005004ED4050053D4050041
:10C0900070B58EB0044601A80E4617F0B5FA18B96F
:10C0A000002420460EB070BD204625F00FFF58B189
:10C0B0001F4827F035FE1F4A01460546204628F056
:10C0C0000DFD294627F092FF304628F06BF8054613
:10C0D000F8B125F013FF80B92946174821F04CF834
:10C0E000EB89A3F500739BB2EB81EC8914F4F05457
:10C0F000D6D1284626F01CFCD3E7EB89A3F50073C4
:10C100009BB2EB81EB8903F4F05313B9284626F078
:10C110000FFC204601223146FFF7E0FE044618B12D
:10C12000014601A816F0ECFC01A817F0FFF9B8E7EA
:10C130009CD50500A0D505005AD4050070B58EB079
:10C1400004460D4601466846164617F079FD48B389
:10C150003EB140F2FF339D42A8BF1D46012DB8BF3E
:10C160000125BDF9143002330FD10F49204629F0C3
:10C1700023F90E49204629F01FF90D49204629F0E0
:10C180001BF90C49204629F017F96846ADF8145000
:10C1900017F01CFDE38903F500739BB2E381204691
:10C1A0000EB070BD0446FAE74FD3050054D3050026
:10C1B00059D305005ED305002DE9F04D2DED028B1E
:10C1C00090B004460E46014602A890461F469DF8D0
:10C1D000685017F035FD002800F09980304629F0AE
:10C1E00049FC4046B0EE408AF0EE608A29F042FCFD
:10C1F00038465BEC10AB29F03DFC8DED000BB8F13F
:10C20000000F7ED0002F7CD00022424B51EC180B47
:10C210002EF09CFB2EF04AFE00223E4B074659466C
:10C2200050462EF093FB2EF041FE9DED000B0022B8
:10C23000384B064651EC100B2EF088FB2EF036FEE4
:10C24000BDF80D2012F4607287F3080386F3080628
:10C2500080F3080008D0B2F5C07F29D020D8802A0A
:10C260002AD0B2F5807F2CD09DF81320102A2FD130
:10C27000D910B210C90241EA421141EAE000002D92
:10C2800043D0059002A817F0A1FCE38903F50073E1
:10C290009BB2E381204610B0BDEC028BBDE8F08D6F
:10C2A000B2F5007F11D0B2F5207FDDD1324601E03A
:10C2B0001A463346064606E01A46034630461646F8
:10C2C000D2E71A4603461046CEE71A463346F6E74B
:10C2D000202A06D11A0442EA0622104340F07F4089
:10C2E000CDE7182A04D1190441EA06210843C6E71C
:10C2F00033441844B0F5C07F4FF0FF30B8BF002082
:10C30000BDE7304627F086FFB9E70690BAE7044656
:10C31000C0E700BF0000704010B58EB00C4601466B
:10C32000684617F08DFC40B1BDF80530DB0648BF0C
:10C3300084F001041CB1BDF809000EB010BDBDF8B9
:10C340000700FAE72DE9F04F97B00546014608A827
:10C3500017F076FC28B94FF00009484617B0BDE841
:10C36000F08F00F0ABF904460028F4D000212846F5
:10C37000FFF7D2FF012107462846FFF7CDFF05460C
:10C3800038469DF82B6026F078FA3D490246204653
:10C3900028F0C1F9284626F070FA3A4902462046AC
:10C3A00028F0B9F9012E07D0304626F066FA364952
:10C3B0000246204628F0AFF905FB07F0704307302E
:10C3C0000021C01027F046FC814668B9E389A3F537
:10C3D00000739BB2E381E38903F4F053002BBAD1DD
:10C3E000204626F0A5FAB8E70146002203A825F06A
:10C3F000D3FD0025A846AB46AA46DDE903129142CB
:10C4000013D3069850B1C389A3F500739BB2C381BF
:10C41000C38903F4F0530BB926F08AFA4A461B4944
:10C42000204628F078F9A14697E70FFA8BF20FFA29
:10C430008AF108A817F096FB0AF1010A08FA06F833
:10C44000574548EA000806EB050203DC0BF1010B37
:10C450004FF0000A15460AE0083D28FA05F1C9B276
:10C4600003A8019225F024FC019A4FEA1828072D11
:10C47000F2D8D5086FF0070303FB0525BDE700BF21
:10C480005CD2050048D3050062D20500C3F905005F
:10C490002DE9F74F21F00045894616461F464FF01B
:10C4A000FF32414B2946804604462EF0E9FC002825
:10C4B00076D14FF0FF323C4B404629462EF0D6FC59
:10C4C00000286DD132463B46304639462EF0D8FC26
:10C4D000002865D100220023404649462EF0A8FCE2
:10C4E00028B309F1004500220023304639462EF0DA
:10C4F0009FFC10B107F100431F4600220023304685
:10C5000039462EF08BFC78B94FF0FF32264B30467F
:10C5100039462EF097FC38B14FF0FF32224B2046BF
:10C5200029462EF08FFCE8B90024002522E04D4674
:10C53000D9E700221D4B204629462EF007FACDE907
:10C540000001B246BB4652465B46DDE900012EF0D3
:10C5500083FC52465B46E0B9204629462EF03EF861
:10C5600004460D4622462B46304639462EF06AFCDC
:10C570000028DED100220023404649462EF058FC18
:10C5800010B105F100431D462046294603B0BDE821
:10C59000F08F104619462EF023F882468B46D2E7DC
:10C5A0000024034DF0E700BFFFFFEF7F0000E03FF6
:10C5B0000000F87F2DE9F84355EC114B11EE100AFD
:10C5C000294657EC106B2EF071FC0928804619D8CB
:10C5D0002EF052F922462B462EF020FC90B1B8F1F5
:10C5E000000F63D030463946B8F1010F03D141EC5A
:10C5F000100BBDE8F88332463B462EF0A7F908F150
:10C60000FF38F1E700220023304639462EF010FCB7
:10C610000022D8B3284B20462946FFF739FF0022D5
:10C6200000232EF0FBFBF0B300224FF080432046A6
:10C630002946FFF72DFF002200232EF0EFFBB04626
:10C6400007F1004949EC108B68B12CF0CDF9224676
:10C650002B4651EC100B2EF079F9BDE8F84341EC74
:10C66000100B2CF03DB92CF0BFF922462B4651ECB3
:10C67000100B2EF06BF941EC100B2CF031F953EC50
:10C68000102B10EE100A03F10041B0E700233046F2
:10C6900039462EF0C3FB30B1002200232046294644
:10C6A0002EF0D0FB28B147EC106BCEE700200249FA
:10C6B0009DE7002000219AE70000F03F052025F0CB
:10C6C000E1BFFFF7FBBFFFF7F9BF2DE9F8430F46C6
:10C6D0009046814618B1067A0025AE4201D8BDE8E1
:10C6E000F883D9F80030D9F8040033F8353018440D
:10C6F00027F016FB044601464046B8475CB1E38983
:10C70000A3F500739BB2E381E38903F4F05313B9FB
:10C71000204626F00DF90135DFE728F093BE000032
:10C720000022014920F07EBC50B6050010B5044639
:10C7300030B902460549032020F0ECF9204610BD2F
:10C74000C38903F500739BB2C381F7E72EF105009F
:10C75000024B03495868052228F016B8682D0020BE
:10C76000D0ED0500F8B5051E0C4606DC2949012070
:10C7700020F0D0F900242046F8BD084625F0A6FB9D
:10C780000646A8B100222449204627F0FDFF28F0E4
:10C79000A8FE002221490646204627F0F5FF28F092
:10C7A000E3FC30F0080309D0102809D01C49DEE76B
:10C7B00024B122461B49012020F0ACF9012400E0FD
:10C7C00002242946204626F06EF907469EB12946E6
:10C7D000204626F068F905461349002020F0C4FAE7
:10C7E000044610B10FB146B13DB92A46394620463C
:10C7F00027F0D0FBBEE73546EEE73A460B49204628
:10C8000027F089FF002DB6D02A460949204627F097
:10C8100082FFB0E780F605009FF60500BEF6050032
:10C82000ACF60500C3F60500FAF60500C3F90500ED
:10C8300003F7050070B50D1E064606DA0B49012008
:10C8400020F068F90024204670BD1B2025F01AFF57
:10C85000044615F1FF35F6D31FF0D0FD0028F2D1C4
:10C860003146204626F09AFDF3E700BF6CF605003E
:10C8700038B5044625F02AFBD8B100220E492046DF
:10C8800027F082FF054625F04BFC10B1284626F024
:10C89000B6FE04465DB1EB89A3F500739BB2EB8154
:10C8A000EB8903F4F05313B9284626F041F82046EB
:10C8B00038BD0446FBE700BF33F60500F8B5064671
:10C8C0000F46144625F02CFC0546E8B1204625F01D
:10C8D00039FBD8B1204627F09DFC0546384628F0A4
:10C8E0005BFE044626F08BFE2D1A13D500255CB1A5
:10C8F000E389A3F500739BB2E381E38903F4F0536A
:10C9000013B9204626F014F82846F8BD304626F024
:10C9100076FEE2E7204626F072FE2F18304626F01B
:10C920006EFE8742E2D82A46012321463046F3F7BD
:10C9300033FFB0FA80F56D09D9E7F8B507460D4623
:10C94000164625F0EDFB044698B1284628F024FE53
:10C95000002E05460FDA00245DB1EB89A3F50073C4
:10C960009BB2EB81EB8903F4F05313B9284625F011
:10C97000DFFF2046F8BD26F042FE8419384626F037
:10C980003EFE8442E7D80123324629463846F3F773
:10C9900003FFB0FA80F46409DEE7F0B587B028F051
:10C9A000FBFD0546002842D00146002201A825F0E3
:10C9B000F3FA4FF0FF340027DDE901639E4225D3EF
:10C9C000049850B1C389A3F500739BB2C381C38996
:10C9D00003F4F0530BB925F0ABFFA742DABFE21B1B
:10C9E000013200223946284626F0DDFCEB89A3F50A
:10C9F00000739BB2EB81EB8903F4F053044613B947
:10CA0000284625F095FF204607B0F0BD059800B1F7
:10CA1000805D20F04EFD30B9039B1E4437EA2407A9
:10CA200028BF3746344601A825F038F8C4E7044645
:10CA3000E9E7000070B5002286B00E461D4927F0D8
:10CA4000A3FE044625F06CFB0546B0B1002221464A
:10CA500001A825F0A1FA0025DDE9013293421CD39B
:10CA6000049850B1C389A3F500739BB2C381C389F5
:10CA700003F4F0530BB925F05BFF5CB1E389A3F538
:10CA800000739BB2E381E38903F4F05313B92046AA
:10CA900025F04EFF284606B070BD059800B1C05C79
:10CAA000864214BF284645F00100C5B201A824F013
:10CAB000F5FFD1E728F40500F8B506460D460AB3A0
:10CAC000104627F0A7FB002D044603DA304626F077
:10CAD00096FD0544002C03DA304626F090FD044410
:10CAE0001B2025F0CFFD25EAE57524EAE47407460E
:10CAF00030B1A54204DA631B2A46314626F010FC09
:10CB00003846F8BD00296FF00044E9DADEE7F8B5F1
:10CB100005460C46C2B1104627F07CFB20EAE076C1
:10CB2000002C05DA284626F06AFD044424EAE47461
:10CB30001B2025F0A7FD074620B133462246294693
:10CB400026F0EEFB3846F8BD6FF00046E8E7F8B592
:10CB500007460C46CAB1104627F05CFB20EAE07598
:10CB600024EAE474A542B8BF23464FF01B00BCBFC3
:10CB70002C461D4625F086FD064620B12B1B22467D
:10CB8000394626F0CDFB3046F8BD6FF00040E5E7B2
:10CB900008B508B1036823B91B20BDE8084025F09B
:10CBA00071BD002127F026FBBDE8084028F022BE19
:10CBB00070B5044625F08AF910B90024204670BDEE
:10CBC00000222949204627F0DFFD064625F07EF9A0
:10CBD000002837D000222549304627F0D5FD0546EC
:10CBE00025F08CF908B35EB1F389A3F500739BB20D
:10CBF000F381F38903F4F05313B9304625F098FE1E
:10CC0000002D2ED02C681A4BE31A5C425C41002D9B
:10CC1000D4D0EB89A3F500739BB2EB81EB8903F4CD
:10CC2000F053002BCAD1284618E05DB1EB89A3F57B
:10CC300000739BB2EB81EB8903F4F05313B92846E0
:10CC400025F076FE002EB8D0F389A3F500739BB2D1
:10CC5000F381F48914F4F054AFD1304625F068FE26
:10CC6000ACE72C46D3E700BF50B60500A4FC050096
:10CC7000ED17030008B526F032FB08BD70B5054678
:10CC800086B01B200E4625F0FDFC044630B3284636
:10CC900025F046FA10B3002E20DB3246294601A8C3
:10CCA00025F07AF9DDE901239A420AD2059B03B106
:10CCB0009B5C8DF8033001220DF10301204626F024
:10CCC000D9FB049850B1C389A3F500739BB2C3810B
:10CCD000C38903F4F0530BB925F02AFE204606B0B1
:10CCE00070BD37B505461B2025F0CCFC044628B1A5
:10CCF000294601A824F069FE019810B9204603B026
:10CD000030BD27F04FFA28F02FFA01228DF80300EA
:10CD10000DF10301204626F0ADFB01A824F040FEF2
:10CD2000EAE7000070B506460D4625F0F9F904461D
:10CD300030B93246134903201FF0ECFE204670BD87
:10CD40001149002020F010F832461049044627F01F
:10CD5000C1FC45B1284625F0E3F968B932460949D6
:10CD600003201FF0D7FE002025F087FD084902466A
:10CD7000204627F0D0FCE1E72A460649204627F066
:10CD8000A9FCF0E7ECF305005AB6050017F405001E
:10CD90001EF4050028F4050038B5002208490546B0
:10CDA00027F0F2FC044640B906491FF0DDFF0449B4
:10CDB00004460246284627F08DFC204638BD00BFB9
:10CDC000EA2F0600DFF3050070B505460E4625F094
:10CDD0007DF858B9284625F03FF8044630B92A4670
:10CDE0000E4903201FF096FE204670BD304625F008
:10CDF0006DF818B10A4901201FF08CFEFFF75EFCA8
:10CE000004460028F0D0284625F060F80028EBD032
:10CE10002A460449204627F05DFCE5E734EE05008C
:10CE200067EE050050B60500F8B507460E4625F03A
:10CE30004DF800283CD000221E49384627F0A4FCBB
:10CE4000044625F06DF970B3204626F0D8FB002E7D
:10CE500001DD864206D31749384628F0ADFA25464B
:10CE60002846F8BD32460021204626F09CFA6FF095
:10CE7000004231460546204626F095FA0D49024605
:10CE8000384627F048FC002CEAD0E389A3F500736C
:10CE90009BB2E381E38903F4F053002BE0D12046F9
:10CEA00025F046FDDCE71B2025F0ECFB0546EAE714
:10CEB0000546D5E733F6050038B50C46054651F86A
:10CEC000043B9847002DA2BFA3690133A36100284A
:10CED0000BDB04F11C05C1B2284624F02EFD2846C8
:10CEE00024F022FE63690133636138BD2DE9F04F00
:10CEF00093B000AF0E46154681461BF001FD4FF082
:10CF0000010A044607F11701304687F817A0F4F725
:10CF100059FB002D804606DC4FF0000840464C3798
:10CF2000BD46BDE8F08F1FF071FA05F580738342AE
:10CF300004D95F4950461FF0EDFDEDE7EB1D23F0EE
:10CF40000703ADEB030D132C6E463BD1594B1B78F9
:10CF5000CBB1002307F120024FF040215648C7F81B
:10CF60002230C7F826307B8587F820A087F82180FB
:10CF700087F822507E62F7F72FFF024618B14F491B
:10CF800004201FF0C7FD2946012025F08CFD8046B6
:10CF90000028C1D00146002207F1200026F07CF8CD
:10CFA000354416F8011B07F1200024F0C6FC07F1F8
:10CFB000200024F0B9FDB542F3D107F1200024F0A0
:10CFC00093FCABE7002CA7D13D492246484627F009
:10CFD000DBFB8246014607F118001AF00FFE00281D
:10CFE00059D022463749484627F0CEFB28F079FA37
:10CFF0003B7FB877FF2B4ED07A7FFF2A4BD0F97D4D
:10D0000087F8212087F82030BA6987F822002E4B54
:10D0100093FBF2F307F12000012BD8BF2346F96000
:10D020007B621EF063FD4FEA480101F4FF7141F09D
:10D03000010107F120001EF011FD05F1FF38A8EBFA
:10D0400004035942594108224FF0000B07F1200018
:10D05000C7E901121EF0AAFCBA6879684FEA4B0BC7
:10D06000013A40EA0B0BF1D107F120001EF0CCFC95
:10D07000012197F821000DF055FE06F804B00134A7
:10D08000A542DCD1FB681BB107F120001EF0FAFCC1
:10D0900097F82230BB77B87F25F0E7FB09490246B5
:10D0A000484627F017FB514626F0A0FF6BE700BF6C
:10D0B000CEEC050040C20020F4BA002003ED0500CC
:10D0C00016ED05001FED050090D003002DE9F04F8F
:10D0D00089B000AF0D46924680461BF011FC4FF020
:10D0E000010BF91D0446284687F807B0F4F76AFAE1
:10D0F0000023064607F108015046BB6026F0DCFA23
:10D100000546F0B9504627F0DBFC8146B8601FF0B9
:10D110007DF909F58073834207D9454958461FF0C8
:10D12000F9FC2437BD46BDE8F08F09F1070323F071
:10D130000703ADEB030D6D464A462946504627F0DE
:10D14000AFFCBB68002BECD0132C1DD1394A1278F0
:10D15000002AE6D0F9793848BD61002291427A610F
:10D16000FA61BB754FF0402114BF1346202307F12D
:10D1700014027E75F7F730FE02460028D1D02F4901
:10D1800004201FF0C7FCCCE7002CCAD12C49224652
:10D19000404627F0F9FA8146014607F10C001AF0E3
:10D1A0002DFD90B322462749404627F0EDFA28F09E
:10D1B00098F93B7CB874FF2B27D07A7CFF2A24D0C7
:10D1C0007A753B75B875FA681F4B93FBF2F307F15C
:10D1D0001400012BD8BF2346D7F808B097F807A052
:10D1E000BB611EF083FC710001F4FF7107F11400B4
:10D1F0001EF034FCA34514DCBAF1000F03D007F194
:10D2000014001EF03FFCBB7DBB74B87C25F02DFBE9
:10D210000C490246404627F05DFA494626F0E6FEF4
:10D220007FE7295D07F114001EF018FC0134E1E7E7
:10D2300025B5050040C20020F4BA002073ED0500BA
:10D2400016ED05001FED050090D003002DE9F04F0D
:10D2500089B0894600901BF053FB4946044602A85A
:10D260001AF0CCFC40B3132C40F002819DF80C4026
:10D2700020461BF059FC9DF80D5018B128461BF0B4
:10D2800053FCE0B9224629468A481FF075FFB9F1E0
:10D29000000F00F00A81884A0098494627F01EFCDA
:10D2A00050B1C389A3F500739BB2C381C38903F452
:10D2B000F0530BB925F03CFB09B0BDE8F08F7F4976
:10D2C000029E7F4B04EB840405EB85050C440D4462
:10D2D0009E4294F801806F7858DD7A4B9E42D4BF0D
:10D2E0004FF080664FF0CD66774A784C13785BB389
:10D2F00023681BB1764B1021C3F880104FF04023F8
:10D300004FF0FF31C3F80813D3F800120021C3F81F
:10D310000012C3F80015012184F8221094F8271098
:10D3200079B9D3F808154FF0A04001F5E07140F24B
:10D33000023540F82150D3F80C3503F5E07340F87E
:10D340002350002384F8223094F8223001251570F0
:10D35000FBB108225F4904201FF0DCFB9DF80C4064
:10D3600020461BF0E1FB20B14FF4207120460DF068
:10D37000C5FD9DF80D4020461BF0D6FB002886D049
:10D380004FF4945120460DF0B9FD80E74FF0CC7674
:10D39000AAE79DF81E2084F827209DF81D20A36091
:10D3A000C4E9003384F8253084F8243072B34FEA9E
:10D3B0008800B90000F1A04001F1A04140F20C62E8
:10D3C0004FF0A04BC0F8002705FA08FAC1F8002773
:10D3D000BD4040F20D620193CBF808A5CBF808558B
:10D3E000C0F80027C1F800270420F5F7ABF9019B2E
:10D3F000DBF810150D422BD043B14FF0A04A0420AA
:10D40000CAF80C55F5F79EF9CAF808554FF0A04335
:10D4100008F5E07140F20C6243F8212007F5E07155
:10D4200043F821204FF040231D46C3F80885C3F878
:10D430000C75C3F8246522681AB106210420F7F799
:10D4400025FF0523C5F80035022384F8223085E73F
:10D4500001930420CBF80CA5F5F774F9CBF808A5D7
:10D460000420F5F76FF9019B0133092BC0D1C4E704
:10D47000002C7FF40CAF9DF80C00FF2807D0012191
:10D480000DF050FC03219DF80C000DF059FE9DF8A5
:10D490000D00FF283FF4FBAE01210DF043FC0321FA
:10D4A0009DF80D000DF04CFEF1E60349009827F0C1
:10D4B00083FF01E727ED050016ED050094B6050092
:10D4C00097AB020087F5040040C20020F4BA0020A8
:10D4D00000E100E056ED0500F0B58DB00D461646B2
:10D4E0001C461BF00DFA12289DF8487005D02E49F5
:10D4F00001201FF00FFB0DB0F0BD16B90CB90F24C1
:10D5000003262A4B1B78F6B2E4B25BB92849ADF882
:10D5100010306FF0FF02CDE9011201A8254A0392F5
:10D520000DF00AFDFF2F03D0002138461CF0E2F970
:10D53000284624F007FD70B1284626F06BFE2246EF
:10D540003146C0B2F3F732FFFF2FD4D00121384665
:10D550001CF0D0F9CFE7284624F00DFEE8B1802377
:10D5600083F311880122294601A825F0D8FD01A8DE
:10D5700020F0CBF8054601A825B920F073F885F313
:10D580001188E1E727F004FE22463146C0B2F3F7E6
:10D590000DFF01A820F093F8E9E72A46064901208B
:10D5A0001FF0B8FAD0E700BFD9F5050032C200205D
:10D5B000A08601000001080001F60500F0B58DB05D
:10D5C0000D4616461C461BF09BF912289DF8487024
:10D5D00005D02F4901201FF09DFA0DB0F0BD16B9FE
:10D5E0000CB9032401262B4B1B7806F00F0604F020
:10D5F0000F045BB92849ADF810306FF0FF02CDE998
:10D60000011201A8254A03920DF096FCFF2F03D0CA
:10D61000002138461CF06EF9284624F093FC70B1C6
:10D62000284626F0F7FD22463146C0B2F3F77EFECB
:10D63000FF2FD2D0012138461CF05CF9CDE72846F7
:10D6400024F099FDE8B1802383F311880122294653
:10D6500001A825F064FD01A820F057F8054601A8AF
:10D6600025B91FF0FFFF85F31188E1E727F090FD52
:10D6700022463146C0B2F3F759FE01A820F01FF848
:10D68000E9E72A46064901201FF044FAD0E700BF27
:10D69000B1F5050032C20020A0860100000108009B
:10D6A00001F6050013B50C461BF02AF98DF80700AA
:10D6B0000938052805D80DF107020349204627F04F
:10D6C0008FF802B010BD00BFEDDA020010B50C46B5
:10D6D0001BF0A2F92146BDE810401CF00BB908B5BB
:10D6E0001BF09AF90021BDE808401CF003B908B509
:10D6F0001BF092F90121BDE808401CF0FBB870B5A1
:10D7000086B00E4602AA01A91BF006F960B16EB9F7
:10D71000FF2502AA0199304627F062F8FF2D03D0B9
:10D72000012128461CF0E6F806B070BD31680029DA
:10D73000EEDD0139304626F05DFD044624F0DEFDC5
:10D7400030B320461BF068F90546304627F0E2FD6D
:10D7500050B1C389A3F500739BB2C381C38903F49D
:10D76000F0530BB925F0E4F85CB1E389A3F500733D
:10D770009BB2E381E38903F4F05313B9204625F00B
:10D78000D7F8FF2DC5D0002128461CF0B3F8C0E71C
:10D79000002CBDD0FF25E8E72DE9F04198B00E46FA
:10D7A000174607A908AA1BF0B7F8002800F0A780C1
:10D7B000FF2F03D0002138461CF09CF8304624F09F
:10D7C000C1FB80463046B8F1000F1AD026F022FD8A
:10D7D00008A920EAE070079B9847002804DA08A906
:10D7E0004FF0FF30079B984725F047F80446FF2F7E
:10D7F00003D0012138461CF07DF8204618B0BDE862
:10D80000F08124F08DFC0546002850D01B2024F028
:10D8100039FF31460446424602A824F0BDFB464685
:10D82000DDE902239A4218D30598002832D14645F3
:10D83000DDDD1EF0E3FD0028D9D108A9079B4FF0DC
:10D84000FF30984701228DF807000DF107012046AF
:10D8500008F1010825F00EFEE9E71EF0CFFD0028D3
:10D86000E2D1069808B1029BC05C079B08A99847C3
:10D87000002806F1010609DB8DF8070001220DF1F1
:10D880000701204608F1010825F0F4FD02A824F064
:10D8900005F9C5E7C389A3F500739BB2C381C389AA
:10D8A00003F4F053002BC2D125F042F8BFE7304615
:10D8B00027F006F90146012025F0F5F80446002876
:10D8C00095D001462A460EA8CDE90C5525F0E4FB7B
:10D8D00007AA0C49304626F083FFDDE90C239A4263
:10D8E00003DB0EA824F000F881E71EF087FD002876
:10D8F000F7D107A94FF0FF30FFF7DEFAEDE7044656
:10D900007BE700BFB9CE02007FB50C4605461AF092
:10D91000F7FF21460646684619F03AFFB0B1122ECD
:10D9200016D168460DF008FB54B3184A2146284624
:10D9300027F0D4F850B1C389A3F500739BB2C3811B
:10D94000C38903F4F0530BB924F0F2FF04B070BDA7
:10D95000002EFBD19DF80500FF2802D001210DF01B
:10D96000EFFB9DF80600FF2802D004210DF0E8FB34
:10D970009DF80700FF28D7D001210DF0E1FBD3E788
:10D980000249284627F018FDE0E700BF16ED050024
:10D99000F2F7CFBF28F090BFF0B589B024F058FF60
:10D9A000044638B310224FF4D82500210DEB0200B5
:10D9B0000095F1F7B7FD04A9284628F005FEC8B187
:10D9C00001AD06AE0027059B01330CD196E803009C
:10D9D00085E8030028468DF80C7026F0A1F9014671
:10D9E000204626F0ABFD002204A9684628F03EFE42
:10D9F0000028E8D1204609B0F0BDF7B50746084633
:10DA00000C4616461D4624F061FA00B3002220465B
:10DA1000114609F061FC002504462E46384628F0E0
:10DA200087FF009533462246F3F73AF805465CB186
:10DA3000E389A3F500739BB2E381E38903F4F05318
:10DA400013B9204624F074FF284603B0F0BD002C23
:10DA5000E4D0E28902F5007292B2E281DEE738B5E5
:10DA600028F066FF28F068FE044688B1002125F002
:10DA70005DFEE389A3F500739BB2E381E38903F4C0
:10DA8000F053054613B9204624F052FF284638BD0E
:10DA90000546FBE708B528F04BFFBDE8084028F035
:10DAA0004BBE38B528F044FF28F046FE044680B14E
:10DAB00004F0BEFFE389A3F500739BB2E381E38921
:10DAC00003F4F053054613B9204624F031FF2846ED
:10DAD00038BD0546FBE708B528F02AFFBDE8084039
:10DAE00028F037BE4FF4D82028F05ABE0B78C1B2C8
:10DAF00018461AF07DBC00002DE9F04389B01F469E
:10DB000080460C4691461AF0FBFEA0F10903DBB2F9
:10DB1000052B06463AD80E280FD1374B1B7863B930
:10DB20004FF0FF324FF41651CDE9041204A8334AE6
:10DB300006928DF81C30F7F7CFFB314D8DF8006061
:10DB4000B9F1000F03D0204627F026FD04466A46AF
:10DB50002946204626F044FEB9F1000F0CD05CB1F6
:10DB6000E389A3F500739BB2E381E38903F4F053E7
:10DB700013B9204624F0DCFE2FB169460D20A847DA
:10DB800069460A20A84709B0BDE8F0830028FAD109
:10DB900002461C49404626F0F7FD324605461A4922
:10DBA000404626F0F1FD0DF11008064602462946D2
:10DBB000404619F01BFF5EB1F389A3F500739BB2D9
:10DBC000F381F38903F4F05313B9304624F0B0FE27
:10DBD0005DB1EB89A3F500739BB2EB81EB8903F494
:10DBE000F05313B9284624F0A3FE98E80F006D46C1
:10DBF00007C52B70054DA3E741C2002008000100B6
:10DC00003D9A0400A0EB050016ED0500498B0400C9
:10DC100000231A46FFF770BF01231A46FFF76CBFB7
:10DC200000230122FFF768BFF0B585B004461AF063
:10DC300067FE002205463C49204626F0A5FD064623
:10DC400028B93A4901201EF065FF05B0F0BD002259
:10DC50003749204626F098FD324601460746684679
:10DC600019F0C4FE3946304626F0C0F93049204646
:10DC700027F0A2FB2C49204627F09EFBA5F10903C3
:10DC8000DBB2052B44D900222A49204626F07CFD30
:10DC900008B327F069FAC4B2002120460CF0E0FE78
:10DCA000002019F037FE0546A8B1214624F0C4FF34
:10DCB000044618B10146284627F0A6FA284625F062
:10DCC000EFF820B91C4B1D49586827F075FB294611
:10DCD000204626F08BF99DF80600FF2802D000218F
:10DCE0000DF02EFA9DF80700FF2802D000210DF05C
:10DCF00027FA9DF80400FF2802D000210DF020FA39
:10DD00009DF80500FF28A0D000210DF019FA9CE72E
:10DD1000A5F10D03DBB2012BDDD8FF22002128463F
:10DD20001AF08EFFD7E700BF16ED05007CF5050061
:10DD3000A0EB0500A3F50500682D0020A8F505005F
:10DD4000F0B585B005460F4614461AF0D9FD0646D3
:10DD5000D4B922465B49284626F016FD04462246E1
:10DD60003946684619F042FEA0B95CB1E389A3F5D3
:10DD700000739BB2E381E38903F4F05313B92046A7
:10DD800024F0D6FD05B0F0BDE38903F500739BB226
:10DD9000E381E4E7009824F070FD4B4902462846F1
:10DDA00026F0B9FC7CB122464649284626F0B3FC51
:10DDB000A6F10903DBB2052B0AD80E2EE2D1684684
:10DDC000F7F78AFADEE73F49284627F0F5FAEFE74A
:10DDD000002ED7D19DF80500FF2807D001210DF0B6
:10DDE000AFF901219DF805001BF084FD9DF80400AA
:10DDF000FF280BD005210DF0A3F9602024F0BCFB17
:10DE0000044660B9314901201EF084FE9DF80630B9
:10DE1000FF2BB7D02E4901201EF07CFEB2E7024650
:10DE20002C49284626F077FC204624F0ADF8002641
:10DE300080F8406004460CF08FFF009B9DF80A209C
:10DE400084F85860C4E914369DF8083013449DF8EE
:10DE50000920B24218BF0133C4E9120184F85930D5
:10DE600001219DF804000CF0FBFD044610B324F0E2
:10DE700004FD19490246284626F04DFC012019F000
:10DE800049FD06460028C1D02A46214626F0AEFBB1
:10DE9000F389A3F500739BB2F381F38903F4F05384
:10DEA00013B9304624F044FD013C0C4B0C4A43F8B6
:10DEB0002420ABE79DF804200A4901201EF02AFE29
:10DEC000A4E700BF16ED0500A0EB0500F7F4050080
:10DED00054F505001DF50500A3F5050060C20020FE
:10DEE0003179040025F5050010B50C461AF008FD3F
:10DEF000A0F10903DBB2052B04D82146BDE8104090
:10DF00001BF0B0BF02490120BDE810401EF002BE68
:10DF1000CCF405002DE9F3471F46012313600C697B
:10DF20000646894615460CB10B68E45C30782E280D
:10DF300000F0E3805B282CD101237B7296F801A0CE
:10DF4000BAF15E0F02D12B6801332B604FF000084D
:10DF50000CE03B4601AA4946FFF7DCFF2B68019A1B
:10DF600048EA000813445FFA88F82B602B68F45CD9
:10DF7000F018002C00F0C3805D2CEAD101332B6037
:10DF800000237B72BAF15E0F14BF444688F001048F
:10DF90000BE05C2866D102232B607078642808D1DE
:10DFA000303C092C8CBF00240124204602B0BDE87F
:10DFB000F087442805D1303C092C94BF002401246B
:10DFC000F3E7662864D06E2864D0722864D0732882
:10DFD00005D1204602B0BDE8F0471FF06ABA5328C9
:10DFE00006D120461FF065FA80F00100C4B2DCE7DC
:10DFF000742853D0762853D077280DD1A4F130035C
:10E00000092B7AD920461FF048FA002875D15F2CD9
:10E0100014BF00240124C8E757280CD1A4F1300311
:10E02000092B66D920461FF038FA002861D15F3CE1
:10E0300018BF0124B9E7A0F13003DBB2092B31D9B5
:10E0400078280FD1B3786BB1F3785BB104232B60E0
:10E05000B0781FF0C1F98046F0781FF0BDF940EAB2
:10E060000810C0B27B7AFBB12B68F35C2D2B1BD15F
:10E0700078812868013028603B4601AA494630442F
:10E08000FFF748FF2B68019A134404462B608CE786
:10E090000C20E7E70A20E5E70D20E3E70920E1E7A8
:10E0A0000B20DFE71846DDE73A7A62B1A4F14103BD
:10E0B000192B98BF2034A0F1410398BFE4B2192B6B
:10E0C0009CBF2030C0B2B7F90A30B3F5807F12D0C0
:10E0D000DBB22AB1A3F14102192A9CBF2033DBB283
:10E0E0004FF480729C427A8103D3844201D89842D3
:10E0F00063E7002459E784428AE7012455E702498F
:10E1000001201EF007FD50E7A1F7050082B02DE9C0
:10E11000F047B2B00C463AA9064681E80C001EF062
:10E120006DF930B10025284632B0BDE8F04702B0A5
:10E13000704733780BB17C2B5AD158223AA91CA8CE
:10E140002DF018F9DDE93A67DDF8F48024F080FB62
:10E15000A26823681A440546D21B3946304625F08A
:10E1600022F9002104460246284626F03FFA5CB117
:10E17000E389A3F500739BB2E381E38903F4F053D1
:10E1800013B9204624F0D4FB0DF1800A4FF00009AA
:10E19000C1450DDB384624F070FB91490246284604
:10E1A00026F0B9FA32468F49284626F093FABAE7A4
:10E1B0005AF8041BDAF820203046521A25F0F3F8FA
:10E1C00009F10109044602464946284626F00EFA9E
:10E1D000002CDDD0E389A3F500739BB2E381E389D2
:10E1E00003F4F053002BD3D1204624F0A1FBCFE75A
:10E1F0005E2B09D12368A268D34293D11EF052FF4F
:10E2000000288FD0013607E0242B1DD1D4E900323D
:10E210009A4206F101060CD850223CA968462DF01E
:10E22000A9F83AAB0CCB21463046FFF76FFF054605
:10E2300079E74C223DA968462DF09CF83AAB0ECB0D
:10E24000304600F0FAFAF2E7282B0FD13D9B216807
:10E25000A2683AA80A44191D082B40F8212000EBB7
:10E2600083014A63CADC01333D93C7E7292B0AD1F6
:10E270003D9B002BC2DD3AAA02EB83032168A26812
:10E280000A441A63BAE73AAB1BAA21463046FFF7A5
:10E2900041FE1B9FF35DA3F12A02012A804606EB93
:10E2A000070500F284800137374450B92B2B08D181
:10E2B0004C223DA968462DF05DF83AAB0ECB3846AE
:10E2C000BFE7214614A814AD23F04AFB0FCD0DF192
:10E2D000700CACE80F0050222B68CCF800303CA941
:10E2E00068462DF047F83AAB0CCB1CA93846FFF72F
:10E2F0000DFF05461F9850B1C389A3F500739BB26B
:10E30000C381C38903F4F0530BB924F011FBD4E9A2
:10E3100000239A42BFF407AFB8F1000F3FF403AFF8
:10E32000204623F0BBFB3AAB1BAA21463046FFF741
:10E33000F1FD2146804614A823F012FB0DF1500E8A
:10E34000BEE80F000DF1700CACE80F005022DEF8B3
:10E350000030CCF800303CA968462DF00BF83AAB01
:10E360000CCB1CA93846FFF7D1FE81461F9850B14F
:10E37000C389A3F500739BB2C381C38903F4F0532F
:10E380000BB924F0D5FAB9F1000F0ED05DB1EB89CD
:10E39000A3F500739BB2EB81EB8903F4F05313B93F
:10E3A000284624F0C5FA4D46B1E7A946FBE7D4E973
:10E3B00000239A420BD250B1204623F06FFB1EF08F
:10E3C00071FE00283FF4AEAE1B9B1E4424E74C2296
:10E3D0003DA968462CF0CEFF3AAB0ECB284630E77D
:10E3E000C3F70500C9F705002DE9F047BAB080462C
:10E3F000084614AF27F0D0F800228349054640466E
:10E4000026F0C2F926F0B0FE00228049824640463E
:10E4100026F0BAF9064623F083FE044640B9314699
:10E42000284625F0E3FD20469837BD46BDE8F08735
:10E43000304625F0E4F800F1080323F00703ADEBC4
:10E44000030D0DF15009421C4946304627F07EFA73
:10E450005EB1F389A3F500739BB2F381F38903F4F2
:10E46000F05313B9304624F063FA69214046FEF7B1
:10E47000E1FA4FF48072002387F84800A7F84A2099
:10E480002946524607F1180087F84930FB643D647D
:10E4900023F082FD07F11801384623F061FABC46EB
:10E4A000BCE80F0007F12C040FC45022DCF8003048
:10E4B000236007F148016846C7F844A02CF05AFFD2
:10E4C00007F140030CCB07F12C014846FFF71EFE75
:10E4D0000446B86B564650B1C389A3F500739BB28E
:10E4E000C381C38903F4F0530BB924F021FA07F177
:10E4F000180023F0D3FA07F1400A1CB9D7E9062324
:10E500009A4229D3786A50B1C389A3F500739BB2AC
:10E51000C381C38903F4F0530BB924F009FA5DB148
:10E52000EB89A3F500739BB2EB81EB8903F4F05305
:10E5300013B9284624F0FCF9002C3DD1022024F028
:10E54000A1F800250446284624F097F92E490246F2
:10E55000404626F0E0F866E707F11801384623F058
:10E56000FFF9BC46BCE80F0007F12C040FC40136CC
:10E57000DCF800302360502207F1480168467E64D1
:10E580002CF0F8FE9AE80C0007F12C014846FFF742
:10E59000BDFD0446B86B50B1C389A3F500739BB2AF
:10E5A000C381C38903F4F0530BB924F0C1F907F117
:10E5B000180023F073FAA0E767214046FEF73AFA05
:10E5C00000B30021204625F015FE00221049064622
:10E5D000204626F0D9F826F0C7FD0546304625F03E
:10E5E0000EF80544002EAED0F389A3F500739BB25C
:10E5F000F381F38903F4F053002BA4D1304624F0C7
:10E6000097F9A0E705469EE71EF4050017F40500FC
:10E61000C3F705002DE9F84F05460E4623F080FDAF
:10E6200020B94FF000084046BDE8F88F24F010F9FB
:10E6300080460028F5D01EB9294625F05DFFF2E797
:10E640003046F2F7D1FB002800F08180002024F052
:10E6500014F96A490246304626F05DF829463046EC
:10E66000FFF7C2FE0027044684B1204623F0F4FBE6
:10E67000814618B3E389A3F500739BB2E381E38974
:10E6800003F4F05313B9204624F052F9002024F08B
:10E69000F4F85A490246304626F03DF8284624F060
:10E6A000AEFFB842BFD339466FF00042284624F08F
:10E6B0007AFE0146404625F041FFB4E74946204630
:10E6C00025F098FD4A464E498246204626F05CF8E1
:10E6D00026F04AFD8146504624F091FF8346BAF168
:10E6E000000F0ED0BAF80E20A2F5007292B2AAF86E
:10E6F0000E20BAF80E2002F4F05212B9504624F05F
:10E7000017F9A9EB07023946284624F04CFE0146CA
:10E71000404625F013FFE389A3F500739BB2E38124
:10E72000E38903F4F05309EB0B0713B9204624F0F7
:10E73000FFF8384624F0A1F830490246304625F06B
:10E74000EAFF29463046FFF74FFE04468CE7304685
:10E7500026F022FF064698B124F051FF8146284654
:10E7600024F04DFF002700F1010BABEB090A3C46FA
:10E77000544531DCB9F1000F1CD1C4B90134F7E7BD
:10E780008146ECE75C461FE00146404625F0B4FEBA
:10E79000FB89A3F500739BB2FB81FB8903F4F05363
:10E7A00013B9384624F0C4F804EB0907E6E75445EA
:10E7B0000AD111E05445E5D00123224631462846CE
:10E7C000F1F7EAFF0028D9D1E21B3946284624F0A8
:10E7D000EAFD07460028D7D1002E3FF424AFF38985
:10E7E000A3F500739BB2F381F38903F4F053002B7C
:10E7F0007FF419AF304624F09BF814E71EF40500AF
:10E80000C3F7050038B5FFF7EFFD054620B123F04B
:10E8100023FB80F00100C0B200F001045DB1EB8980
:10E82000A3F500739BB2EB81EB8903F4F05313B9AA
:10E83000284624F07DF8204638BD84B0F0B59BB062
:10E8400021AE054686E80E001EF02CFC68B9044691
:10E8500020461BB0BDE8F04004B070475C2C03D1EB
:10E860006C78002CF4D03D4601352C78002CEFD08C
:10E870007C2C05F10107F1D1DDE9211215A823F067
:10E880008BFB502223A968462CF074FD96E80C00FF
:10E8900015A93846FFF73AFC044618980028D7D047
:10E8A000C389A3F500739BB2C381C38903F4F053FA
:10E8B000002BCDD124F03CF8CAE70000F7B506469E
:10E8C00008460D46144623F019FB30B92A46334951
:10E8D00003201EF01FF903B0F0BD6CB300223049D5
:10E8E000304625F0ABFE0090C0B125F05FFC01235F
:10E8F00000906A460020294619F04EFF0098002833
:10E90000E9D0C389A3F500739BB2C381C38903F423
:10E91000F053002BDFD124F00BF8DCE7214F00226D
:10E920003946304625F030FF044638B92A46394684
:10E93000304625F0CFFECEE71B4FF0E723F0BEFABE
:10E9400078B12946204625F0D7FDE389A3F5007369
:10E950009BB2E381E38903F4F053002BBBD1204643
:10E96000D9E702216846CDE9004525F02CFE39465D
:10E9700005460246304625F0ADFE002DE5D0EB8978
:10E98000A3F500739BB2EB81EB8903F4F053002BEA
:10E99000DBD1284623F0CCFFD7E700BF4EEB0500C4
:10E9A00072EB050044EB050049EB050010B50022B1
:10E9B0000446FFF783FF2046BDE81040FEF7ECB9A0
:10E9C00038B5154601220446FFF778FF25B100222D
:10E9D00029462046FFF772FF2046BDE83840FEF783
:10E9E000DBB900002DE9F04F85B0054623F0C3FBED
:10E9F000044640B92A46484903201EF08BF82046B9
:10EA000005B0BDE8F08F454900201EF0ADF9044681
:10EA10000028F4D048F20801414823F00FFF0646D1
:10EA20000028ECD022463F49DFF8F8B025F052FE2E
:10EA300023F00EFF2946824603A822F0C6FF4FF0BE
:10EA4000000847460398D8B9A7EB080023F015FF44
:10EA500035490246204625F05EFE5246334920469F
:10EA600025F059FEF389A3F500739BB2F381F38976
:10EA700003F4F053002BC2D1304623F059FFBEE718
:10EA800025F090FB0546FEF793F800283BD048F2AE
:10EA90006001274823F0D2FE8146384623F0EDFE80
:10EAA000002102460190484626F092FA019B5BB194
:10EAB000DA89A2F5007292B2DA81DA8902F4F052B0
:10EAC00012B9184623F034FF22465946484625F02D
:10EAD00001FE494632462846FFF772FF494625F0B7
:10EAE00085FA5DB1EB89A3F500739BB2EB81EB89ED
:10EAF00003F4F05313B9284623F01AFF03A8013793
:10EB000022F04EFF9EE72A463946504625F06EFD1C
:10EB100008F10108E5E700BFAFF30500DFF30500EA
:10EB200041EC02008ECD0500D4F30500DAF30500B8
:10EB300081EB020037B5054601910F4848F2080104
:10EB400023F07CFE0446A8B12A460C4925F0C2FDFC
:10EB5000012301AA2146284619F01EFEE389A3F5E8
:10EB600000739BB2E381E38903F4F05313B92046A9
:10EB700023F0DEFE03B030BDFBEE02008ECD0500BB
:10EB80002DE9F0410F46904618490022064625F02F
:10EB9000FBFD26F0E9FA002205461549304625F02E
:10EBA000F3FD0446F8B142463946013D25F01EFD0D
:10EBB000284623F062FE0D490246304625F0ABFDA3
:10EBC0001DB921463046FFF7B5FFE389A3F5007371
:10EBD0009BB2E381E38903F4F05323B92046BDE8F7
:10EBE000F04123F0A5BEBDE8F08100BFD4F30500DD
:10EBF000DAF3050037B5054601910F4848F20801E0
:10EC000023F01CFE0446A8B12A460C4925F062FDFB
:10EC1000012301AA2146284619F0BEFDE389A3F588
:10EC200000739BB2E381E38903F4F05313B92046E8
:10EC300023F07EFE03B030BDF5EE02008ECD050060
:10EC400038B500220D460D49044625F09DFDA0B1C2
:10EC5000C389A3F500739BB2C381C38903F4F05346
:10EC60000BB923F065FE2046044926F0A5FB294692
:10EC70002046BDE83840FFF7BDBF38BDDAF30500D8
:10EC80002DE9FF41064610460191144623F016F97E
:10EC90000746002852D0214603A822F096FE002401
:10ECA000039810BB4549304626F086FB4449304660
:10ECB00026F082FB00224349304625F065FD41499C
:10ECC0000546304626F078FB1DF046FB80460028BE
:10ECD0003ED001462846FFF78DFF2A462146404692
:10ECE00025F058F904B0BDE8F08125F05BFA01ABDE
:10ECF0000122314605461FF0EDFFEFB950B1C28940
:10ED0000A2F5007292B2C281C38903F4F0530BB929
:10ED100023F00EFE5DB1EB89A3F500739BB2EB818E
:10ED2000EB8903F4F05313B9284623F001FE03A83E
:10ED300022F036FE0027B3E70446EBE7002CB1D003
:10ED4000204601AB012231461FF0C4FF0446A9E76B
:10ED50004DB32046FDF72CFF50B348F208011A4886
:10ED600023F06CFD48F208010646184823F066FDC2
:10ED70000746A6B198B12A461549304625F0AAFCA7
:10ED80002A461349384625F0A5FC01223146204683
:10ED9000FFF794FD424639462046FFF78FFD39467E
:10EDA000304625F023F92946204625F01FF999E73A
:10EDB00021462846FFF7BEFEF5E700BF44EB0500FD
:10EDC00049EB0500EA2F060035EB0200F5EB0200E7
:10EDD0008ECD0500414B2DE9F047B2F100080E46FB
:10EDE0004FF000023E493F4F054608BF1F4625F041
:10EDF000CBFC044668B1C389A3F500739BB2C38101
:10EE0000C38903F4F053002B66D1BDE8F04723F02B
:10EE10008FBD012023F029FD31490246284625F007
:10EE20007AFC22463946284625F0AEFC04460028E6
:10EE30004ED102462C49DFF8B090284625F0A4FCBC
:10EE40000446CCB9B8F1000F3BD0324627492846DA
:10EE500025F040FC002C3FD0224631462846FFF7E3
:10EE60000FFFE389A3F500739BB2E381E38903F409
:10EE7000F0538BBB2046C8E700223946204625F0D8
:10EE800083FC8246024648B131462046FFF7F8FE31
:10EE900021465046BDE8F04725F0A8B8494620462F
:10EEA00025F072FCE389A3F500739BB2E381E3894B
:10EEB00003F4F053824613B9204623F039FD54463B
:10EEC000BFE732460A490120BDE8F0471DF022BEE7
:10EED000B8F1000FC0D0B8E7BDE8F08749EB0500F6
:10EEE0007BEB050044EB0500EA2F060072EB050002
:10EEF00080EB05000022FFF76DBF0122FFF76ABF1C
:10EF00002DE9F74F0BF028FF8946074623F076FAE4
:10EF100083460BF021FF80468A46FDF7CFFB04466F
:10EF2000002800F0A580554B55495868002225F06F
:10EF30002BFC0546002800F09F8023F0A5FFEB89FD
:10EF4000A3F500739BB2EB81EB8903F4F053064603
:10EF500013B9284623F0ECFC4A49002501235A1E28
:10EF600012018818B0F80EC01CF03F0F0DD0CDE98B
:10EF7000003223F000F80135009B424928B1019A84
:10EF80008A580F32120913441544013340F6CA025D
:10EF90009342E4D9B018AB1B401B009323F06DFCE7
:10EFA00039490246204625F0B6FB009B184623F05F
:10EFB00064FC36490246204625F0ADFB40F6CA0007
:10EFC00023F05BFC32490246204625F0A4FB304684
:10EFD00023F053FC2A490246204625F09CFB584664
:10EFE00023F04BFC2B490246204625F094FBB8EB5E
:10EFF00007006AEB09012BF07BFC0022264B2BF06B
:10F00000A5FC264B00222BF0A1FC41EC100B23F0B9
:10F0100022FC23490246204625F07DFB214823F0AF
:10F020002CFC21490246204625F075FB002023F0E8
:10F0300024FC1E490246204625F06DFB1C4823F0A7
:10F040001CFC1C490246204625F065FB4FF4D820E5
:10F0500023F013FC18490246204625F05CFB4FF4D0
:10F06000002023F00AFC15490246204625F053FBF8
:10F07000204603B0BDE8F08F06466DE7682D0020FE
:10F0800041F30500882D002049F305004EF30500EB
:10F0900054F305005AF3050000408F400000B03ED5
:10F0A0005DF3050048CF002064F3050074F305000C
:10F0B0001C67060080F3050091F30500A2F305002C
:10F0C00010B5FDF7FBFA0446294824F029FE29492A
:10F0D0000246204625F01FFB274824F021FE274941
:10F0E0000246204625F017FB254824F019FE254945
:10F0F0000246204625F00FFB4FF4002023F0BDFB15
:10F1000021490246204625F006FB4FF4803023F0CB
:10F11000B4FB1E490246204625F0FDFA04F052FEDB
:10F120001B490246204625F0F6FA1A4B1B78093B8C
:10F13000DBB20A2B96BF184A184852F8230024F075
:10F14000EFFD17490246204625F0E5FA154824F060
:10F15000E7FD15490246204625F0DDFA134823F065
:10F160008CFB13490246204625F0D5FA204610BDF7
:10F17000ABF20500B4F20500BCF20500C4F20500D4
:10F18000CFF20500D6F20500DCF20500DD0706002F
:10F19000E2F20500B82C002018EB0500A4310600AF
:10F1A000E9F20500F1F2050033F30500BC2C002064
:10F1B0003BF3050038B50849054600201DF0D4FD95
:10F1C000044638B1284623F060FB04490246204635
:10F1D00025F0A1FA204638BD4AF1050051F7050097
:10F1E00010B519F019FC044619F09EFC20B1204618
:10F1F000BDE8104023F049BB10BD2DE9F74F0D4687
:10F2000003210446CDE900230BF09AFF4FF0000BD9
:10F210004FF0010A4FF08008D94615F1FF3502D2B0
:10F2200003B0BDE8F08F009B0AEA0306019B0BEADE
:10F23000030756EA070316D088F3118800212046F9
:10F240000BF070FD0A2009F00BFD012120460BF0A8
:10F2500069FD89F31188372009F002FD1AEB0A0ACB
:10F260004BEB0B0BD9E788F31188002120460BF0FC
:10F2700059FD412009F0F4FC012120460BF052FD1C
:10F2800089F311880520E7E710B40C7802460023C3
:10F29000204608215DF8044BFFF7AFBF2DE9F84386
:10F2A0000D46032107460BF04BFF002401264FF0CB
:10F2B0008008A14615F1FF3502D22046BDE8F8834B
:10F2C00088F31188002138460BF02CFD032009F04B
:10F2D000C7FC012138460BF025FD0A2009F0C0FCCF
:10F2E00038460BF00BFD00B1344389F3118835200B
:10F2F00009F0B6FC7600DDE710B5032104460BF0FB
:10F300001FFF002120460BF00DFD4FF4FA7009F0AD
:10F31000A7FC012120460BF005FD502009F0A0FCC0
:10F3200020460BF0EBFC04464FF4D27009F098FC39
:10F3300084F00100C0B210BD08B50022034925F0D9
:10F3400023FABDE8084019F0C3BB00BF51F7050020
:10F350002DE9F04F8BB00C46FFF7EEFF064619F093
:10F36000E3FB28B94FF0000840460BB0BDE8F08F32
:10F3700023F06EFA80460028F4D0631EFF2B28BFCE
:10F38000F0242246E317CDE900234FF00009304670
:10F39000FFF7B2FF0028E7D0DDE90023082130465F
:10F3A000FFF72BFF01240025AA46274601213046FE
:10F3B000FFF774FF01215FFA80FB3046FFF76EFF15
:10F3C000BBF1010FC0B22BD101283AD1402FCBDDC8
:10F3D0009DF80C30002BC7D005AC0DF10C090025B1
:10F3E000A34619F8017B38091DF01AF8207007F0C0
:10F3F0000F001DF015F80135082D607004F10204AE
:10F40000EFD1002358468DF8243024F089FC0146C2
:10F41000404625F093F8D146BAF1000FA4D0B6E7E4
:10F420000AAB2B44834513F81C3C2DD14F4524DAFD
:10F430001C4214BF4FF0010B4FF0000BBBF1000F4B
:10F4400021D00AAB2B444FF0010B13F81C3C234393
:10F450000AAA2A44012102F81C3C30465A460023DD
:10F460006400FFF7CAFE14F0FF0404BF0135012455
:10F47000072D07F1010799DDA8E70CBF4FF0010B3D
:10F480004FF0000BDAE7BA4623EA0403E0E770B571
:10F490008AB00C46FFF750FF064619F045FB68B3EB
:10F4A000204622F04FFD18B3204624F0B3FE01465B
:10F4B0000546012023F0F7FA044650B10146002228
:10F4C000684623F0E9FD15F1FF3505D2684622F0C4
:10F4D0000BFA20460AB070BD08213046FFF7DEFE69
:10F4E000C1B2684622F029FA684622F01DFBEAE71D
:10F4F00008213046FFF7D2FE23F0BFF90446E8E7C3
:10F5000037B50D461446FFF717FF8DF8070019F0C1
:10F510000BFB80B10DF107020C49284625F060F97C
:10F520009DF807004CB101210BF0FCFB01219DF877
:10F5300007000BF005FE03B030BD04210BF000FE08
:10F5400001219DF807000BF0EDFBF4E789F20200C2
:10F5500010B5FFF7F1FE044619F0E6FA38B120467F
:10F56000CC2200230821BDE81040FFF746BE10BDA5
:10F570002DE9F04786B00C46FFF7DEFE074619F08E
:10F58000D3FA40B1204622F0CBFD38B922463049AB
:10F5900003201DF0BFFA06B0BDE8F087204624F036
:10F5A0002EF81028F2D13846FFF7A6FE2146002299
:10F5B00001A822F0F1FC0024A146A046A246059B2A
:10F5C0000BB1019A9B5C8DF8003001A822F066FA1D
:10F5D000059B0BB1019A9B5C8DF8013001A822F0CC
:10F5E0005DFA00231A46102168468DF802A01DF02E
:10F5F0006BFFA4F12002C4F12003A14000FA02F243
:10F6000020FA03F31143A0401943083440EA0906E5
:10F6100041EA0805402CB146A846D0D1049850B123
:10F62000C389A3F500739BB2C381C38903F4F0536C
:10F630000BB923F07DF93846552200230821FFF746
:10F64000DCFD32462B4640213846FFF7D6FDA2E7C7
:10F6500052F1050010B5FFF76FFE044619F064FA89
:10F6600020B12046BDE81040FFF746BE10BD73B57F
:10F6700023F0EEF80646A8B1FDF76AF8054688B112
:10F68000014601A822F0A1F9019C74B9EB89A3F508
:10F6900000739BB2EB81EB8903F4F05313B9284656
:10F6A00023F046F9304602B070BDE38903F50073DC
:10F6B0009BB20022E3811146204625F0FDFB014666
:10F6C000304624F03BFFE389A3F500739BB2E3814E
:10F6D000E38903F4F05313B9204623F029F901A874
:10F6E00022F05EF9D0E710B1012125F015BA70477C
:10F6F0002DE9F74305460F46904622F0FFFB0446EE
:10F7000040B92A466E4903201DF004FA204603B092
:10F71000BDE8F083284622F0A7FB002835D0A98851
:10F72000286823F08BF804460028EFD02946684665
:10F7300022F04BF9009E002E37D0F38903F50073B9
:10F740009BB2F381304624F02DFD8146304622F0F5
:10F750003BFD20B3B9F1000F33D00121304625F035
:10F76000DBF9054678B10146204624F017FEEB8907
:10F77000A3F500739BB2EB81EB8903F4F05313B94B
:10F78000284623F0D5F801250AE0284622F0ADFBF3
:10F79000002814BF0820072022F074FFC3E70546A5
:10F7A0004946304624F022FC6DB9B8F1000F0ED165
:10F7B000009D002D57D13A464249204624F08AFF49
:10F7C000A4E74D46ECE7684622F0EAF8B2E7414686
:10F7D00001A822F0FAF801980028E9D024F0E2FC10
:10F7E000009D0646A5B1EB8903F500739BB2EB8142
:10F7F000284622F0E9FC88B9EB89A3F500739BB297
:10F80000EB81EB8903F4F05313B9284623F090F809
:10F8100032460021204625F0DBFB13E001220021C7
:10F82000284625F049FB3146804624F0E5FA41465A
:10F83000204624F0B3FD2846414624F0D7FB684615
:10F8400022F0AEF85EB1F389A3F500739BB2F381A9
:10F85000F38903F4F05313B9304623F069F801A893
:10F8600022F09EF8B7E7EB8903F500739BB2012203
:10F87000EB811146284625F01FFB064678B101466C
:10F88000204624F08BFDF389A3F500739BB2F3812E
:10F89000F38903F4F05313B9304623F049F8EB89A8
:10F8A000A3F500739BB2EB81EB8903F4F05313B91A
:10F8B000284623F03DF8684622F072F878E700BF4A
:10F8C00054EC05008ECD05002DE9F04F8FB0814638
:10F8D00002AF10468A46164622F04DFC0446002828
:10F8E0005ED0304623F0BFFE4028834680460AD9CA
:10F8F0000246304901201DF00DF90024204634371E
:10F90000BD46BDE8F08F8300DA1D22F00702ADEBA3
:10F91000020D02AD2A462B440021934219D1012247
:10F920003146381D23F0FBFB381D1DF0EEFE98B963
:10F93000381D1DF097FE00231946CDE9008552467B
:10F9400048461EF0DDFC29460446404624F0D0FA25
:10F95000D4E742F8041BE0E7381D24F049F90446D7
:10F9600022F0D5FC58B1204624F054FC061E06DBDC
:10F97000B34504DD381D24F0C3FC45F826005CB116
:10F98000E389A3F500739BB2E381E38903F4F053A9
:10F9900013B9204622F0CCFF381D1DF090FEC3E7BE
:10F9A0002EB13246044901201DF0B4F8A6E7B04656
:10F9B0003546C0E7D1EB050019EC050010B5FCF7A2
:10F9C000C7FE044678B125F01BFDE389A3F500735B
:10F9D0009BB2E381E38903F4F05323B92046BDE8E9
:10F9E000104022F0A5BF10BD2DE9F347044608469C
:10F9F0000D4622F083FA30B9564903201DF08AF8EB
:10FA000002B0BDE8F087204622F02EFA06462846CE
:10FA100022F02AFA864208D0284622F025FAE38905
:10FA2000002855D043F04003E381204622F05DFAE0
:10FA30000646284622F059FA86420BD0284622F084
:10FA400054FAE3899BB223F03F03002845D043F0EA
:10FA50000803E38100224049DFF8FC90DFF8FCA0B6
:10FA6000204624F0EBFD00223C490746204624F0C6
:10FA7000E5FD0646204625F0C3FC294601A821F0F5
:10FA8000A4FF019D65BB7FB13946204624F086FC6A
:10FA9000FB89A3F500739BB2FB81FB8903F4F05350
:10FAA00013B9384622F044FF002EA9D03146204633
:10FAB00024F074FCF389A3F500739BB2F381F389FE
:10FAC00003F4F053002B9BD1304622F031FF97E72F
:10FAD00023F040031B041B0CA6E743F00703B8E721
:10FAE000EB8903F500739BB201A8EB8121F058FF6D
:10FAF0004946284623F082FAE8B95146284623F0C1
:10FB00007DFAC0B90121284625F006F8804690B15B
:10FB10000146204624F042FCB8F80E30A3F50073ED
:10FB20009BB2A8F80E30B8F80E3003F4F05313B9B6
:10FB3000404622F0FDFEEB89A3F500739BB2EB81FA
:10FB4000EB8903F4F053002B9BD1284622F0F0FE02
:10FB500097E700BF8BEC0500C9EC0500342C0600CC
:10FB600070B5064622F0DCFA28B91B490120BDE831
:10FB700070401CF0CFBFFCF7EBFD054650B30022F0
:10FB8000314625F0FFF8044690B93246134901206A
:10FB90001CF0C0FFEB89A3F500739BB2EB81EB89EE
:10FBA00003F4F053B3B92846BDE8704022F0C0BE5C
:10FBB0000146284625F028FBE389A3F500739BB294
:10FBC000E381E38903F4F053002BE3D1204622F0D4
:10FBD000AFFEDFE770BD00BFD8ED050006EE050003
:10FBE0002DE9F74305460F46914622F0AFFB30B9A9
:10FBF000464903201CF08EFF03B0BDE8F083384671
:10FC000022F08EFA08B94249F3E7484622F076F925
:10FC100028B9484622F084FA08B93E49E9E739464E
:10FC20003D4823F0D1FB04460028E5D001460122DF
:10FC3000284625F0A7F8E389A3F500739BB2E3817A
:10FC4000E38903F4F053064613B9204622F070FE10
:10FC5000304624F0A7FA8046002830D14946304685
:10FC600024F0CAF83146404624F0C0F92B49384602
:10FC700023F0C4F90028BFD000222949284624F0E7
:10FC800083FD019022F04CFA48B126492846012311
:10FC900001AA18F0CFFD2249284625F08DFB0198D6
:10FCA0000028A9D0C389A3F500739BB2C381C3897F
:10FCB00003F4F053002B9FD122F03AFE9CE722F090
:10FCC000FDF820B14946404624F016FCCAE722F070
:10FCD000BFFD4146044624F00FFC4946204624F06F
:10FCE0000BFC2146304624F087F8002CBAD0E3897B
:10FCF000A3F500739BB2E381E38903F4F053002B77
:10FD0000B0D1204622F014FEACE700BFADEF0500F5
:10FD1000E4EF05001BF0050073F005005AD505005F
:10FD200033F6050079F00500F8B506460846144696
:10FD30001F4623F0F5FF39460546204622F07EFD9A
:10FD40002946044602463046FFF74AFF2946204628
:10FD5000BDE8F84024F04AB9F0B585B006460D4636
:10FD600022F0F4FA20B9304903201CF0D3FE2CE035
:10FD7000284622F0D5F950B329462C4823F024FB1D
:10FD8000054610B301460122304624F0FBFFEB8903
:10FD9000A3F500739BB2EB81EB8903F4F0530446A7
:10FDA00013B9284622F0C4FD7CB12146304625F027
:10FDB0002BFAE389A3F500739BB2E381E38903F493
:10FDC000F05313B9204622F0B3FD05B0F0BD4DBB92
:10FDD000314603A821F0F9FD154F039C002CF4D007
:10FDE000E38903F500739BB2E38103A821F0D8FDFA
:10FDF0000095002301223946204623F071F818B1FE
:10FE00002146304625F000FAE389A3F500739BB242
:10FE1000E381E38903F4F053002BDED1204622F086
:10FE200087FDDAE703499FE7ADEF050073F00500B2
:10FE300081F0050085F0050038B50546084623F039
:10FE40006FFF044688B101462846FFF785FFE38926
:10FE5000A3F500739BB2E381E38903F4F05323B964
:10FE60002046BDE8384022F063BD38BDF8B50746EE
:10FE70000C46164622F06AFA28B935490320BDE837
:10FE8000F8401CF047BE204622F04AF900285CD01A
:10FE90002146304823F098FA0546002857D00146FD
:10FEA0000122384624F06EFFEB89A3F500739BB264
:10FEB000EB81EB8903F4F053044613B9284622F092
:10FEC00037FD204624F06EF9054688B186421ED1E2
:10FED0002146384625F098F9EB89A3F500739BB2CB
:10FEE000EB81EB8903F4F05313B9284622F020FD8F
:10FEF0006CB3E389A3F500739BB2E381E38903F458
:10FF0000F05323BB2046BDE8F84022F011BD21F09C
:10FF1000D5FF0028E0D031460122284627F002FA1A
:10FF200006460028D8D00146284625F06DF9F38909
:10FF3000A3F500739BB2F381F38903F4F053002B14
:10FF4000CAD1304622F0F4FCC6E7034996E7F8BD73
:10FF5000ADEF050073F00500DAF005002DE9F04380
:10FF600087B000AF81460C461546E84622F0EEF910
:10FF700040B9354903201CF0CDFD1C37C546BD46B0
:10FF8000BDE8F083204622F0CBF808B92F49F1E70D
:10FF900021462F4823F018FA06460028EDD02946BE
:10FFA000381D21F012FD0024786830B1042C3FD1B7
:10FFB0002246284903201CF0ADFD786850B1C38962
:10FFC000A3F500739BB2C381C38903F4F0530BB94B
:10FFD00022F0AEFC00223146484624F0D3FE24F045
:10FFE000E5F8F389A3F500739BB2F381F38903F479
:10FFF000F053054613B9304622F09AFC95B12346DA
:020000023000CC
:1000000007F108022946484618F0C6FBEB89A3F51C
:1000100000739BB2EB81EB8903F4F05313B92846CC
:1000200022F086FC07F10801204623F061FFA4E7D7
:1000300024F0B8F807F1080343F82400381D21F034
:10004000AFFC0134B0E700BFADEF05003AEF0500AB
:1000500073F0050073EF0500F7B5014601A821F024
:10006000B4FC254F0026019820B324F09BF80446E9
:1000700000283CD021F0F0FE0546002839D120466A
:1000800021F024FF30BB2246394603201CF042FDFC
:100090000125E389A3F500739BB2E381E38903F4AF
:1000A000F05313B9204622F043FC01A821F078FC5C
:1000B000002DD8D0019850B1C389A3F500739BB22D
:1000C000C381C38903F4F0530BB922F031FC3046ED
:1000D00003B0F0BD36B9E38903F500739BB2E38149
:1000E0002646D6E72146304624F0A9FED1E705464C
:1000F000DBE70025CDE700BF1AEE050070B5054629
:100100000E4621F0FBFE10B30122164928461CF0D2
:1001100089FF044621F04CFEF8B92246124903201B
:100120001CF0F8FC5CB1E389A3F500739BB2E3819A
:10013000E38903F4F05313B9204622F0F9FB25B10B
:10014000EB8903F500739BB2EB81284670BD28460E
:1001500021F0BCFE0028D7D1DBE73146204623F052
:100160004BFEDFE750B605001DF105002DE9F84311
:1001700004460F46164621F0A9FE054640B9284917
:10018000224601201CF0C6FC2C462046BDE8F88320
:10019000304621F09BFE054610B932462149F0E772
:1001A000384626F039F900221F498146304624F0AE
:1001B000EBFA002207461D49304624F0E5FA804656
:1001C000AFB9A0B900221A49304624F0DDFA05463D
:1001D0002A464946204624F011FE2946484623F087
:1001E00005FFE38903F500739BB2E381CDE70620A9
:1001F00022F048FA054660B11FB13A460A4924F098
:1002000069FAB8F1000F04D042460849284624F0A4
:1002100061FA4146384623F0E9FE002DD8D1D1E7F6
:10022000E2EE05000BEF0500BC0606001B0506000C
:100230007AF6050073B504460D4621F047FE0646E2
:1002400040B91949224601201CF064FC344620467E
:1002500002B070BD284621F039FE064610B92A4684
:100260001249F0E7294601A821F0AFFB019D2DB905
:10027000E38903F500739BB2E381E8E7EB8903F5BB
:1002800000739BB2EB81284623F08CFF294606467B
:1002900002462046FFF76AFF3246294623F07AFEDF
:1002A00001A821F07DFBE1E78DEE0500B7EE05002A
:1002B000F0B5064689B0084626F0AEF80546304649
:1002C00022F044F8044600B300222946304624F0C8
:1002D00059FDD0B1C389A3F500739BB2C381C38913
:1002E00003F4F0530BB922F023FB5DB1EB89A3F5C6
:1002F00000739BB2EB81EB8903F4F05313B92846EA
:1003000022F016FB204609B0F0BD304621F0DEFD9C
:10031000044608B10024E8E7304616F093FF07468C
:100320000028F7D020226946284625F00FFB6A46B0
:100330003146384617F0EEF80028D6D0C389A3F529
:1003400000739BB2C381C38903F4F0530BB922F04D
:10035000EFFA0124C9E70000F8B507460C46FFF79D
:10036000A7FF10B900252846F8BD204626F054F80E
:1003700001220146054638461CF0C2FD04465DB127
:10038000EB89A3F500739BB2EB81EB8903F4F05387
:1003900013B9284622F0CCFA002CE3D0FCF78EF9F2
:1003A000054668B9E389A3F500739BB2E381E3894D
:1003B00003F4F053002BD5D1204622F0B9FAD2E74E
:1003C000204621F025FD0646384621F0A7FD0746C8
:1003D000012022F04AFA2D490246284624F09BF9D2
:1003E000002F4BD02046B84780F00100C0B200F08B
:1003F000010022F03AFA26490246284624F08BF9F9
:1004000086F00100C0B222F030FA224902462846A6
:1004100024F081F9204624F023FE064621F0C0FC9A
:1004200070B300221C49304624F0AEF91A49024646
:10043000284624F070F900221849304624F0A4F927
:1004400016490246284624F066F95EB1F389A3F501
:1004500000739BB2F381F38903F4F05313B9304670
:1004600022F066FAE389A3F500739BB2E381E38986
:1004700003F4F053002B7FF476AF9DE70120B6E73D
:10048000204623F08FFE06490246DBE78CEF05008D
:1004900095EF0500A0EF0500BC0606001B05060051
:1004A0007AF6050010B5142994B0A8BF14210C46A3
:1004B00025F0E0FA24EAE4740A2351EC100B0093CF
:1004C00002AA462301941BF0B3FF02A823F028FCE4
:1004D00014B010BD30B5044695B008460D4621F065
:1004E000EEFE48B3204621F02DFD28B3284623F028
:1004F00091FE831E222B05461ED8204621F0DFFEEA
:1005000060B1204623F086FE2B46012202A91CF092
:10051000B1F802A823F004FC15B030BD204625F048
:10052000A9FA4FF0FF33CDE9005302AA462351EC5C
:10053000100B1BF07DFFECE7204625F02DF8EBE7D4
:1005400010B5044621F0BAFC40B12CB90024204675
:10055000BDE8104022F091B92468F8E7204621F068
:1005600091FC08B16488F2E7204621F0D9FD20B162
:10057000204623F044F80446E9E7204621F0BEFC7B
:1005800090B1204623F0EEFF0028DFD0C389046835
:10059000A3F500739BB2C381C38903F4F053002B0E
:1005A000D5D122F0C5F9D2E710BD7FB5039021F077
:1005B0008DFC40B1039CE38903F500739BB2E3819A
:1005C000204604B070BD039821F078FC0028F1D1DA
:1005D000039821F093FC04460028EBD1039816F011
:1005E000E1FA18B9FCF76AF80446E9E71BF08CFD5C
:1005F00005460028F6D023F0D5FD03AB0193012377
:10060000009322462346294606461DF079FE3146D0
:100610000446284623F0EAFCD2E700000000000070
:1006200070B508B1036823B90020BDE8704022F01E
:1006300024B9002123F0DEFD044621F03FFC002810
:1006400046D00CB1236843B9002022F016F90546C4
:1006500034B9002D3DD0284670BD012B0ED00025A9
:10066000E389A3F500739BB2E381E38903F4F053BC
:10067000002BEED1204622F05BF9EAE7002120466C
:1006800023F0B8FD064621F04BFDB8B1304621F00D
:1006900064FD98B1002022F0F0F80546002EDFD06E
:1006A000F389A3F500739BB2F381F38903F4F0534C
:1006B000002BD5D1304622F03BF9D1E7304621F06E
:1006C000A1FD18B9304625F00FFDE6E70025E5E766
:1006D0002CB99FED0F0BBDE8704022F0BCB820464E
:1006E00021F0F4FB05460028B9D1204621F018FD81
:1006F00040B1204621F031FD20B1284622F0BDF85E
:100700000546ADE7204625F0EFFCF9E7AFF30080A2
:10071000000000000000F87F2DE9F04786B018F0D7
:100720007BF9824618F000FA20B90024204606B072
:10073000BDE8F087FBF7C2FF04460028F5D04FEA7A
:100740008A08394F08EB0A03FD18FB5C40338DF82B
:10075000043001A800238DF8053023F0E1FA334975
:100760000246204623F0D7FF687822F086F8304909
:100770000246204623F0CFFFAD788DB1FBF79EFFF8
:10078000814668B122F064F8064600283DD105F0A4
:100790001F0022F072F827490246204623F0BBFFD3
:1007A000FBF78CFF81460028C0D008EB0A003844D4
:1007B000B0F803601EB3FBF781FF0546F8B102AA4B
:1007C00008213046F0F77EFB02A823F0A9FA1A4967
:1007D0000246284623F09FFF06F00F0022F04DF856
:1007E00016490246284623F096FF02AA0321304606
:1007F000F0F768FB2A4602A9484623F08CFF4A46D8
:100800000F49204623F087FF90E7AB0606D501206D
:1008100022F033F80146304623F090FE3246094973
:10082000484623F078FFB2E794B60500BCD5050032
:1008300074F105007DF105000864060085F10500EE
:1008400088F1050078F1050038B518F0E5F805469F
:1008500018F06AF9044650B128460AF0F5F980F01C
:100860001000C0F300142146284619F043F8204632
:1008700038BD10B50C4618F0CFF821460022BDE86F
:10088000104002F0D5BB08B518F0C6F8BDE8084026
:1008900002F020BD1FB50C468DED000B18F0BCF822
:1008A0009DED000B8DF80F00002251EC100B0A4B50
:1008B0002AF04CF80022094B2AF048F80022064B97
:1008C0002AF06EF92AF0A2FB23460DF10F02F0F791
:1008D0008BFC04B010BD00BF00408F4000003041D1
:1008E00008B518F099F8BDE808401AF083BD00007B
:1008F00070B506460D4621F013FC28B91F490120AA
:10090000BDE870401CF006B9284621F009FC20B96A
:10091000284621F0F3FA0028F0D0FBF719FF04462F
:1009200050B328461AF082FD054690B93246144964
:1009300001201CF0EFF8E389A3F500739BB2E3817B
:10094000E38903F4F053BBB92046BDE8704021F0C1
:10095000EFBF02463146204624F050FAEB89A3F55A
:1009600000739BB2EB81EB8903F4F053002BE2D1CF
:10097000284621F0DDFFDEE770BD00BF87ED0500F2
:10098000B7ED050070B5A0B0054621F0C9FB0446DF
:1009900028B95C492A4603201CF0BCF80BE08022F1
:1009A0006946284624F0D2FF7F2807D956490320FC
:1009B0001CF0B0F80024204620B070BDFBF7C8FE44
:1009C00005460028F6D00022694623F037FE23F0C2
:1009D000EDFBEB89A3F500739BB2EB81EB8903F48C
:1009E000F053044613B9284621F0A2FF002CE2D1AF
:1009F000464968462AF0E6FC00286AD04449684621
:100A00002AF0E0FC00286CD0424968462AF0DAFC63
:100A1000002868D0404968462AF0D4FC002864D0F9
:100A20003E4968462AF0CEFC002860D03C49684622
:100A30002AF0C8FC00285CD03A4968462AF0C2FC7B
:100A4000002858D0384968462AF0BCFC002854D009
:100A5000364968462AF0B6FC002850D068462AF08D
:100A6000C3FC082803D96A463149012094E7684647
:100A700025F06DFF25F060FE05460028F3D01AF042
:100A8000D5FCEB89A3F500739BB2EB81EB8903F4F2
:100A9000F053064613B9284621F04AFF002EE2D053
:100AA0003446FBF755FE0546002884D022466946A9
:100AB00023F010FEEB89A3F500739BB2EB81EB8969
:100AC00003F4F053002B7FF476AF284621F030FF7B
:100AD00071E71848002121F0B1FE0028BED004467D
:100AE000DFE71548F6E71548F4E71548F2E715483B
:100AF000F0E71548EEE71548ECE71548EAE7154832
:100B0000E8E700BF2EF405005EF4050083F405005D
:100B100089F4050091F40500F12606009CF4050017
:100B2000A2F40500A7F40500B1F405002AF30500BE
:100B3000B8F40500F15C0400D95C0400D55C040045
:100B4000C95C0400BD5C0400B55C04009D5C04004D
:100B5000855C04007D5C040038B5164C164B1546C8
:100B6000002291420CBF2146194623F00DFE044697
:100B7000F0B15DB100232B7021F084F930B1A3886E
:100B800003F00F03022B04BF01232B70204622F039
:100B90005BFAE389A3F500739BB2E381E38903F475
:100BA000F053054613B9204621F0C2FE284638BD51
:100BB0000546FBE7C3F9050003F705000000000048
:100BC0002DE9F04F8FB0CDE900230D4600229C495E
:100BD000DDF860A09DF864B0044623F0D5FD24F054
:100BE00080FC30B1974901201BF094FF0FB0BDE8A5
:100BF000F08F284617F098FF08B99349F3E7DDE92D
:100C0000006323F000474FF0FF32904B30463946E7
:100C10002AF036F980B94FF0FF328C4B3046394616
:100C20002AF024F940B984A3D3E90023DDE90001C7
:100C30002AF0FEF8074608B18549D4E70AF08CF897
:100C4000CDE90201504621F041F90646002800F0A6
:100C500087803A467F49504623F096FD25F028FAD2
:100C600021F000490F464FF0FF32784B49460646C7
:100C70002AF006F900BB4FF0FF32744B304649466C
:100C80002AF0F4F8C0B900220023304639462AF091
:100C9000EDF888B10022704B3046394629F056FEF7
:100CA00000226E4B29F052FE00226B4B29F078FF98
:100CB0002AF0ACF9CDE9020100226949504623F03F
:100CC00063FD24F00EFC06464FF0000841460DF18E
:100CD000170220468DF81780FFF73EFF4246074671
:100CE00001212046FFF738FF9DF817308046002B82
:100CF0003FD0BBF1000F14BF4FF005094FF00609BC
:100D0000DDE900230020544929F04AFF0022534B1B
:100D100029F01CFE0022504B29F042FF2AF076F900
:100D200026B1B8F1000F14BF46463E46029B08901C
:100D30001818039B8DF8349043EB0101B9F1030FB0
:100D4000CDE9060102D0B9F1050F1AD1454B33F8B0
:100D50001530ADF8323013BB43481CF0EDF937E0E5
:100D6000BAF1000FB0D05246404901201BF0D2FE2C
:100D7000AAE7BBF1000F14BF4FF003094FF00409BD
:100D8000BEE709F00509B9F1040FE5D1384B05EBD1
:100D9000850213449B78002BDED08DF83250002F53
:100DA00047D0344BFB1A1B1101339BB2ADF82830EE
:100DB00026B1304BF61A36110136B6B206A8ADF898
:100DC0002A6017F0D3F906A816F0FCFF0028C3D05C
:100DD0004146384623F00AF9012021F046FD184922
:100DE0000246204623F097FC9DED000B21F033FDD9
:100DF00021490246204623F08EFC204B20495868AA
:100E0000032223F0C1FC054600283FF4EFAE214643
:100E100023F072FBEB89A3F500739BB2EB81EB89A6
:100E200003F4F053002B7FF4E1AE284621F080FD5F
:100E3000DCE63B46BAE700BFFCA9F1D24D62503F69
:100E4000D7D505002DF7050049F70500FFFFEF7F17
:100E500055F705005FF3050000408F40000030416A
:100E600075F7050080C200207CF70500C3F6050079
:100E700094B60500882D002097F70500682D002006
:100E80009CF705002DE9F04F684B694958688DB013
:100E9000002223F079FC0746A8B1014602A820F001
:100EA00094FDDFF8A8A1DFF8A8B1029878B9FB8912
:100EB000A3F500739BB2FB81FB8903F4F05313B9D4
:100EC000384621F035FD00200DB0BDE8F08F23F04D
:100ED00069F900225146044623F056FC24F001FB38
